:020000040800F2
:1000000030AE00209D0100083D3B0108BD250108E0
:10001000613801083536000839D6010800000000B3
:1000200000000000000000000000000061680108FE
:10003000C56D0008000000003144010891720108FC
:10004000B7010008B7010008B7010008B7010008B0
:10005000B7010008B7010008C96D0008B701000822
:10006000B7010008D56D0008E16D0008B701000870
:100070002568000835680008B7010008B7010008C6
:10008000B7010008B7010008B7010008B701000870
:100090003936000849360008B7010008ED6D000840
:1000A00085730108B7010008B7010008B70100080F
:1000B000B7010008B7010008B7010008B701000840
:1000C000B7010008B7010008B7010008B701000830
:1000D000B70100084DA40108B7010008B7010008E6
:1000E000B7010008B7010008B7010008B701000810
:1000F000B7010008B7010008B7010008456800080B
:10010000B7010008B7010008B7010008B7010008EF
:10011000B7010008B7010008B7010008957301088E
:10012000B701000855680008656800087568000890
:10013000B7010008B7010008B7010008B7010008BF
:100140005936000869360008B7010008AD3B0108C0
:100150008568000895680008A568000869A401087A
:10016000B7010008B7010008B7010008B70100088F
:10017000B7010008B7010008B7010008000000003F
:10018000B7010008B7010008DFF80CD000F0C4FB8D
:100190000048004791D9010830AE0020064880474A
:1001A00006480047FEE7FEE7FEE7FEE7FEE7FEE75C
:1001B000FEE7FEE7FEE7FEE7657301088901000838
:1001C0002DE9F05F0546002092469B46884606468C
:1001D000814640241BE0284641464746224600F01F
:1001E0002DFA53465A46C01A914110D3114618466B
:1001F000224600F014FA2D1A67EB01084F462246FA
:100200000120002100F00BFA17EB00094E41201EDF
:10021000A4F10104DFDC484631462A464346BDE8E6
:10022000F09F00000649074A0868504343F239022C
:10023000104408604008704701490860704700009A
:10024000000000206D4EC64140EA01039B0703D029
:1002500009E008C9121F08C0042AFAD203E011F805
:10026000013B00F8013B521EF9D27047D2B201E0C7
:1002700000F8012B491EFBD270470022F6E710B5AB
:1002800013460A4604461946FFF7F0FF204610BD04
:1002900010B5044604E00B7800F8013B03B1491C9B
:1002A000521EF8D2204610BD421C10F8011B002936
:1002B000FBD1801A704710B5002200E0521C835C0D
:1002C0008C5CA34201D1002BF8D1D8B2E1B2401A24
:1002D00010BD034611F8012B00F8012B002AF9D1BB
:1002E0001846704730B505460020034600E05B1C09
:1002F000934205D2EC5CC85C201A01D1002CF6D1E7
:1003000030BD2DE9FE4F804681EA0300C00F0C4648
:10031000009021F0004123F00045B8EB0200A94114
:1003200005D24046214690461C460B46024623F025
:100330000040104347D0270DC7F30A00C3F30A510A
:100340000290401A019040286BDAC3F3130040F486
:10035000801B0098924620B10023D2EB030A63EB86
:100360000B0B01985946C0F14002504600F057F976
:1003700006460D4650465946019A00F06FF910EBBB
:1003800008006141002487EA115284EAE7731A43A6
:1003900040D0009A62B3019A012A4FEA075215DC55
:1003A000001B61EB02014FF0004202EA0752CDE967
:1003B0000042001C41F5801132462B4600F0A6F9A0
:1003C00003B0BDE8F08F40462146F9E7001B61EB22
:1003D0000201001C41F5801300185B412018A2F5B2
:1003E000001747EB030140EAD570B6196D4111E0E3
:1003F0006D084FEA360645EAC0754FEA0752001B02
:1004000061EB0201001C41F5801149084FEA300000
:100410000019514132462B4603B0BDE8F04F00F0C1
:1004200066B90098012240000023D0EB020263EB82
:10043000E073009821464FEAE074B8EB000061EBEE
:100440000401E9E783F000435BE781F0004158E7EE
:100450002DE9FE4F81EA030404F0004421F000413D
:1004600000944FF0000B23F0004350EA01045ED0EB
:1004700052EA03045BD0C3F30A54C1F30A552C4477
:10048000A4F2F3340194A0FB0254C1F3130141F42C
:100490008011C3F3130343F4801301FB024400FBF8
:1004A000034E840A970A44EA815447EA8357A4FB1F
:1004B000076802958D0A05FB07854FEA932C04FB1C
:1004C0000C542705029D4FEA065847EA1637B5EB4C
:1004D00008056EEB070C870E920E47EA811742EA79
:1004E0008312A7FB0201B6EB0B0164EB00042B0D9A
:1004F00043EA0C335E1844EB1C50DA465146E7FBE6
:100500000201C5F313044FEA0B3343EA14534FEAD5
:100510000432019C43EA0603A4F10C040294009CFB
:10052000CDE900B400F0F2F803B0BDE8F08F002090
:100530000146F9E70EB5C10F80EAE0700844CA072A
:10054000002140F233438DE80E000A460B4600F0CE
:10055000DDF803B000BD70B5C1F30A5201F00045EB
:100560000024C1F3130140F2FF3341F480119A4299
:1005700001DA002070BD40F233439A42A2F23342C6
:1005800003DC524200F05AF800E090402C43F1D0D6
:10059000404270BD00F0004230F000400AD0C10D72
:1005A00001F56071C0F3160042EA0151C20840072C
:1005B0001143704700200146704701F0004330B4FA
:1005C00021F0004150EA010206D00A0DA2F5607246
:1005D000C1F31301002A02DC30BC00207047440F35
:1005E00044EAC104C100E01830BC00EBC25000F086
:1005F00047B830B50B46014600202022012409E00F
:1006000021FA02F59D4205D303FA02F5491B04FACB
:1006100002F52844151EA2F10102F1DC30BD202AAA
:1006200004DB203A00FA02F1002070479140C2F149
:10063000200320FA03F3194390407047202A04DB7B
:10064000203A21FA02F00021704721FA02F3D0404B
:10065000C2F120029140084319467047202A06DB68
:10066000CB17203A41FA02F043EAE07306E041FA80
:1006700002F3D040C2F1200291400843194670476E
:100680000029A8BF7047401C490008BF20F00100A6
:10069000704710B4B0FA80FC00FA0CF050EA010484
:1006A00004BF10BC704749B1CCF1200421FA04F416
:1006B00011FA0CF118BF012121430843A3EB0C01EF
:1006C000CB1D4FEA00614FEA102042BF002010BC52
:1006D000704700EBC35010440029A4BF10BC704702
:1006E000401C490008BF20F0010010BC704710B545
:1006F000141E73F1000408DA401C41F10001921845
:100700005B411A4301D120F0010010BD2DE9F04DED
:1007100092469B4611B1B1FA81F202E0B0FA80F242
:1007200020329046FFF77BFF04460F4640EA0A005E
:1007300041EA0B0153465A46084313D0114653EA87
:10074000010019D0C8F140025046FFF777FF054677
:100750000E46504659464246FFF761FF084305D012
:10076000012004E020463946BDE8F08D0020054315
:1007700046EAE0762C4337430A986305E40AA0EB87
:1007800008000022FD0A44EA47540A3002D500203E
:100790000146E9E7010510196941DDE9084500193D
:1007A0006941BDE8F04DA2E72DE9F04D81EA03046F
:1007B00004F0004B21F0004514464FF0000A23F0EE
:1007C000004150EA050220D054EA01021DD0C5F3D1
:1007D0000A570246C5F31303C1F31300C1F30A56C7
:1007E00040F4801543F48013A7EB0608101BD6468F
:1007F00008F2FD3873EB050002D308F1010801E0AF
:1008000092185B41B8F1000F03DA00200146BDE801
:10081000F08D00204FF48011064684460EE0171B31
:1008200073EB050705D3121B63EB050306434CEA84
:10083000010C49084FEA300092185B4150EA010769
:10084000EDD152EA030012D082EA040083EA0501E6
:10085000084305D0101BAB4106D20122002306E05D
:1008600000224FF0004302E06FF0010253101AEB38
:1008700006004CEB085110EB0A0041EB0B01BDE800
:10088000F04DFFF734BFC1F30A52C1F3130140F238
:10089000FF3341F480119A4202DA0020014670478A
:1008A00040F233439A42A2F2334202DC5242FFF753
:1008B000C5BEFFF7B4BE000030B5041E71F10004E0
:1008C00004DB4FF00044404264EB0101141E73F15D
:1008D000000405DB1C464FF00043524263EB040367
:1008E0008B4208BF824230BD30B5041E71F1000456
:1008F00004DB4FF00044404264EB0101141E73F12D
:10090000000405DB1C464FF00043524263EB040336
:10091000994208BF904230BD064C074D06E0E068A2
:1009200040F0010394E8070098471034AC42F6D336
:10093000FFF72EFC3C6002085C6002080EB540F236
:10094000334102910021CDE900110A460B46FFF721
:10095000DDFE03B000BD70B58C1810F8015B15F01A
:10096000070301D110F8013B2A1106D110F8012B21
:1009700003E010F8016B01F8016B5B1EF9D12B0746
:1009800005D40023521E0DD401F8013BFAE710F8FC
:10099000013BCB1A921C03E013F8015B01F8015BE9
:1009A000521EF9D5A142D8D3002070BD80B582B0C7
:1009B000019042F20030C4F20100009000994868B2
:1009C00020F440304860019842680099486810431C
:1009D000486001980168486820F480704860019878
:1009E00001680269486840EA02204860019801688D
:1009F000486820F040704860019801688268486843
:100A00001043486001980168886820F4006088609D
:100A100001980168C2688868104388600198806AFC
:100A20000121C0F60071884219D0FFE701980168E2
:100A3000886820F07060886001980168826A886820
:100A40001043886001980168886820F040508860F1
:100A500001980168C26A8868104388600CE00198B8
:100A60000168886820F07060886001980168886873
:100A700020F040508860FFE701980168886820F006
:100A8000020088600198027E0168886840EA42009E
:100A90008860019890F8200060B3FFE70198406AF1
:100AA00030B1FFE70198406A082801D8FFE708E065
:100AB00045F24E20C0F6020040F2A6711CF0C2FEC4
:100AC000FFE701980168486840F4006048600198B9
:100AD0000168486820F46040486001980168426AF3
:100AE0004EF20000CFF6FF7000EB42324868104330
:100AF000486006E001980168486820F4006048609A
:100B0000FFE701980168C86A20F47000C862019884
:100B10000168C2690020CFF6F07000EB0252C86A8B
:100B20001043C86201980168886820F400708860EA
:100B3000019890F830200168886840EA4220886077
:100B400001980168886820F48060886001980168D5
:100B50004269886840EA8220886002B080BD000057
:100B600080B58AB008900791089820B9FFE7FF2068
:100B70008DF827009BE0079820B9FFE7FF208DF84C
:100B8000270094E0079890ED000A90ED013A90ED6F
:100B9000021A90ED032A20EE030A21EE021A30EE2B
:100BA000010A30EE000A8DED060A079890ED010A61
:100BB00090ED021A20EE000A21EE011A30EE010A31
:100BC00030EE001AB7EE000A8DED010A30EE410A50
:100BD0008DED050A9DED060ADDED050A21F06CFF9D
:100BE0009DED011A089880ED010A079890ED000A22
:100BF00090ED013A90ED024A90ED032A20EE040AAE
:100C000022EE032A30EE420A30EE000A8DED040A8D
:100C10009DED040AB0EEC00AB4EE410AF1EE10FAFE
:100C20000ADBFFE7DDED040A9FED230A1CF01EFE40
:100C3000089880ED020A07E09DED040A21F038FCD7
:100C4000089880ED020AFFE7079890ED000A90ED02
:100C5000011A90ED022A90ED033A20EE030A21EEEC
:100C6000021A30EE010A30EE000A8DED030A0798F1
:100C700090ED020A90ED031A20EE000A21EE011A0F
:100C800030EE010A30EE001AB7EE000A30EE410AEB
:100C90008DED020A9DED030ADDED020A21F00CFF45
:100CA000089880ED000A00208DF82700FFE79DF9E5
:100CB00027000AB080BD00BFDB0FC93F80B58CB0F4
:100CC0000A9009918DED080A0A9820B9FFE7FF20E4
:100CD0008DF82F0029E19DED081AB7EE000A80EE8D
:100CE000010A0A9880ED040A0A994FF07E500860C4
:100CF0000A99002048600A9988600A99C860099892
:100D0000002800F00E81FFE7099801680091406813
:100D1000FFF740FC0246009801920A46019942EC16
:100D2000101B8DED020BFFF735FC9DED020B41EC26
:100D3000110B21F0C1FD8DED040B9DF8170080F023
:100D400080008DF8170004980599FFF736FC07908E
:100D5000099890ED000AB5EE400AF1EE10FA2BD199
:100D6000FFE7099890ED010AB5EE400AF1EE10FA9E
:100D700022D1FFE7099890ED020AB5EE400AF1EEA4
:100D800010FA19D1FFE70A9940F2C560C3F64D7019
:100D900008600A9944F62D20C3F60D4048600A9970
:100DA0004AF25640CBF6393088600A9944F2AD7069
:100DB000C3F61970C860B3E09DED070A9FED5D1A98
:100DC000B4EE410AF1EE10FA08DBFFE79DED070AE9
:100DD000B5EE400AF1EE10FA19DDFFE70A9945F683
:100DE0006E10C3F67F7008600A9945F20C30C3F6A6
:100DF000B01048600A9948F6AB00CBF6BB3088606B
:100E00000A9949F28550C3F69750C86087E09DED76
:100E1000070A9FED491AB4EE410AF1EE10FA0ADB17
:100E2000FFE79DED070A9FED431AB4EE410AF1EE8C
:100E300010FA19DDFFE70A9940F2C560C3F64D705C
:100E400008600A9944F62D20C3F60D4048600A99BF
:100E50004AF25640CBF6393088600A9944F2AD70B8
:100E6000C3F61970C86059E09DED070A9FED331A6B
:100E7000B4EE410AF1EE10FA0ADBFFE79DED070A36
:100E80009FED2D1AB4EE410AF1EE10FA19DDFFE7DD
:100E90000A9940F2C560C3F64D7008600A9944F69D
:100EA0002D20C3F60D4048600A994AF25640CBF611
:100EB000393088600A9944F2AD70C3F61970C86081
:100EC0002BE09DED070A9FED1D1AB4EE410AF1EEED
:100ED00010FA08DBFFE79DED070AB5EE400AF1EED8
:100EE00010FA19DDFFE70A9940F2C560C3F64D70AC
:100EF00008600A9944F62D20C3F60D4048600A990F
:100F00004AF25640CBF6393088600A9944F2AD7007
:100F1000C3F61970C860FFE7FFE7FFE7FFE7FFE7E9
:100F2000FFE700208DF82F00FFE79DF92F000CB0A0
:100F300080BD00BFDB0FC93FDB0F49400000B4425A
:100F400081B000900099002088604860086001B07E
:100F50007047000080B52DED048BB2B030902F911A
:100F60002E922D93309828B9FFE7FF208DF8C70007
:100F700000F0F7BD2F9828B9FFE7FF208DF8C700D4
:100F800000F0EFBD2E9828B9FFE7FF208DF8C700CD
:100F900000F0E7BD40F28411C2F200014EF69E70EF
:100FA000C3F6275008602D9848B9FFE730982F996D
:100FB0002E9A00F0DDFD8DF8C70000F0D2BD2D980F
:100FC000006809902D98406808902D9880680790D7
:100FD0009DED090AB5EE400AF1EE10FA19D1FFE7CE
:100FE0009DED080AB5EE400AF1EE10FA11D1FFE7C7
:100FF0009DED070AB5EE400AF1EE10FA09D1FFE7C0
:1010000030982F992E9A00F0B3FD8DF8C70000F0AC
:10101000A8BD2F98006806902F98406805902F98DB
:10102000806804902E98006803902E984068029083
:101030002E988068019030989DED033A90ED010A5A
:1010400090ED022A90ED031A20EE430A9DED023A3C
:1010500022EE032A30EE420A9DED012A21EE021A09
:1010600030EE410AB6EE001A20EE010A8DED270A95
:1010700030989DED034A90ED000A90ED023A90ED14
:10108000032A20EE040A9DED014A23EE043A30EED5
:10109000030A9DED023A22EE032A30EE420A20EEC8
:1010A000010A8DED260A30989DED024A90ED000A66
:1010B00090ED013A90ED032A20EE040A9DED014ADD
:1010C00023EE043A30EE430A9DED033A22EE032A62
:1010D00030EE020A20EE010A8DED250A30989DEDD2
:1010E000014A90ED000A90ED013A90ED022A20EEBF
:1010F000040A9DED024A23EE043A30EE030A9DED08
:10110000033A22EE032A30EE420A20EE010A8DED68
:10111000240A9DED060AB5EE400AF1EE10FA11D14F
:10112000FFE79DED050AB5EE400AF1EE10FA09D190
:10113000FFE79DED040AB5EE400AF1EE10FA00F06B
:101140009984FFE79DED060A20EE000A9DED051A41
:1011500021EE011A30EE010A9DED041A21EE011A6A
:1011600030EE010A11F0B0FA8DED2C0A9DED2C1A2B
:101170009DED060A20EE010A8DED060A9DED2C1A62
:101180009DED050A20EE010A8DED050A9DED2C1A54
:101190009DED040A20EE010A8DED040A9DED090A79
:1011A00020EE000A9DED081A21EE011A30EE010A28
:1011B0009DED071A21EE011A30EE010A11F084FAB2
:1011C0008DED2C0A9DED2C1A9DED090A20EE010AE9
:1011D0008DED090A9DED2C1A9DED080A20EE010AFD
:1011E0008DED080A9DED2C1A9DED070A20EE010AEF
:1011F0008DED070A309890ED000A30EE000A9DED63
:10120000091A20EE010A8DED210A309890ED000AAE
:1012100030EE000A9DED081A20EE010A8DED200A3D
:10122000309890ED000A30EE000A9DED071A20EE8E
:10123000010A8DED1F0A309890ED010A30EE000A88
:101240009DED091A20EE010A8DED1E0A309890EDF1
:10125000000A30EE000A8DED190A309890ED010A6F
:1012600030EE000A8DED180A309890ED020A30EE4B
:10127000000A8DED170A309890ED030A30EE000A4F
:101280008DED160A309890ED000A90ED021A30EEBE
:10129000000A20EE010A8DED150A309890ED020A41
:1012A00090ED031A30EE000A20EE010A8DED140ACB
:1012B000309890ED000A20EE000A8DED130A309868
:1012C00090ED000A90ED011A20EE010A8DED120A50
:1012D000309890ED000A90ED021A20EE010A8DED93
:1012E000110A309890ED000A90ED031A20EE010AE1
:1012F0008DED100A309890ED010A20EE000A8DED78
:101300000F0A309890ED010A90ED021A20EE010AC2
:101310008DED0E0A309890ED010A90ED031A20EE43
:10132000010A8DED0D0A309890ED020A20EE000AB8
:101330008DED0C0A309890ED020A90ED031A20EE24
:10134000010A8DED0B0A309890ED030A20EE000A99
:101350008DED0A0A9DED091A9DED130A21EE000A92
:101360009DED202A309890ED025A90ED033A22EE3E
:10137000032A30EE420A9DED1F2A22EE052A30EEA6
:10138000020A9DED0F2A21EE022A30EE020A9DED9F
:10139000182A9DED084A22EE044A24EE054A30EE52
:1013A000040A9DED074A22EE042A22EE032A30EEBB
:1013B000020A9DED0C2A21EE022A30EE420A9DED32
:1013C0000A2A21EE021A30EE410A8DED230A9DED24
:1013D000210A309890ED015A90ED024A90ED033ABF
:1013E00020EE030A9DED081A9DED132A21EE022A34
:1013F00030EE020A9DED1F2A22EE052A30EE420A47
:101400009DED1E2A22EE042A30EE020A9DED0F2ADF
:1014100021EE022A30EE420A9DED0C2A21EE022A2C
:1014200030EE020A9DED172A9DED074A22EE042AAE
:1014300022EE032A30EE020A9DED0A2A21EE021A5C
:1014400030EE410A8DED220A9DED230A20EE000ABE
:101450009DED221A21EE011A30EE010A11F034F945
:10146000B7EE006A86EE000A8DED1D0A9DED210A99
:10147000309890ED012A90ED021A90ED033A20EE9B
:10148000011A9DED200A20EE020A30EE412A9DED60
:10149000071A9DED130A21EE000A30EE022A9DED97
:1014A0001E0A20EE030A30EE020A9DED0F2A21EEFD
:1014B000022A30EE420A9DED172A9DED084A22EEDF
:1014C000042A22EE032A30EE020A9DED0C2A21EEB8
:1014D000022A30EE420A9DED0A2A21EE021A30EE6F
:1014E000010A8DED1C0A9DED1D0A30EE000A8DEDFE
:1014F0001B0A9DED1C0A30EE000A8DED1A0A9DEDC7
:10150000170ADDED0D0A30EEA02A9DED151A31EE19
:10151000422A9DED061A31EE021A20EE010A9DEDD7
:10152000181ADDED123A33EEA32A9DED143A32EE8D
:10153000032A9DED053A32EE432A21EE021A70EE9F
:10154000014A9DED1C3A309890ED011A90ED020A87
:10155000D0ED032A63EE001A9DED1D2A9DED0C7A55
:10156000B6EE004A8DED004A77EE445A9DED0A5AD8
:1015700035EE255A62EE055A9DED115A75EE606AF8
:1015800063EE266A75EEA66ADDED095A75EEA65A77
:1015900061EEA51A71EEA41A62EE222A23EE011A58
:1015A00031EE621ADDED0E2ADDED104A72EEE42A0C
:1015B00062EE222ADDED0B4A73EEA43A63EE233A83
:1015C00072EEA32ADDED083A72EEE32A21EE221A2A
:1015D00031EE211A22EE000A35EE205A22EE052ABB
:1015E0009DED0F5A34EE455A35EE475A23EE053A33
:1015F00032EE032A9DED073A32EE432A20EE020A2C
:1016000030EE010A8DED2B0A9DED160ADDED0D2A57
:1016100032EEA21A9DED152A31EE421A9DED062AF0
:1016200031EE421A20EE010A9DED191ADDED126A23
:1016300036EEA62A9DED143A32EE032A9DED053AC8
:1016400032EE432A21EE021A30EE011A3098D0ED24
:10165000005AD0ED014AD0ED023A90ED032AB1EEE6
:10166000000A24EE803A9DED0F7A37EE075A75EEA8
:10167000461ADDED0C0A30EEA05A75EE211A9DEDEA
:10168000045A35EE215A23EE053A31EE031A9DED48
:101690001C5A65EE027A9DED1D3A74EE601A9DEDBE
:1016A0000A8A71EEC81A23EE218ADDED111A32EE94
:1016B000E19A25EE099A38EE098A9DED099A38EEED
:1016C000498A67EE887A31EE271A63EE233A65EE8F
:1016D000255A73EEA53ADDED0E5ADDED107A75EE62
:1016E000E75A63EE255ADDED0B7A76EEA76A65EED2
:1016F000266A75EEA65ADDED086A75EEE65A63EEC7
:10170000A53A31EE231A23EE022ADDED1A3A63EEF2
:10171000A43A32EE632A71EEA21A23EE213A34EE95
:10172000477A37EE607A25EE075A33EE053A9DED9B
:10173000075A33EE453A22EE032A31EE021A8DEDB6
:101740002A1A9DED191ADDED0D0A30EEA03A9DED35
:10175000152A32EE433A9DED062A32EE032A21EE97
:10176000021A9DED162ADDED124A34EEA43A9DEDE3
:10177000145A33EE053A9DED055A33EE453A22EE02
:10178000032A31EE022A309890ED001AD0ED011AAA
:10179000D0ED022AD0ED033A22EE800A9DED0F5AD9
:1017A00035EE053A33EE467A9DED0C6A36EE063A92
:1017B00033EE077A9DED043A33EE073A20EE030A42
:1017C00070EE025A9DED1B0A20EE620A9DED1C3A56
:1017D00023EE012A30EE420A9DED1D2A34EE467AB0
:1017E000DDED0A6A37EE667A62EE076A9DED117AE0
:1017F00070EEC77A63EE277A76EEA76ADDED097A96
:1018000076EEE76A20EE260A30EE250A62EE211A0D
:1018100063EE233A71EEA31ADDED0E3ADDED105AB8
:1018200073EEE53A62EE233ADDED0B5A74EEA54A0B
:1018300063EE244A73EEA43ADDED084A73EEE43A0F
:1018400061EEA31A30EE210A22EE011ADDED1A1A1A
:1018500061EEA21A31EE611A37EE207A22EE072AE3
:1018600034EE455A35EE465A23EE053A32EE032A57
:101870009DED073A32EE432A21EE021A30EE010ABC
:101880008DED290A9DED180A9DED0D7A37EE071AA8
:101890009DED152A31EE421A9DED062A31EE421ACF
:1018A00020EE010A9DED171ADDED122A32EEA22A72
:1018B0009DED143A32EE032A9DED053A32EE432AAD
:1018C00021EE021A70EE013A9DED1B1A3098D0ED10
:1018D000001A90ED010AD0ED020A90ED032A21EEE4
:1018E000022A9DED1C3A23EE001A31EE421A9DEDBC
:1018F0001D2A9DED0C5A34EE456ADDED0A4A36EE9E
:10190000646A62EE064A9DED116A77EE465A63EE0E
:10191000255A74EEA54ADDED095A74EEE54A21EE2A
:10192000241A31EE231A62EE211A63EE200A70EEB9
:10193000E10ADDED0E1ADDED103A71EEE31A62EE0A
:10194000211ADDED0B3A72EEA32A63EE222A71EE24
:10195000A21ADDED082A71EEE21A60EEA10A31EE5C
:10196000201A22EE000A36EE076A22EE062A9DEDC4
:101970000F6A34EE464A34EE454A23EE043A32EE1C
:10198000032A9DED073A32EE432A20EE020A30EE9A
:10199000010A8DED280A9DED2B0A20EE000A9DED2F
:1019A0002A1A21EE011A30EE010A9DED291A21EEC4
:1019B000011A30EE010A9DED281A21EE011A30EECF
:1019C000010A10F081FE8DED2C0A9DED2C1A9DED83
:1019D0002B0A20EE010A8DED2B0A9DED2C1A9DEDB0
:1019E0002A0A20EE010A8DED2A0A9DED2C1A9DEDA2
:1019F000290A20EE010A8DED290A9DED2C1A9DED94
:101A0000280A20EE010A8DED280A40F28410C2F265
:101A1000000090ED000A9DED2B1A20EE011A9DEDBD
:101A2000270A30EE410A8DED270A90ED000A9DED60
:101A30002A1A20EE011A9DED260A30EE410A8DED9C
:101A4000260A90ED000A9DED291A20EE011A9DED5F
:101A5000250A30EE410A8DED250A90ED000A9DED34
:101A6000281A20EE011A9DED240A30EE410A8DED70
:101A7000240AFFE79DED271A309890ED000A90EDBB
:101A8000042A21EE021A30EE010A80ED000A9DEDD3
:101A9000261A309890ED010A90ED042A21EE021AE0
:101AA00030EE010A80ED010A9DED251A309890ED87
:101AB000020A90ED042A21EE021A30EE010A80EDAE
:101AC000020A9DED241A309890ED030A90ED042A45
:101AD00021EE021A30EE010A80ED030A309890EDF3
:101AE000000A90ED013A90ED022A90ED031A20EEE3
:101AF000000A23EE033A30EE030A22EE022A30EE09
:101B0000020A21EE011A30EE010A10F0DDFD8DED22
:101B10002C0A9DED2C1A309890ED000A20EE010A57
:101B200080ED000A9DED2C1A309890ED010A20EE10
:101B3000010A80ED010A9DED2C1A309890ED020A01
:101B400020EE010A80ED020A9DED2C1A309890EDEE
:101B5000030A20EE010A80ED030A00208DF8C70079
:101B6000FFE79DF9C70032B0BDEC048B80BD0000DB
:101B700080B5A0B01E901D911C921E9820B9FFE761
:101B8000FF208DF87F00D3E21D9820B9FFE7FF20EA
:101B90008DF87F00CCE21C9820B9FFE7FF208DF87C
:101BA0007F00C5E240F28411C2F2000142F6023029
:101BB000C3F6075008601D9800681B901D98406888
:101BC0001A901D98806819901C98006818901C98AD
:101BD000406817901C98806816901E989DED183AE2
:101BE00090ED010A90ED022A90ED031A20EE430ACF
:101BF0009DED173A22EE032A30EE420A9DED162A99
:101C000021EE021A30EE410AB6EE001A20EE010A69
:101C10008DED100A1E989DED184A90ED000A90ED8A
:101C2000023A90ED032A20EE040A9DED164A23EEB7
:101C3000043A30EE030A9DED173A22EE032A30EE05
:101C4000420A20EE010A8DED0F0A1E989DED174AFB
:101C500090ED000A90ED013A90ED032A20EE040A7F
:101C60009DED164A23EE043A30EE430A9DED183AF4
:101C700022EE032A30EE020A20EE010A8DED0E0A52
:101C80001E989DED164A90ED000A90ED013A90EDF8
:101C9000022A20EE040A9DED174A23EE043A30EEA4
:101CA000030A9DED183A22EE032A30EE420A20EE96
:101CB000010A8DED0D0A9DED1B0AB5EE400AF1EE0D
:101CC00010FA11D1FFE79DED1A0AB5EE400AF1EEC8
:101CD00010FA09D1FFE79DED190AB5EE400AF1EEC1
:101CE00010FA00F0AE81FFE79DED1B0A20EE000A1E
:101CF0009DED1A1A21EE011A30EE010A9DED191A16
:101D000021EE011A30EE010A10F0DEFC8DED150A0D
:101D10009DED151A9DED1B0A20EE010A8DED1B0AA3
:101D20009DED151A9DED1A0A20EE010A8DED1A0A95
:101D30009DED151A9DED190A20EE010A8DED190A87
:101D40001E9890ED000A30EE000A8DED0C0A1E98E8
:101D500090ED010A30EE000A8DED0B0A1E9890ED11
:101D6000020A30EE000A8DED0A0A1E9890ED030A71
:101D700030EE000A8DED090A1E9890ED000AB1EED2
:101D8000003A20EE030A8DED080A1E9890ED010A34
:101D900020EE030A8DED070A1E9890ED020A20EE50
:101DA000030A8DED060A1E9890ED010AB2EE001AA4
:101DB00020EE010A8DED050A1E9890ED020A20EE34
:101DC000010A8DED040A1E9890ED000A20EE000A2B
:101DD0008DED030A1E9890ED010A20EE000A8DEDAC
:101DE000020A1E9890ED020A20EE000A8DED010A0B
:101DF0001E9890ED030A20EE000A8DED000A9DED7D
:101E0000081A9DED010A21EE000A9DED0A2A9DEDBA
:101E10001B4A22EE042A30EE020A9DED022A21EE30
:101E2000021A30EE010A9DED0B1A9DED1A2A21EEE1
:101E3000021A30EE410A8DED140A9DED071A9DED50
:101E4000000A21EE000A9DED092A9DED1B4A22EEB3
:101E5000042A30EE420A9DED032A22EE032A1E9840
:101E600090ED014A22EE042A30EE020A9DED0C2A82
:101E70009DED1A4A22EE042A30EE420A30EE410A63
:101E80009DED052A9DED024A22EE044A30EE040A39
:101E90009DED014A22EE042A30EE020A9DED192A38
:101EA00021EE021A30EE010A8DED130A9DED030AB0
:101EB00020EE030A1E9890ED021A20EE010A9DED15
:101EC0000C1A9DED1B2A21EE021A30EE010A9DED3F
:101ED000061A9DED002A21EE022A30EE020A9DED3F
:101EE000092A9DED1A4A22EE042A30EE420A30EE0B
:101EF000410A9DED042A9DED024A22EE044A30EE8D
:101F0000040A9DED014A22EE042A30EE020A9DEDFC
:101F1000192A21EE021A30EE010A8DED120A9DED0A
:101F2000020A20EE030A1E9890ED032A20EE020A10
:101F30009DED0B1A9DED1B4A21EE041A30EE410A6D
:101F40009DED011A21EE031A21EE021A30EE010A6C
:101F50009DED0A1A9DED1A2A21EE021A30EE410A71
:101F60008DED110A9DED140A20EE000A9DED131A65
:101F700021EE011A30EE010A9DED121A21EE011A2E
:101F800030EE010A9DED111A21EE011A30EE010A20
:101F900010F09AFB8DED150A9DED151A9DED140AB2
:101FA00020EE010A8DED140A9DED151A9DED130A20
:101FB00020EE010A8DED130A9DED151A9DED120A12
:101FC00020EE010A8DED120A9DED151A9DED110A04
:101FD00020EE010A8DED110A40F28410C2F20000D9
:101FE00090ED000A9DED141A20EE011A9DED100AE5
:101FF00030EE410A8DED100A90ED000A9DED131AA6
:1020000020EE011A9DED0F0A30EE410A8DED0F0A08
:1020100090ED000A9DED121A20EE011A9DED0E0AB8
:1020200030EE410A8DED0E0A90ED000A9DED111A79
:1020300020EE011A9DED0D0A30EE410A8DED0D0ADC
:10204000FFE79DED101A1E9890ED000A90ED042A0E
:1020500021EE021A30EE010A80ED000A9DED0F1A02
:102060001E9890ED010A90ED042A21EE021A30EE3E
:10207000010A80ED010A9DED0E1A1E9890ED020AEC
:1020800090ED042A21EE021A30EE010A80ED020AD8
:102090009DED0D1A1E9890ED030A90ED042A21EE95
:1020A000021A30EE010A80ED030A1E9890ED000A34
:1020B00090ED013A90ED022A90ED031A20EE000A0D
:1020C00023EE033A30EE030A22EE022A30EE020A31
:1020D00021EE011A30EE010A10F0F6FA8DED150A24
:1020E0009DED151A1E9890ED000A20EE010A80ED74
:1020F000000A9DED151A1E9890ED010A20EE010AC6
:1021000080ED010A9DED151A1E9890ED020A20EE51
:10211000010A80ED020A9DED151A1E9890ED030A42
:1021200020EE010A80ED030A00208DF87F00FFE712
:102130009DF97F0020B080BD84B00290019102988B
:1021400020B9FFE7FE208DF80F001FE0019820B9AD
:10215000FFE7FE208DF80F0018E0029900200090A4
:1021600081F847000299C1F81B0088614861086145
:10217000C860886048600199886148610861C860EA
:102180008860486008608DF80F00FFE79DF90F0038
:1021900004B0704780B584B00290FFE7029840B960
:1021A000FFE745F2ED50C0F602002D211BF046FA84
:1021B000FFE7FFE742F2B430C2F200000078C00748
:1021C00020B1FFE7FD208DF80F002DE0FFE71BF0A9
:1021D000F9FF42F6E871C2F20001086040B9FFE77A
:1021E00045F2ED50C0F602002F211BF027FAFFE761
:1021F000FFE742F22552C0F60002022001900321BF
:1022000001F07CF9019842F20D52C0F6000208215B
:1022100001F074F942F2B431C2F2000101200870F9
:1022200000208DF80F00FFE79DF90F0004B080BD7E
:1022300082B001900091019840680099086001986F
:102240008068009948600198007FC0F3C000009941
:1022500008760198007FC0090099487601980069C6
:102260000099C860019840690099086101988069E7
:102270000099486102B0704780B584B00390029124
:1022800001920399C42081F826000399DDF808C063
:10229000DCF80000DCF80420DCF80830DCF80CC0C6
:1022A000C1F833C0C1F82F30C1F82B20C1F8270086
:1022B0000399019B18685A689B68C1F83F30C1F8C0
:1022C0003B20C1F837000399002081F843000398B0
:1022D00090F84600012808D1FFE7039991F84300E0
:1022E00040F0010081F843001DE0039890F846009B
:1022F000022808D1FFE7039991F8430040F002005B
:1023000081F843000EE0039890F84600032808D1B6
:10231000FFE7039991F8430040F0040081F843007F
:10232000FFE7FFE7FFE7039827301D214FF6FF7215
:1023300002F030FA0399A1F84400002004B080BDF7
:1023400080B582B0019000910199A820C8770098CB
:1023500040880199088400988088019948840198F0
:10236000203004214FF6FF7202F014FA019988849C
:10237000002002B080BD000080B584B0029042F61B
:102380000040C2F200001B2102F020FA08B9FFE76A
:102390001BE00299012081F847000298043042F6C0
:1023A0000041C2F2000100911B22FDF74DFF009990
:1023B00000200190C1F8170048610861C86088607A
:1023C000486008608DF80F000AE041F28411C2F203
:1023D0000001086801300860FF208DF80F00FFE75A
:1023E0009DF90F0004B080BD80B582B0009002203E
:1023F00001F024F842F60041C2F200011B220FF066
:102400007FFF20B9FFE700208DF8070003E0FF20E1
:102410008DF80700FFE79DF9070002B080BD0000BE
:1024200080B584B002908DF807109DF80700C007B2
:1024300090B1FFE7022001F001F802991F31272235
:102440000FF0EEFF20B9FFE700208DF80F0015E038
:10245000FF208DF80F0011E0022000F0EFFF02993D
:10246000263120220FF0DCFF20B9FFE700208DF895
:102470000F0003E0FF208DF80F00FFE79DF90F002C
:1024800004B080BD80B54FF48040012100221BF0D4
:102490000BFEA0F58040B0FA80F0400980BD00003E
:1024A00084B08DED030ACDED020A9DED030A9DED8A
:1024B000021AB1EE411AB4EE410AF1EE10FA07DA4F
:1024C000FFE79DED020AB1EE400A8DED010A18E02A
:1024D0009DED030A9DED021AB4EE410AF1EE10FAE9
:1024E00005DDFFE79DED020A8DED000A04E09DED9C
:1024F000030A8DED000AFFE79DED000A8DED010A4C
:10250000FFE79DED010A04B07047000080B542F678
:10251000E870C2F2000000684FF480411BF072FDC9
:1025200080BD000080B542F6E870C2F2000000688D
:102530004FF480411BF066FD80BD000080B542F67F
:10254000D870C2F20000006802211BF05BFD80BD64
:1025500080B582B040F6B812C2F2000200200190AD
:102560001221132300F06EFA019802B080BD000022
:1025700080B5082001214FF0FF321BF095FD80BD92
:1025800081B000909FED010A01B070470000C84380
:1025900080B542F6D870C2F20000006801211BF03D
:1025A00031FD80BD82B00190019890ED000A0020BD
:1025B0009FED141AB4EE410AF1EE10FA00901BDA06
:1025C000FFE7019890ED010A00209FED0E1AB4EE8E
:1025D000410AF1EE10FA00900EDAFFE7019890ED53
:1025E000020A9FED081A0020B4EE410AF1EE10FA3B
:1025F000B8BF01200090FFE7009800F0010002B092
:10260000704700BF8FC2F53C80B540F6B810C2F2EB
:102610000000C21D01200221062300F013FA002051
:1026200080BD000080B5042001214FF0FF321BF077
:102630003BFD80BD80B58CB00A9009910A9820B905
:10264000FFE7FE208DF82F00B5E0099820B9FFE7DD
:10265000FE208DF82F00AEE042F2B030C2F2000052
:102660000078C00720B1FFE7FD208DF82F00A2E021
:102670001BF0A8FD42F6D871C2F20001086020B933
:10268000FFE7FE208DF82F0095E009980A99C861B0
:10269000002008907E21B622069200F087FA069A62
:1026A0000120142100F082FA1E20079000F01CFB8C
:1026B0000799089800F00CFA0899084600F008FA03
:1026C0001E2804D0FFE7FC208DF82F0073E00120C6
:1026D000002100F0FDF90F2804D0FFE7FC208DF861
:1026E0002F0068E01020039000F0A6FB202004904B
:1026F00000F0A2FB42F6CD12C0F6000201210291C9
:10270000084600F079FE039842F23D51C0F6000100
:1027100000F006FC049842F29151C0F6000100F06E
:10272000FFFB002005904021AA2200F03FFA029A08
:102730000598412100F03AFA05985321082200F04B
:1027400035FA059858210422019200F02FFA019AD7
:1027500005987D2100F02AFA322000F0C5FA029A8D
:102760000F21104600F022FA02980399032200F08C
:102770001DFA0298059A162100F018FA029A1821FB
:10278000104600F013FA02981521802200F00EFA8C
:102790000A2000F0A9FA0299039842F2B032C2F27C
:1027A0000002117000F082FB049800F07FFB059896
:1027B0008DF82F00FFE79DF92F000CB080BD0000C1
:1027C00084B00290029820B9FFE7FE208DF80F0038
:1027D0006AE040F6B811C2F20001B1F80100ADF8AC
:1027E0000600B1F80300ADF80400B1F80500ADF83B
:1027F0000200BDF9060000EE100AB8EEC00A029809
:1028000080ED000ABDF9040000EE100AB8EEC00A1F
:10281000029880ED010ABDF9020000EE100AB8EE40
:10282000C00A029880ED020A029890ED000A9FED1E
:10283000201A80EE010A80ED000A029890ED010A4C
:1028400080EE010A80ED010A029890ED020A80EE06
:10285000010A80ED020A487C897CC00040EA5110E0
:10286000ADF80000BDF90000B0F5806F07DBFFE7B1
:10287000BDF80000A0F50060ADF80000FFE7BDF96D
:10288000000000EE100AB8EEC00AB4EE001A20EE06
:10289000010AB3EE071A30EE010A029880ED060A2B
:1028A00000208DF80F00FFE79DF90F0004B070477E
:1028B00000A0AA4584B00290029820B9FFE7FE204C
:1028C0008DF80F007AE040F6B810C2F20000B0F8C0
:1028D0000710ADF80610B0F80910ADF80410B0F804
:1028E0000B00ADF80200BDF9060000EE100AB8EECC
:1028F000C00A029880ED030ABDF9040000EE100A38
:10290000B8EEC00A029880ED040ABDF9020000EE9C
:10291000100AB8EEC00A029880ED050A029890ED00
:10292000030A9FED281A80EE010A80ED030A02983F
:1029300090ED040A80EE010A80ED040A029890ED01
:10294000050A80EE010A80ED050A029890ED030A5F
:102950009FED1D1A20EE010A80ED030A029890ED0A
:10296000040A20EE010A80ED040A029890ED050A9F
:1029700020EE010A80ED050A0298C16991ED001A66
:1029800090ED030A30EE410A80ED030A0298C16916
:1029900091ED011A90ED040A30EE410A80ED040A2F
:1029A0000298C16991ED021A90ED050A30EE410AD4
:1029B00080ED050AFE208DF80F00FFE79DF90F005E
:1029C00004B070476F12034235FA8E3C80B5002088
:1029D000C4F20200102108F03FFD80B9FFE700209B
:1029E000C4F202001021012208F060FD42F6D87006
:1029F000C2F20000006808211BF004FBFFE740F270
:102A00000040C4F20200012108F026FD88B9FFE76A
:102A100040F20040C4F202000122114608F046FDD7
:102A200042F6D870C2F20000006804211BF0EAFAF6
:102A3000FFE780BD80B5032001214FF0FF321BF07E
:102A400033FB80BD80B586B08DF817008DF8161069
:102A500004928DF80F30049808B9FFE736E09DF82E
:102A600017000146029120B1FFE70298012808D023
:102A700010E00020C4F202001021002208F016FD30
:102A800008E040F20040C4F202000121002208F0F8
:102A90000DFDFFE79DF8160040F0800040F6CB11D9
:102AA000C2F20001009108700120019000F084FC46
:102AB0000099019A14230BF037FF019800F07CFC79
:102AC00004999DF80F200BF0F1FDFFE706B080BDE3
:102AD00080B586B08DF816008DF81510012000F035
:102AE00003F99DF816000146049120B1FFE7049810
:102AF000012808D010E00020C4F2020010210022BA
:102B000008F0D4FC08E040F20040C4F202000121C9
:102B1000002208F0CBFCFFE79DF8150040F0800094
:102B200040F6CB11C2F20001019108700120009023
:102B300000F042FC009A0199142302930BF0F4FE7A
:102B4000009800F039FC0199029B02220BF096FCE0
:102B50009DF816000146039120B1FFE70398012874
:102B60000FD01EE00020C4F202001021012208F064
:102B70009DFC40F6CB10C2F2000040788DF81700A3
:102B80000FE040F20040C4F202000122114608F0BA
:102B90008DFC40F6CB10C2F2000000788DF81700D3
:102BA000FFE79DF8170006B080BD000080B584B037
:102BB0008DF80F008DF80E108DF80D209DF80E0089
:102BC00000F07F0040F6CB11C2F2000108709DF8C2
:102BD0000D004870012000F087F89DF80F000146B5
:102BE000029120B1FFE70298012808D010E00020F0
:102BF000C4F202001021002208F058FC08E040F264
:102C00000040C4F202000121002208F04FFCFFE75F
:102C1000012000F0D1FB40F6CB11C2F200010222EC
:102C200014230BF081FE9DF80F000146019120B1A5
:102C3000FFE70198012808D010E00020C4F202004C
:102C40001021012208F032FC08E040F20040C4F2FA
:102C500002000122114608F029FCFFE704B080BD04
:102C600083B08DF807009DF807000146009150B130
:102C7000FFE7009801280CD1FFE741F23C70C2F257
:102C80000000029008E041F21470C2F200000290CD
:102C900002E000200290FFE7029803B070470000B6
:102CA00082B08DF806008DF805100092009820B9CA
:102CB000FFE7FE208DF8070011E000989DF8061050
:102CC00040F2F823C2F20003342211FB02319DF8D6
:102CD000052041F8220000208DF80700FFE79DF94C
:102CE000070002B07047000080B586B004901AF06B
:102CF00011FF01464FF47A70B0FBF1F00390049895
:102D00000399B0FBF1F002901AF0C6FE0146481C90
:102D1000019198B1FFE70198022820D3FFE70198BD
:102D200002280FD0FFE701980338022806D3FFE7F7
:102D300001986FF00041884215D1FFE7FF208DF820
:102D4000170014E0029818B1FFE70298009002E023
:102D500001200090FFE700981AF058FE03E0049865
:102D600007F00EFEFFE700208DF81700FFE79DF942
:102D7000170006B080BD000080B588B007900798A6
:102D8000E0B1FFE707980B2818D8FFE707980490F1
:102D900000200290022006900120059007F050FFCD
:102DA000FFE7322004F0D8FA08B1FFE7F9E702A8FC
:102DB00001A907F007FE07F0B5FEFFE708B080BDE8
:102DC00080B584B003900291019202980399019A10
:102DD000FDF73AFA04B080BD80B584B0039002914B
:102DE000019207F02DFFFFE70198C0B1FFE7FFE771
:102DF000322004F0B1FA08B1FFE7F9E7039902982D
:102E000002780023184607F097FE039801300390DC
:102E1000029801300290019801380190E4E707F030
:102E200081FE04B080BD000080B582B001900198A1
:102E30001CF0AEFF02B080BD80B582B0ADF80400DA
:102E4000BDF804000138014600911F2822D80099DE
:102E5000DFE801F0182020202020201C2020202046
:102E60002020201020202020202020202020202072
:102E7000202020140A2008F041FF0FE0172008F05E
:102E80003DFF0BE0062008F039FF07E0092008F0BD
:102E900035FF03E0FF208DF8070003E000208DF8E8
:102EA0000700FFE79DF9070002B080BD80B582B042
:102EB000ADF80400BDF804000138014600911F2858
:102EC00022D80099DFE801F0182020202020201CC3
:102ED0002020202020202010202020202020202002
:102EE00020202020202020140A2008F01FFF0FE0BF
:102EF000172008F01BFF0BE0062008F017FF07E083
:102F0000092008F013FF03E0FF208DF8070003E01D
:102F100000208DF80700FFE79DF9070002B080BD93
:102F200083B0ADF808000191019820B9FFE7FE20B9
:102F30008DF80B0025E000208DF80300FFE79DF8D9
:102F400003000F2819DCFFE7BDF808009DF8031007
:102F5000C840C00750B1FFE701989DF8032040F238
:102F60007C31C2F2000141F8220006E0FFE79DF843
:102F7000030001308DF80300E1E700208DF80B001D
:102F8000FFE79DF90B0003B07047000080B588B0E3
:102F9000082004900120059000200690079041F23F
:102FA000CC60C2F2000004A904F09EFE18B1FFE755
:102FB00003F022FFFFE741F2CC60C2F20000019073
:102FC00005F0CCFA0198052105F032FA019804F0D9
:102FD000EBFF03909DED030AB8EE400A40F2EC20AF
:102FE000C2F2000090ED001A20EE010A9FED041AD3
:102FF00020EE010A8DED020A9DED020A08B080BDA7
:103000005D74214180B588B01020049001200590A6
:1030100000200690079041F28460C2F2000004A9EB
:1030200004F062FE18B1FFE703F0E6FEFFE741F2AD
:103030008460C2F20000019005F090FA0198052129
:1030400005F0F6F9019804F0AFFF03909DED030A37
:10305000B8EE400A40F2EC20C2F2000090ED001AF7
:1030600020EE010A8DED020A9DED020A9FED061A7F
:1030700030EE010A9FED051A20EE010AB3EE091A9F
:1030800030EE010A08B080BD5C8F42BF0000C8432B
:1030900080B588B006AA0392024603988DF81E20D8
:1030A0008DF81D1080ED000A90ED000AB7EE001AB1
:1030B000B4EE410AF1EE10FA04DDFFE7FF208DF8CF
:1030C0001F0097E0039890ED000A9FED4C1A20EE48
:1030D000010ABDEEC00A10EE100AADF812009DF80C
:1030E0001E0001460291F0B1FFE70298012804D0CA
:1030F000FFE7029802280BD020E0BDF8120042F250
:10310000D011C2F200010968C8630820059015E0DB
:10311000BDF8120042F2D011C2F2000109688863C2
:10312000042005900AE0BDF8120042F2D011C2F26C
:1031300000010968486300200590FFE79DF81D0025
:103140000146019140B1FFE70198012814D0FFE743
:103150000198022820D049E0059942F2D010C2F22D
:1031600000000EF011F8059A42F2C831C2F20001D7
:1031700008681043086039E0059942F2D010C2F2A5
:1031800000000EF0E3F9059A42F2C831C2F20001E4
:1031900008689043086029E042F2C830C2F200009B
:1031A00000680599084210D0FFE7059942F2D01057
:1031B000C2F200000EF0CAF9059A42F2C831C2F21A
:1031C00000010868904308600FE0059942F2D010B2
:1031D000C2F200000DF0D8FF059A42F2C831C2F2E7
:1031E0000001086810430860FFE7FFE700208DF842
:1031F0001F00FFE79DF91F0008B080BD00FF7F475B
:1032000080B582B0019001981CF09EFA02B080BD9A
:1032100080B586B004A90291014602988DF8161077
:1032200080ED000A90ED000AB7EE001AB4EE410AF4
:10323000F1EE10FA04DDFFE7FF208DF817006AE0D9
:10324000029890ED000AB5EE400AF1EE10FA03DAAA
:10325000FFE700200490FFE79DF81600014601916A
:1032600020B1FFE70198012815D029E0029890EDE0
:10327000000A42F2F800C2F20000006890ED0B1A5A
:10328000B8EE411A20EE010ABDEEC00A10EE100A97
:10329000ADF80E0014E0029890ED000A42F2B00082
:1032A000C2F20000006890ED0B1AB8EE411A20EE51
:1032B000010ABDEEC00A10EE100AADF80E00FFE7DD
:1032C000BDF80E0001281DDBFFE79DF81600014642
:1032D000009120B1FFE70098012809D011E0BDF866
:1032E0000E0042F2F801C2F200010968486308E0EA
:1032F000BDF80E0042F2B001C2F200010968486355
:10330000FFE704E09DF8160000F02CF8FFE700202E
:103310008DF81700FFE79DF9170006B080BD00008B
:1033200080B582B08DF807009DF807000146009136
:1033300020B1FFE70098012808D00FE042F2F80022
:10334000C2F2000000210DF01FFF07E042F2B000C2
:10335000C2F2000000210DF017FFFFE7002002B0CD
:1033600080BD000080B584B08DF80F009DF80F007F
:103370000146029120B1FFE70298012808D00FE032
:1033800042F2F800C2F2000000210EF0DFF807E080
:1033900042F2B000C2F2000000210EF0D7F8FFE7C1
:1033A00041F20040C4F2020040210022019208F0E4
:1033B0007DF8019804B080BD83B08DF807009DF8BA
:1033C00007000146009120B1FFE70098012806D0D0
:1033D0000BE042F25800C2F20000029008E042F214
:1033E0000000C2F20000029002E000200290FFE71D
:1033F000029803B07047000082B08DF806008DF887
:1034000005100092009820B9FFE7FE208DF8070014
:1034100010E000989DF8062040F24041C2F2000101
:1034200001EB42119DF8052041F8220000208DF8A3
:103430000700FFE79DF9070002B0704783B08DF8E1
:1034400007009DF807000146009140B1FFE7009892
:1034500001280AD0FFE7009802280CD011E042F2C0
:10346000EC20C2F2000002900EE042F2A820C2F26C
:103470000000029008E042F23030C2F200000290F8
:1034800002E000200290FFE7029803B070470000BE
:1034900080B582B00190019800680068C0060028DD
:1034A0002AD5FFE7FFE70020009001980068006838
:1034B000009001980068406800900098FFE701982C
:1034C00016F0A8F800EBC00140F2C040C2F20000C4
:1034D00000EB8100006A70B1FFE7019816F09AF8DE
:1034E00000EBC00140F2C040C2F2000000EB8100DE
:1034F000006A8047FFE7FFE702B080BD82B08DF829
:1035000006008DF805100092009820B9FFE7FE2014
:103510008DF8070012E000989DF8061001EBC1023B
:1035200040F2C041C2F2000101EB82019DF805208A
:1035300041F8220000208DF80700FFE79DF9070001
:1035400002B0704783B080B585B0099308920791A7
:1035500003900020ADF8060007A80290039A029B92
:1035600049F24020C2F2000040F2FF311EF05AFF43
:10357000ADF80600BDF8060001280CDBFFE7BDF83A
:10358000061049F24020C2F2000000F02FF800209F
:103590008DF8130003E0FE208DF81300FFE79DF97E
:1035A000130005B0BDE8804003B0704749F2C01079
:1035B000C2F200000078704780B582B00090009899
:1035C00020B9FFE7FE208DF807000BE0009841F2DC
:1035D000E011C2F20001086000F068FC00208DF8E4
:1035E0000700FFE79DF9070002B080BD80B582B0FB
:1035F0000190ADF8021000208DF80100FFE701985E
:10360000BDF8021000F078FC48B1FFE79DF801001A
:1036100001308DF801000A20FFF766FB00E005E0AD
:10362000FFE79DF801000328E9DBFFE7002002B077
:1036300080BD0000FFE7FEE780B541F21470C2F2E2
:10364000000005F0AFFC80BD80B541F21470C2F2FD
:10365000000005F0A7FC80BD80B541F23C70C2F2CD
:10366000000005F09FFC80BD80B541F23C70C2F2C5
:10367000000005F097FC80BD80B582B0002001906D
:10368000FFF7EEFA019942F66C12C2F200020092C4
:1036900002F11C0305F07CFB0099019B41F2E41050
:1036A000C2F200000068D0F8C8001A461AF0C8FB41
:1036B00002B080BD80B582B001200090FFF7D0FA43
:1036C000009942F69012C2F20002019202F11C032C
:1036D00005F05EFB019941F2E410C2F200000068BF
:1036E000D0F8C80000231A461AF0AAFB02B080BD29
:1036F00083B0029001918DED000A029900200871BB
:1037000000980199086003B07047000080B588B048
:10371000079006910798006805909DED050A9FEDBA
:10372000181A20EE010ABDEEC00A10EE100AADF81C
:10373000120042F6B411C2F2000101914FF404707C
:103740000860002003908860C860082008619DF828
:103750001320084600F8182F0290BDF81200487692
:103760000698D0F8B400C078FFF77AFA0199029A67
:10377000069BC43305F04AF8039808B080BD00BF2B
:103780000000C84282B0019000910098008800EECD
:10379000100AB8EEC00A9FED151A80EE010A0198D2
:1037A00080ED000A0098408800EE100AB8EEC00ACA
:1037B00080EE010A019880ED010A0098808800EEF1
:1037C000100AB8EEC00A80EE010A019880ED020AE4
:1037D0000098C08800EE100AB8EEC00A80EE010A18
:1037E000019880ED030A02B0704700BF0000C84294
:1037F00083B001900091019820B9FFE700208DF877
:103800000B000AE00198006800990840401AB0FADD
:1038100080F040098DF80B00FFE79DF80B0003B026
:103820007047000083B001900091019820B9FFE734
:10383000FE208DF80B0008E0009A0199086890437B
:10384000086000208DF80B00FFE79DF90B0003B026
:103850007047000082B000900098006846F60001B2
:10386000C4F20001884204D1FFE701208DF807006F
:1038700010E00098006846F20041C4F2000188425E
:1038800004D1FFE700208DF8070003E003208DF846
:103890000700FFE79DF8070002B0704780B592B0BF
:1038A00010900F91109820B9FFE7FE208DF8470087
:1038B0007DE042F2B130C2F200000078C00720B1D2
:1038C000FFE7FD208DF8470071E01AF07BFC42F61F
:1038D000DC71C2F20001086020B9FFE7FE208DF81C
:1038E000470064E020202421002204921AF028FAE4
:1038F0001099C1F8C8000F981099C1F8B40005A834
:1039000002902821FCF7B9FC04980A9005900690D3
:103910000B90012103910C91079008900D910E21BD
:1039200001910E910990FFF79BF9029905F092F829
:103930000498FFF795F906F03FF9049843F279628D
:10394000C0F600020621FFF7ABF90498FFF788F9EB
:10395000022104F01FFF019903980A910990FFF7D3
:103960007FF9029905F076F80398FFF779F906F0E8
:1039700023F9039843F2B562C0F600020821FFF76D
:103980008FF90398FFF76CF9102104F003FF0399F6
:103990000498109A41F2E413C2F200031A6042F252
:1039A000B132C2F2000211708DF84700FFE79DF9B5
:1039B000470012B080BD000080B590B08DF83E0089
:1039C0000E910D920E9820B9FFE7FE208DF83F0072
:1039D00013E19DF83E000146079158B1FFE70798B3
:1039E0000138022869D3FFE7079803380228C0F09E
:1039F000A980FDE00E9890ED000A9FED821A20EE5E
:103A0000010ABDEEC00A10EE100AADF832000E98A1
:103A100090ED010A20EE010ABDEEC00A10EE100A78
:103A2000ADF830000E9890ED020A20EE010ABDEECE
:103A3000C00A10EE100AADF82E000E9890ED030AA1
:103A400020EE010ABDEEC00A10EE100AADF82C00FF
:103A500042F6B411C2F2000105914FF40070086003
:103A600000208860C860082008619DF8332008465F
:103A700000F8182F0690BDF8320048769DF8310006
:103A80008876BDF83000C8769DF82F000877BDF81D
:103A90002E0048779DF82D008877BDF82C00C87758
:103AA0000D98D0F8B4000078FFF7DAF80599069A77
:103AB0000D9BB83304F0AAFE9BE00E9890ED040A2B
:103AC0009FED521A20EE010ABDEEC00A10EE100A58
:103AD000ADF82A000E9890ED050A20EE010ABDEE21
:103AE000C00A10EE100AADF8280042F6B411C2F276
:103AF0000001039140F2FF20086000208860C86048
:103B000008220A619DF82B300A4602F8183F0492F9
:103B1000BDF82A204A769DF829208A76BDF828200B
:103B2000CA76087748778877C8770D98D0F8B400B8
:103B30004078FFF795F80399049A0D9BBC3304F085
:103B400065FE56E00E9890ED070A9FED2E1A20EEC6
:103B5000010ABDEEC00A10EE100AADF826000E985C
:103B600090ED080A20EE010ABDEEC00A10EE100A20
:103B7000ADF824000E9890ED090A9FED231A20EE6F
:103B8000010ABDEEC00A10EE100AADF8220042F69E
:103B9000B411C2F20001019140F2FF100860002050
:103BA0008860C86008220A619DF827300A4602F83A
:103BB000183F0292BDF826204A769DF825208A7685
:103BC000BDF82420CA769DF823200A77BDF822206C
:103BD0004A778877C8770D98D0F8B4008078FFF7D7
:103BE0003FF80199029A0D9BC03304F00FFE00E0EC
:103BF000FFE700208DF83F00FFE79DF93F0010B080
:103C000080BD00BF0000804600401C460060EA46C0
:103C100083B00290019101980178407840EA012038
:103C2000ADF8020001980179407940EA0120ADF831
:103C30000000BDF8020000EE100AB8EEC00A9FEDC9
:103C4000191A80EE010A9FED181A20EE010A029857
:103C500080ED000A01988178C07840EA012000B226
:103C600000EE100AB8EEC00A029880ED010ABDF914
:103C7000000000EB8000800000EE100AB8EEC00AE1
:103C80009FED0A1A80EE010A029880ED020A01985F
:103C9000807900EE100AB8EE400A029880ED030A1F
:103CA00003B0704700000046DB0FC94000008046AB
:103CB00080B586B004900391049820B9FFE7FE20F8
:103CC0008DF8170089E0039820B9FFE7FE208DF8F2
:103CD000170082E0039800680190A0F201200428F8
:103CE00017D3FFE70198A0F20520032828D3FFE7A8
:103CF0000198A0F2092002283AD3FFE7019840F288
:103D0000112188424CD0FFE70198B0F5207F53D0B5
:103D10005EE003980068A0F20120029004980299E6
:103D200000EB0110043003991C31FFF771FF029979
:103D3000012000FA01F2049908681043086048E085
:103D400003980068A0F2052002900298811D0120CE
:103D500000FA01F204990868104308600498029977
:103D600000EB0110643003991C31FFF751FF30E084
:103D700003980068A0F2092002900298011D01201A
:103D800000FA01F204990868104308600498029947
:103D900000EB0110443003991C31FFF739FF18E0A4
:103DA0000499086840F40070086004989C300399F6
:103DB0001C31FFF7E7FC0CE00499086840F48060D0
:103DC00008600498AC3003991C3100F00BF800E057
:103DD000FFE700208DF81700FFE79DF9170006B0F8
:103DE00080BD000082B00190009100980178427877
:103DF0008078000440EA0220084400EE100AB8EE81
:103E0000C00A9FED0A1A80EE010A019880ED000AAF
:103E10000098C0780199087100990879497940EAB9
:103E200001200199C88002B0704700BF00007A44A9
:103E300084B08DF80F000291ADF806209DF80F00B8
:103E40000146009123281DD80099DFE801F01213E4
:103E50001415161B1B1B1B1B1B1B1B1B1B1B1B1BC4
:103E60001B1B1B1B1B1B1B1B1B1B1B1B1B1B1718A9
:103E7000191A08E007E006E005E004E003E002E0CC
:103E800001E000E0FFE7002004B070470020704729
:103E900080B541F2B430C2F2000049F2C011C2F262
:103EA000000116F0E5FC002080BD000080B541F265
:103EB000B430C2F2000016F095FC002080BD000076
:103EC00080B582B00190009141F2E010C2F2000092
:103ED000006801211AF096F8002002B080BD0000B1
:103EE00083B0029001918DF8032000208DF802002C
:103EF0009DF9020003B0704780B586B00490ADF81C
:103F00000E1000208DF80D0041F2B430C2F2000016
:103F1000D0F8BC0202900298D0F8140220B1FFE75A
:103F200001208DF8170013E00499BDF80E2041F22E
:103F3000B430C2F20000019016F0B4FC019816F003
:103F40009FFD8DF80D009DF80D008DF81700FFE71F
:103F50009DF8170006B080BD80B588B00690059129
:103F60008DF8132005989DF8131000F08DF88DF84A
:103F7000120005989DF8131000F078F88DF81100E4
:103F80009DF8120010280DD1FFE70698007F00F081
:103F900001008DF810000598807A00F001008DF87E
:103FA0000F0025E09DF8120011280DD1FFE70698BB
:103FB000407F00F001008DF810000598C07A00F0F5
:103FC00001008DF80F0012E00698C08B9DF81210CA
:103FD000C84000F001008DF81000059840889DF859
:103FE0001210C84000F001008DF80F00FFE7FFE756
:103FF0009DF811000146029140B1FFE702980128A7
:1040000017D0FFE70298022824D02AE09DF810106C
:104010000020C907019031B1FFE79DF80F0080F043
:1040200001000190FFE7019800F001008DF81F00EA
:1040300017E09DF810100020C907009021B9FFE794
:104040009DF80F000090FFE7009800F001008DF848
:104050001F0006E09DF8100000F001008DF81F0021
:10406000FFE79DF81F0008B080BD000082B00190FE
:104070008DF80310019800699DF8031000EB4100D2
:10408000007A02B07047000082B001908DF80310F2
:10409000019800699DF8031000EB4100407A02B0DE
:1040A0007047000081B000900098407800F0010057
:1040B00001B0704783B001900091019820B9FFE7EB
:1040C000FF208DF80B000FE0009820B9FFE7FF20DC
:1040D0008DF80B0008E00199002008700099019A02
:1040E00011618DF80B00FFE79DF90B0003B07047DD
:1040F00083B001908DF803109DF80300102807D1BC
:10410000FFE70198007F00F001008DF80B0015E03B
:104110009DF80300112807D1FFE70198407F00F0C8
:1041200001008DF80B0009E00198C08B9DF8031089
:10413000C84000F001008DF80B00FFE79DF80B0070
:1041400003B0704784B0029001918DED000A02988F
:1041500020B9FFE7FF208DF80F003EE0019820B95D
:10416000FFE7FF208DF80F0037E002980068019903
:104170008862029840680199C8620298C0680199F3
:104180008861029800690199C861029840690199A3
:1041900008620298407EC00720B1FFE70199042021
:1041A000087503E0019902200875FFE70298007E78
:1041B000C00748B1FFE70199022081F83400019956
:1041C000012081F8360004E00199012081F83400D3
:1041D000FFE700208DF80F00FFE79DF90F0004B006
:1041E0007047000080B584B0029001918DED000A07
:1041F000029820B9FFE7FF208DF80F0056E00198E4
:1042000020B9FFE7FF208DF80F004FE0029804214E
:10421000FFF76EFF80B1FFE702980521FFF768FF07
:1042200050B1FFE702980621FFF762FF20B1FFE7D8
:10423000019901200870FFE702980421FFF758FF59
:1042400080B1FFE702980521FFF752FF50B1FFE769
:1042500002980721FFF74CFF20B1FFE701990020EA
:104260000870FFE70298407D20B1FFE70298007DCB
:1042700020B9FFE7019800F03DFA13E001980078BB
:10428000C00738B1FFE7029801999DED000A00F0E0
:1042900011F806E0029801999DED000A00F08CF9F2
:1042A000FFE7FFE700208DF80F00FFE79DF90F0003
:1042B00004B080BD80B584B0039002918DED010AF9
:1042C0000299012081F824000398B0F9160000EE4D
:1042D000100AB8EEC00A9DED011A20EE010A0298FC
:1042E000016991ED001A20EE010A80ED0A0A039897
:1042F000B0F91800404200EE100AB8EEC00A9DED79
:10430000011A20EE010A0298016991ED001A20EECF
:10431000010A80ED0B0A02980022C26102988261B4
:10432000029880F8382003980299FFF715FE58B1DB
:10433000FFE70298016991ED091A90ED070A30EE46
:10434000010A80ED070AFFE7039802990122FFF7AF
:1043500003FE58B1FFE70298016991ED091A90ED4B
:10436000070A30EE410A80ED070AFFE70398029939
:104370000222FFF7F1FD58B1FFE70298016991EDC4
:10438000091A90ED060A30EE410A80ED060AFFE7B1
:10439000039802990322FFF7DFFD58B1FFE7029867
:1043A000016991ED091A90ED060A30EE010A80EDDF
:1043B000060AFFE7039802990422FFF7CDFDA8B192
:1043C000FFE70298016991ED0A1A90ED060A20EEC6
:1043D000010A80ED060A0298016991ED0A1A90ED32
:1043E000070A20EE010A80ED070AFFE70398029909
:1043F0000522FFF7B1FDA8B1FFE70298016991ED31
:104400000B1A90ED060A20EE010A80ED060A0298CA
:10441000016991ED0B1A90ED070A20EE010A80ED7B
:10442000070AFFE7039802990622FFF795FD48B1B6
:10443000FFE70299022081F834000299012081F8F7
:10444000360008E00299022081F834000299002029
:1044500081F83600FFE7039802990722FFF77CFDF9
:10446000B0B1FFE7029991F83500013081F83500CD
:10447000029991F835004AF6AB22CAF6AA22A0FBAF
:104480000232520802EB4202801A81F83500FFE73F
:10449000039802990B22FFF75FFD38B1FFE70299FD
:1044A00004200875029902204875FFE703980299D5
:1044B0000A22FFF751FD40B1FFE7029991F837203A
:1044C0000120904381F83700FFE703980299082202
:1044D000FFF742FD20B3FFE70298007B02280BD1D3
:1044E000FFE702983930042100F012F90299002008
:1044F00048700299087312E00298007B012801D1EC
:10450000FFE70BE002983930032100F001F902992E
:1045100002200873029901204870FFE7FFE7FFE7D8
:10452000039802990922FFF717FDD8B1FFE7029817
:10453000007B01280BD1FFE7029900204870029907
:10454000087302983930022100F0E2F809E002987D
:1045500001210173029841700298393000F0D8F8B7
:10456000FFE703E0029900204870FFE703980299F3
:104570000C22FFF7F1FC28B1FFE70299012081F836
:104580003800FFE7039802990D22FFF7E5FC20B100
:10459000FFE7029902200875FFE70398C08B029994
:1045A00048800299039AD2F81600D2F81A208A603D
:1045B000486004B080BD000085B0049003918DED8B
:1045C000020A0498407D01460191032828D80199E8
:1045D000DFE801F01E02140B03990120087503990E
:1045E00000200873039948701AE0039902200875A7
:1045F0000399002008730399487011E00399002083
:10460000487503990420087303990120487007E056
:104610000399002008750399087303994870FFE710
:104620000498007D01460091032831D80099DFE805
:1046300001F02702170A0399012081F82400039949
:1046400081F8340024E00399012081F824000399C3
:10465000002081F836000399022081F8340017E029
:104660000399012081F82400039A022182F8341072
:10467000039A002182F83510039981F8360007E08B
:104680000399002081F82400039981F83400FFE7A2
:104690000398007B28B1FFE703984078C00738BB38
:1046A000FFE70498006803998861049840680399BB
:1046B000C861049890ED020A9DED021A20EE010AED
:1046C0000398016991ED011A20EE010A80ED0A0AB2
:1046D000049890ED030A9DED021A20EE010A03985A
:1046E000016991ED011A20EE010A80ED0B0AFFE746
:1046F00005B0704781B000900099002008750099BE
:1047000081F82400009981F8340001B0704700005E
:1047100083B001908DF80310019820B9FFE7FF20C6
:104720008DF80B001BE00198C078022806DCFFE73B
:104730000198C078B0F1FF3F04DCFFE7FF208DF85F
:104740000B000CE09DF803000199CA788854019988
:10475000C8780130C87000208DF80B00FFE79DF984
:104760000B0003B07047000081B0ADF802008DF877
:104770000110BDF802109DF801004840C2B244F695
:10478000B030C0F6020030F8120080EA112001B00B
:104790007047000080B584B003900291ADF8062008
:1047A000FFE70298411E029158B1FFE7BDF80600ED
:1047B00003994A1C03920978FFF7D6FFADF806006B
:1047C000EFE7BDF8060004B080BD000080B584B0FE
:1047D000029001910198012804D8FFE700208DF88C
:1047E0000F001BE00298019902394FF6FF72FFF7A4
:1047F000D1FFADF80200BDF80200029A019901F064
:1048000001031A4421F00101114431F8021C401A3D
:10481000B0FA80F040098DF80F00FFE79DF80F0017
:1048200004B080BD83B0029001918DF80320FFE7B2
:104830000198411E019178B1FFE79DF803000299AC
:104840004A1C02920978414044F6B050C0F602007A
:10485000405C8DF80300EBE79DF8030003B0704760
:1048600080B584B0029001910198012804D8FFE737
:1048700000208DF80F0015E0029801990139FF2200
:10488000FFF7D0FF8DF803009DF80300029A01990D
:10489000114411F8011C401AB0FA80F040098DF85B
:1048A0000F00FFE79DF80F0004B080BD85B002A99E
:1048B00000910146009880ED010AC0ED000A8DF8D4
:1048C000071090ED010AB5EE400AF1EE10FA03D19F
:1048D000FFE7002004906DE09DF80700C007A0B33B
:1048E000FFE7009890ED010AB2EE0E1AB4EE410A0D
:1048F000F1EE10FA06D1FFE74FF20000C4F291503A
:10490000049057E0009890ED010AB3EE021AB4EE5D
:10491000410AF1EE10FA06D1FFE748F20000C4F2B6
:10492000A250049046E0009890ED010AB3EE0E1AF2
:10493000B4EE410AF1EE10FA06D1FFE74BF20000A7
:10494000C4F2E550049035E022E0009890ED010AB1
:10495000B2EE041AB4EE410AF1EE10FA06D1FFE706
:1049600041F20000C4F28B50049023E0009890EDD7
:10497000010AB3EE001AB4EE410AF1EE10FA06D1C4
:10498000FFE744F20000C4F2B550049012E0FFE7E4
:10499000009890ED010A9FED0A1A20EE010A90EDB1
:1049A000001A9FED082A21EE021A80EE010A80ED1E
:1049B000020AFFE7009890ED020A05B0704700BFB9
:1049C00000007042DB0FC94080B584B003900291B3
:1049D000019202980078012805D0FFE702988068CC
:1049E000019908600CE0029890ED010AD0ED020AEE
:1049F00090ED031A0FF04EFD019880ED000AFFE7DD
:104A00000399012008710398D0ED020A90ED030A82
:104A1000B2EE081A00F0BAF8039880ED000A04B06C
:104A200080BD000082B0019000910198006800995B
:104A30000860019800790099087102B07047000081
:104A400084B08DED030A9DED030A20EE000A8DED82
:104A5000010A9DED010A9DED031A20EE010A8DED7C
:104A6000000A9DED030A9FED3E1AB4EE410AF1EEF5
:104A700010FA03DAFFE70020029053E09DED030AED
:104A80009FED381AB4EE410AF1EE10FA1DDAFFE795
:104A90009DED000A9FED391A20EE010A9DED011AE5
:104AA0009FED372A21EE021A30EE010A9DED031A1E
:104AB0009FED342A21EE021A30EE010A9FED321AE0
:104AC00030EE010A8DED020A2BE09DED030A9FED09
:104AD000261AB4EE410AF1EE10FA1DDAFFE79DED59
:104AE000000A9FED221A20EE010A9DED011A9FEDAA
:104AF000202A21EE021A30EE010A9DED031A9FEDE5
:104B00001D2A21EE021A30EE010A9FED1B1A30EE2B
:104B1000010A8DED020A03E04FF07E500290FFE79C
:104B2000FFE7FFE79DED020AB5EE400AF1EE10FA4D
:104B300003DAFFE7002002900EE09DED020AB7EED7
:104B4000001AB4EE410AF1EE10FA04DDFFE74FF06F
:104B50007E500290FFE7FFE79DED020A04B0704728
:104B600000009C413333AF410000CC4161E0B93CCF
:104B700046B6D3BF295C21423333A4C31399B93B52
:104B8000FB5CADBEE17AD84014AE34C284B08DED8A
:104B9000030ACDED020A8DED011A9DED030A9DED8C
:104BA000012A30EE420A9DED021A31EE421A80EEE1
:104BB000010A8DED000A9DED000AB5EE400AF1EE06
:104BC00010FA03DAFFE7002000900EE09DED000AE6
:104BD000B7EE001AB4EE410AF1EE10FA04DDFFE779
:104BE0004FF07E500090FFE7FFE79DED000A04B014
:104BF000704700000000000080B588B08DED070A06
:104C0000CDED060A05909DED050AB8EE400A10EEBE
:104C1000100AFBF7BFFC41EC100B9FED2B1B53EC74
:104C2000112B51EC100BFBF713FC41EC100B51EC6A
:104C3000100BFBF7C2FC00EE100A1EF03DFA9FEDD0
:104C4000261A20EE010A10EE100AFBF7A3FC41EC35
:104C5000100B51EC100B9FED1E0B52EC103BD20FC2
:104C600062F3DF7141EC100B8DED020B0798FBF73F
:104C700091FC9DED021B41EC100B51EC110B53EC20
:104C8000102BFBF73EFB41EC100B51EC100BFBF72C
:104C900094FC04909DED040A9FED101AB4EE410AB5
:104CA000F1EE10FA05DDFFE79DED060A8DED010A34
:104CB00004E09DED040A8DED010AFFE79DED010A78
:104CC00008B080BD00BF00BFFCA9F1D24D62503FCB
:104CD0000000000000000000CDCC4C3ECDCC4C3F8D
:104CE00080B58EB007AB05930C900B910A920C988F
:104CF00020B9FFE7FE208DF8370067E10B9820B957
:104D0000FFE7FE208DF8370060E10A990C980268F1
:104D1000891A00EE101AB8EE400A9FEDAE1A80EE26
:104D2000010A80ED010A0A980C9908600C980B9909
:104D300009780A9A00F02EFB0C98007C0146049139
:104D400000B3FFE7049801280DD0FFE7049802386C
:104D5000032817D3FFE7049805280AD0FFE7049833
:104D600006280FD04CE00C99002048610C9988610E
:104D700046E00B9840680C9948610B9840680C9984
:104D800088613DE005980C9991ED080AC96891ED9C
:104D9000001A30EE410A80ED020A90ED020A1EF080
:104DA00047F8059880ED010A90ED020A1EF084F99B
:104DB000059880ED000A90ED010A0B9991ED011A1A
:104DC00091ED022A20EE010A90ED001A21EE021A5E
:104DD00030EE410A0C9981ED050A90ED000A0B991D
:104DE00091ED011A91ED022A20EE010A90ED011ACF
:104DF00021EE021A30EE010A0C9880ED060AFFE758
:104E00000C98007C01460391062848D80399DFE8F6
:104E100001F00404081A300408000C990020C8614D
:104E20003DE00C9901F13800CA6892ED000AD1ED1D
:104E3000011AD1ED080A9FED6B1A0FF091F80C984A
:104E400080ED070A2BE00C9901F13800CA6892ED59
:104E5000000A9FED631A30EE010AD1ED011AD1ED7F
:104E6000080A9FED601A0FF07BF80C9880ED070A96
:104E700015E00C9890ED0B0A8DED020A0A989FED53
:104E8000560ADFED560AFFF7B7FEB0EE401A9DED69
:104E9000020A20EE010A0C9880ED070AFFE70C9B3E
:104EA00003F1120003F114011A6B93F911309FED15
:104EB0004E0A0EF0D9FC00208DF81B00FFE79DF88C
:104EC0001B000C9991F9111088427BDAFFE70C98CE
:104ED000416A406F9DF81B2000EB421001EB8201FC
:104EE00091ED000A0DF02CFC0C98406A9DF81B1007
:104EF00000EB810080ED000A0C98007C01460191D6
:104F0000E0B3FFE701980138052804D3FFE70198D3
:104F1000062821D03AE00C99486B9DF81B30C3EB72
:104F2000031200EB82000A6B02EB830292ED000A8F
:104F30004A6A02EB8302D2ED000AD1ED011A9FED1D
:104F4000291A0FF00DF80C98C06F9DF81B1000EB9C
:104F5000810080ED000A19E00C989DF81B10026B8F
:104F6000C06F02EB810292ED000A9FED201A80EEE5
:104F7000010A00EB810080ED000A07E00C98C16F88
:104F80009DF81B20002041F82200FFE70C999DF8B6
:104F90001B20886FC96F00EB421001EB820191ED7D
:104FA000000A0DF0CDFB0C98C06F9DF81B1000EBB4
:104FB000810080ED000AFFE79DF81B0001308DF8AD
:104FC0001B007CE700208DF83700FFE79DF93700D4
:104FD0000EB080BD00007A449A99193FCDCC4C3F69
:104FE000AB611C3F0000000000C0DA4500A00C4689
:104FF00083B00290019100208DF80300FFE79DF837
:105000000300029991F91110884210DAFFE7029823
:10501000C06F9DF8032050F82200019941F822004A
:10502000FFE79DF8030001308DF80300E7E703B0C8
:105030007047000082B0019000910198007C0099B7
:105040000870019890ED080AC06890ED001A30EEE3
:10505000410A009880ED010A02B0704780B58AB01D
:1050600005AB03930346039808930791069280EDDE
:10507000000A089820B9FFE7FE208DF827001CE100
:10508000079808998860089900200874069808997C
:10509000C860079890F84C00C00728B1FFE708984F
:1050A000C06800F0DBFAFFE70898806800780146E6
:1050B0000291062832D80299DFE801F0040B121899
:1050C0001F2C250008990420487400208DF8130037
:1050D00024E008990420487401208DF813001DE095
:1050E0000899022048748DF8130017E008990420ED
:1050F000487403208DF8130010E0089904204874C8
:105100008DF813000AE008990120487405208DF8F5
:10511000130003E0FC208DF82700CEE0089890F9FA
:1051200011008000FEF76CF8089948620898406A00
:1051300008B9FFE7A5E0089890F911008000FEF794
:105140005FF8089988620898806A08B9FFE798E0D4
:10515000089890F911008000FEF752F8089908634A
:105160000898006B08B9FFE78BE0089890F91100E8
:10517000C0EB00108000FEF743F8089948630898D8
:10518000406B08B9FFE77CE0089890F911008000B7
:10519000FEF736F80899C8670898C06F08B9FFE7A6
:1051A0006FE0089890F911004001FEF729F808997E
:1051B00048670898406F08B9FFE762E0089890F9DF
:1051C00011004001FEF71CF8089988670898806F65
:1051D00008B9FFE755E000208DF81200FFE79DF8C1
:1051E0001200089991F91110884233DAFFE7039A07
:1051F00008988168406B9DF81230C3EB031300EBF5
:10520000830092ED000A0A1D00210FF021F8039A95
:1052100008988168406F9DF8123000EB431092EDC2
:10522000000AD1ED110A0DF0E7FA039A0898816897
:10523000806F9DF8123000EB431092ED000AD1ED23
:10524000120A0DF0D9FAFFE79DF8120001308DF82F
:105250001200C4E7039A089901F1380092ED000AA0
:10526000896801F12402002101910EF0F1FF0898F4
:1052700012309DF813100EF049FC01988DF82700AC
:105280001BE00898406AFDF7CFFD0898006BFDF71A
:10529000CBFD0898406BFDF7C7FD0898C06FFDF780
:1052A000C3FD0898406FFDF7BFFD0898806FFDF7BC
:1052B000BBFDFE208DF82700FFE79DF927000AB00F
:1052C00080BD000080B584B003900291019200205F
:1052D000009001980078012805D0FFE70020C4F273
:1052E000FA40009042E002980079012833D1FFE7AC
:1052F000029890ED000A9FED231AB4EE410AF1EEF8
:1053000010FA28DDFFE7029890ED000AB7EE001AC8
:10531000B4EE410AF1EE10FA05DDFFE70020CBF60E
:105320008070009016E0019890ED010A029890EDCF
:10533000001A9FED152A31EE021A9FED142A81EE14
:10534000021A9FED132A21EE021A30EE010A8DEDAA
:10535000000AFFE709E0019890ED010AD0ED020A8A
:105360000FF048F98DED000AFFE7FFE79DED000A19
:10537000039A516AD06F92F911200FF0C7F80020FC
:1053800004B080BD9A99993E9A9999BE3333333FC0
:105390000000C84280B586B004908DF80F100292CC
:1053A000049820B9FFE7FE208DF8170066E09DF80D
:1053B0000F000499097C884204D1FFE700208DF892
:1053C00017005BE09DF80F0004281CD1FFE704984C
:1053D000007C042817D0FFE70298FAF72DFFFAF7B0
:1053E00021FF00EBD07121F00101411A01200029B9
:1053F00018BF4FF0FF3000EE100AB8EEC00A049854
:1054000080ED0B0AFFE700208DF80700FFE79DF80D
:105410000700049991F91110884227DAFFE70498F0
:10542000406B9DF80710C1EB011100EB81000EF0FD
:10543000DBFF0498406F9DF8071000EB41109FEDD3
:10544000110A8DED000A0DF075FA9DED000A049821
:10545000806F9DF8071000EB41100DF06BFAFFE72D
:105460009DF8070001308DF80700D0E79DF80F0088
:105470000499087400208DF81700FFE79DF91700C4
:1054800006B080BD0000000084B002900191029837
:1054900020B9FFE7FE208DF80F0048E0019820B901
:1054A000FFE7FE208DF80F0041E00298806890F839
:1054B0004C00C00758B1FFE7019890ED111A9FED1D
:1054C0001E0A30EE410A029880ED080A04E00198B5
:1054D000406C02990862FFE700208DF80300FFE7A7
:1054E0009DF80300029991F9111088421BDAFFE739
:1054F00001989DF8032000EB021080680299496A28
:1055000041F8220001989DF8032000EB0210C068CA
:105510000299896A41F82200FFE79DF803000130F3
:105520008DF80300DCE700208DF80F00FFE79DF900
:105530000F0004B0704700BFDB0FC94084B0039078
:105540008DED020ACDED010A039890ED000A9DED64
:10555000021A30EE010A8DED000A9DED010AB5EE4A
:10556000400AF1EE10FA26DDFFE79DED000A9DED01
:10557000011AB4EE410AF1EE10FA09DBFFE79DEDE6
:10558000011A9DED000A30EE410A8DED000A11E08E
:105590009DED000AB5EE400AF1EE10FA09DAFFE7D8
:1055A0009DED011A9DED000A30EE010A8DED000A15
:1055B000FFE7FFE7FFE700980399086004B0704732
:1055C00085B08DED040ACDED030A8DED021A9DED37
:1055D000040A9DED031A30EE410A8DED010A9DED9E
:1055E000020AB5EE400AF1EE10FA32DDFFE79DED5A
:1055F000020AB0EE001A80EE010A8DED000A9DED60
:10560000010A9DED001AB4EE410AF1EE10FA09DD2F
:10561000FFE79DED021A9DED010A30EE410A8DED86
:10562000010A15E09DED010A9DED001AB1EE411A47
:10563000B4EE410AF1EE10FA09DAFFE79DED021A25
:105640009DED010A30EE010A8DED010AFFE7FFE74B
:10565000FFE79DED010A05B07047000081B00090A2
:10566000009890ED001A9FED040A30EE410A80ED9B
:10567000000A01B0704700BFDB0FC94083B0029041
:105680008DED010ACDED000A029890ED000A9DED26
:10569000001AB4EE410AF1EE10FA04DDFFE70098BB
:1056A00002990860FFE7029890ED000A9DED011A4B
:1056B000B4EE410AF1EE10FA04DAFFE7019802991C
:1056C0000860FFE703B0704780B5B4B03290319105
:1056D0003092329818B9FFE700203390FDE13198FD
:1056E000013831900020ADF84E0040F26030C2F237
:1056F0000000007801461291072800F2C881129933
:10570000DFE811F008001A002C0097003601610153
:10571000A301B4013298319945F61852C0F602023D
:105720001CF052FE40F26031C2F2000108780130F4
:10573000087001203390D0E13298319945F6464205
:10574000C0F602021CF040FE40F26031C2F20001DD
:1057500008780130087001203390BEE142F61C60E9
:10576000C2F200001190C06818F01CFE1198806B06
:1057700014A90022052318F083FAC0B1FFE732987C
:10578000319945F61842C0F602021CF01DFE40F2A7
:105790006031C2F200010720087042F61C60C2F2BC
:1057A0000000C06818F0DEFD0120339095E142F65C
:1057B0001C60C2F20000C06818F0D4FD14A8FCF709
:1057C000F1FE90B1FFE73298319945F6EE42C0F60E
:1057D00002021CF0F9FD40F26031C2F200010878CB
:1057E000013008700120339077E140F26130C2F25D
:1057F0000000017801310170007802280FDCFFE71A
:105800003298319945F66442C0F602021CF0DCFD84
:1058100040F26031C2F200010120087006E040F25F
:105820006031C2F2000107200870FFE701203390C9
:1058300053E13298319945F63952C0F602021CF014
:10584000C3FD17A8109000F01BFF109800212991AC
:105850002A912B9100F0D2FFFFE7BDF84E00B0F582
:105860007A7F4BDAFFE742F61C60C2F20000806BE1
:1058700014A90F910022052318F002FA01460F988F
:10588000B1FA81F149098DF84D10FCF78BFE8DF8C6
:105890004C009DF84D00C00778B3FFE79DF84C0021
:1058A000C00750B3FFE79DED141A40F26430C2F216
:1058B000000090ED000A30EE010A80ED000A9DED37
:1058C000151A40F26830C2F2000090ED000A30EE86
:1058D000010A80ED000A9DED161A40F26C30C2F20A
:1058E000000090ED000A30EE010A80ED000ABDF8DC
:1058F0004E000130ADF84E00FFE7AEE7BDF84E00B8
:1059000000EE100AB8EE401A40F26430C2F2000015
:1059100090ED000A80EE010A80ED000ABDF84E000D
:1059200000EE100AB8EE401A40F26830C2F20000F1
:1059300090ED000A80EE010A80ED000ABDF84E00ED
:1059400000EE100AB8EE401A40F26C30C2F20000CD
:1059500090ED000A80EE010A80ED000A40F260310D
:10596000C2F2000108780130087001203390B4E0E1
:105970003298319945F6C042C0F602021CF024FD6F
:1059800017A80E9000F07CFE0E9840F26431C2F22F
:1059900000010968299140F26831C2F200010968EA
:1059A0002A9140F26C31C2F2000109682B9100F09B
:1059B00025FF40F26031C2F2000108780130087022
:1059C0000120339089E032980C9031980D9040F28C
:1059D0006430C2F200000068FAF7DCFD41EC100B05
:1059E0008DED0A0B40F26830C2F200000068FAF751
:1059F000D1FD41EC100B8DED080B40F26C30C2F282
:105A000000000068FAF7C6FD9DED081B9DED0A0B2E
:105A100002460C980B460D9943EC122B6A4682ED18
:105A2000042B82ED021B82ED000B45F67C52C0F682
:105A300002021CF0C9FC40F26031C2F20001087899
:105A4000013008700120339047E03298319945F6D3
:105A5000AD42C0F602021CF0B7FC40F26031C2F267
:105A60000001082008700120339036E03298319907
:105A700045F63142C0F602021CF0A6FC40F260314D
:105A8000C2F20001082008700120339025E040F2A6
:105A90006431C2F2000100200790086040F26831D2
:105AA000C2F20001086040F26C31C2F200010860ED
:105AB00040F26131C2F2000108703298319945F626
:105AC0004C62C0F602021CF07FFC079840F2603185
:105AD000C2F2000108703390FFE7339834B080BD04
:105AE00080B5B0B02E902D912C922E9818B9FFE76A
:105AF00000202F9060E22D9801382D902C980121E4
:105B00002BAA01F081FC28902C9802212AAA01F0EE
:105B10007BFC27902C98032129AA01F075FC269084
:105B200028982B9A45F25B51C0F60201FAF7DAFB8E
:105B3000A0B9FFE72E982D9945F69872C0F602029B
:105B400045F61F03C0F602031CF03EFC40F2703124
:105B5000C2F20001002008702F902DE228982B9AA5
:105B600045F6B671C0F60201FAF7BCFB00285BD11E
:105B7000FFE7279818B9FFE7269808B1FFE70BE27F
:105B800040F27030C2F20000007801460A9120B164
:105B9000FFE70A98012810D045E02E982D9945F688
:105BA000CB62C0F602021CF00FFC40F27031C2F270
:105BB0000001012008702F90FEE10DA809906421DA
:105BC000FAF75BFB45F20B60C0F60200089000F0AC
:105BD0009DFD189045F20E60C0F60200069000F0A0
:105BE000D7FD069A014609981791142107911CF0D8
:105BF000EBFB0799089A099814301CF0E5FB09980B
:105C000000F0FCFD2E982D9945F68762C0F6020241
:105C10001CF0DAFB40F27031C2F200010220087081
:105C200001202F90C8E19DE128982B9A45F6C77175
:105C3000C0F60201FAF756FB002840F0CF80FFE7DC
:105C4000279818B1FFE7269808B1FFE7A4E1279845
:105C50002A9A45F6C171C0F60201FAF743FB002803
:105C600057D1FFE700F088FD0C9040F27030C2F28F
:105C7000000000780146059120B1FFE70598012852
:105C800010D045E02E982D9945F63672C0F60202E6
:105C90001CF09AFB40F27031C2F200010120087042
:105CA0002F9089E10C9840F27131C2F2000109781D
:105CB00050F83100E0B1FFE72E982D990C9A40F290
:105CC0007133C2F2000304931B7852F8333045F667
:105CD0009472C0F602021CF077FB04990878013038
:105CE000087040F27031C2F20001012008700CE02F
:105CF00040F27131C2F200010020087040F27031B0
:105D0000C2F2000102200870FFE701202F9053E14A
:105D100063E027982A9A45F6BB71C0F60201FAF7AC
:105D2000E1FA002857D1FFE700F02CFD0B9040F27C
:105D30007030C2F2000000780146039120B1FFE705
:105D40000398012810D045E02E982D9945F64D7204
:105D5000C0F602021CF038FB40F27031C2F20001C2
:105D6000012008702F9027E10B9840F27131C2F2A8
:105D70000001097850F83100E0B1FFE72E982D9925
:105D80000B9A40F27133C2F2000302931B7852F86F
:105D9000333045F69472C0F602021CF015FB0299EE
:105DA00008780130087040F27031C2F20001012021
:105DB00008700CE040F27131C2F20001002008705E
:105DC00040F27031C2F2000102200870FFE70120AA
:105DD0002F90F1E000E0DFE0FFE7C2E028982B9A87
:105DE00045F6A171C0F60201FAF77CFA002840F0EE
:105DF000B780FFE7279818B1FFE7269808B9FFE7B3
:105E0000CAE027982A9A45F6BB71C0F60201FAF754
:105E100069FA00283ED1FFE740F27030C2F200007C
:105E20000078B0BBFFE70DA800F02AFC269800F030
:105E3000AFFC88B9FFE72E982D9945F68F62C0F622
:105E400002021CF0C1FA40F27031C2F200010220DD
:105E5000087001202F90AFE02E982D9945F64F62E3
:105E6000C0F602021CF0B0FA269B45F69872C0F606
:105E700002020DA8019014211CF0A6FA019800F06E
:105E8000BDFC40F27031C2F20001012008702F9079
:105E900092E04BE027982A9A45F6C171C0F60201BC
:105EA000FAF720FA00283FD1FFE740F27030C2F243
:105EB00000000078B8BBFFE70DA800F0E1FB2698D2
:105EC00000F024FC88B9FFE72E982D9945F61E7244
:105ED000C0F602021CF078FA40F27031C2F2000102
:105EE0000220087001202F9066E02E982D9945F62B
:105EF0004F62C0F602021CF067FA0DA80090143041
:105F0000269B45F69872C0F6020214211CF05CFA3A
:105F1000009800F073FC40F27031C2F200010120E1
:105F200008702F9048E000E036E0FFE740F2703064
:105F3000C2F200000078012811D1FFE72E982D99B8
:105F400045F6F162C0F602021CF03EFA40F27031F2
:105F5000C2F200010220087001202F902CE0FFE720
:105F6000FFE7FFE7FFE740F27030C2F20000007881
:105F7000022810D1FFE72E982D9945F25652C0F60F
:105F800002021CF021FA40F27031C2F2000100203E
:105F900008702F9010E0FFE72E982D9945F6B93242
:105FA000C0F602021CF010FA40F27031C2F2000199
:105FB000002008702F90FFE72F9830B080BD0000C0
:105FC00080B588B0069005910492069818B9FFE74D
:105FD000002007908DE005980138059042F21120CD
:105FE000ADF80E00BDF80E00ADF80C009DF80E00E7
:105FF0009DF80F1040EA0120ADF80A0040F272301F
:10600000C2F20000007801460191032861D801998D
:10601000DFE801F00214283C0698059945F639623C
:10602000C0F602021CF0D0F940F27231C2F2000157
:10603000087801300870012007905AE00698059909
:10604000BDF80C3045F60C62C0F602021CF0BCF93B
:1060500040F27231C2F2000108780130087001206C
:10606000079046E006980599BDF80A3045F6DF52DC
:10607000C0F602021CF0A8F940F27231C2F200012F
:106080000878013008700120079032E0BDF80C005C
:10609000BDF80A10884209D1FFE70698059945F630
:1060A000C752C0F602021CF08FF908E00698059965
:1060B00045F6BA52C0F602021CF086F9FFE740F23C
:1060C0007231C2F200010878013008700120079097
:1060D0000FE00698059945F64C62C0F602021CF0E6
:1060E00073F940F27231C2F200010020087007908B
:1060F000FFE7079808B080BD80B5DAB05890579197
:106100005692589818B9FFE700205990C9E057985F
:106110000138579040F27330C2F200000078014617
:106120000991042800F2AD800999DFE801F0032409
:10613000778899000AA800F0A3FA58980790579812
:1061400008902298FAF726FA024607980B46089913
:1061500043EC102B6A4682ED000B45F6AA52C0F6BE
:1061600002021CF031F940F27331C2F20001012049
:106170000870599095E042F61C60C2F2000006904B
:10618000C06818F00FF90698406F23A900220A236F
:1061900017F076FD80B1FFE742F61C60C2F2000006
:1061A000C06818F0DFF840F27331C2F2000103203A
:1061B00008700120599074E00AA8039000F060FA7A
:1061C00042F61C60C2F20000C06818F0CBF80398D9
:1061D0003899229100F012FB039800F051FA589878
:1061E0000490579805902298FAF7D4F9024604983B
:1061F0000B46059943EC102B6A4682ED000B45F6E1
:106200007A62C0F602021CF0DFF840F27331C2F28B
:106210000001022008700120599042E058985799D7
:1062200045F6F162C0F602021CF0CEF840F273317E
:10623000C2F20001052008700120599031E0589801
:10624000579945F6E932C0F602021CF0BDF840F25B
:106250007331C2F20001052008700120599020E03E
:106260005898579945F6A762C0F602021CF0ACF8A0
:1062700040F27331C2F200010520087001205990EC
:106280000FE05898579945F64C62C0F602021CF090
:106290009BF840F27331C2F200010020087059905F
:1062A000FFE759985AB080BD80B5E2B060905F9129
:1062B0005E92609818B9FFE700206190C2E05F9895
:1062C00001385F9040F27430C2F20000007801465D
:1062D000119148B1FFE71198012817D0FFE71198F5
:1062E000022800F08E809DE060985F9945F6535239
:1062F000C0F602021CF068F840F27431C2F20001EC
:10630000087801300870012061909BE012A800F02D
:10631000B7F942F61C60C2F200001090C06818F095
:1063200041F81098406F2BA90022052317F0A8FC14
:10633000C0B1FFE760985F9945F6FD32C0F60202F2
:106340001CF042F840F27431C2F2000102200870E1
:1063500042F61C60C2F20000C06818F003F8012089
:1063600061906FE042F61C60C2F20000C06817F056
:10637000F9FF3C9827904098289012A800F03EFA28
:1063800060980E905F980F90279828990691299908
:106390000891FAF7FFF80246069807920A4607990D
:1063A00042EC101B8DED0C0BFAF7F4F8024608983E
:1063B00009920A46099942EC101B8DED0A0BFAF777
:1063C000E9F89DED0A1B9DED0C0B02460E980B465D
:1063D0000F9943EC122B6A4682ED042B82ED021BCF
:1063E00082ED000B45F65A62C0F602021BF0ECFF8C
:1063F00040F27431C2F20001032008700120619064
:1064000020E060985F9945F63142C0F602021BF029
:10641000DBFF40F27431C2F200010320087001205A
:1064200061900FE060985F9945F64C62C0F60202F9
:106430001BF0CAFF40F27431C2F200010020087064
:106440006190FFE7619862B080BD000080B596B0B2
:10645000149013911292149818B9FFE70020159028
:106460000AE113980138139040F27530C2F200002F
:10647000007801460A91092800F2EE800A99DFE8C7
:1064800001F00517243643557385BCCE1498139A32
:1064900045F61C11C0F60201F9F7FAFE40F275311B
:1064A000C2F2000108780130087001201590E3E085
:1064B00014981AF04BF840F27531C2F200010878D6
:1064C0000130087001201590D6E01498139A45F613
:1064D000AB21C0F60201F9F7DBFE40F27531C2F2E2
:1064E000000108780130087001201590C4E014986C
:1064F00019F09AFF40F27531C2F2000108780130BC
:10650000087001201590B7E01498139A45F6AB1166
:10651000C0F60201F9F7BCFE40F27531C2F200018B
:1065200008780130087001201590A5E00BA819F03B
:1065300097FC149813990B9AC2F5C04C6B46C3F89C
:1065400004C01A6045F69652C0F602024FF4C043EA
:106550001BF03AFF40F27531C2F2000108780130B9
:1065600008700120159087E01498139A45F62C21A5
:10657000C0F60201F9F78CFE40F27531C2F200015B
:106580000878013008700120159075E01498089083
:106590001398099042F61C60C2F20000D0F8B010C7
:1065A0000491D0F8B800F9F7F5FF02460498059277
:1065B0000A46059942EC101B8DED060BF9F7EAFF30
:1065C0009DED060B024608980B46099943EC112BEA
:1065D0006A4682ED021B82ED000B45F6A252C0F620
:1065E00002021BF0F1FE40F27531C2F200010878A0
:1065F00001300870012015903EE01498139A45F67A
:106600003831C0F60201F9F743FE40F27531C2F2AB
:106610000001087801300870012015902CE01498D2
:10662000139942F61C62C2F2000202F1D003EC465A
:10663000CCF8003002F1BC0345F6D652C0F6020297
:106640001BF0C2FE40F27531C2F200010878013041
:106650000870012015900FE01498139945F64C62CC
:10666000C0F602021BF0B0FE40F27531C2F200012A
:10667000002008701590FFE7159816B080BD000047
:1066800080B582B0019001990020C0F60E0064220E
:10669000FCF796FB0198143000F038F80199C862B5
:1066A000019800F075F8019988620198806A38B9FC
:1066B000FFE7019940F28810C2F200008862FFE70C
:1066C0000198C06A38B9FFE7019944F6E820C0F69E
:1066D0000200C862FFE70198806A013038B9FFE71D
:1066E000019940F28810C2F200008862FFE7019829
:1066F000C06A013038B9FFE7019944F6E820C0F6D6
:106700000200C862FFE702B080BD000080B584B01F
:106710000290029818B9FFE70020039029E00020BA
:106720000190FFE7019945F24C00C0F6020050F8D5
:106730003100D8B1FFE7019945F24C00C0F60200E4
:1067400050F831000299F9F7B6FD50B9FFE7019909
:1067500045F24C00C0F6020000EBC1004068039017
:1067600007E0FFE7019801300190DBE7002003908C
:10677000FFE7039804B080BD45F24C00C0F602006C
:106780007047000045F26400C0F602007047000048
:1067900080B584B00290029818B9FFE700200390FA
:1067A00029E000200190FFE7019945F26400C0F65E
:1067B000020050F83100D8B1FFE7019945F26400BA
:1067C000C0F6020050F831000299F9F774FD50B993
:1067D000FFE7019945F26400C0F6020000EBC1003A
:1067E0004068039007E0FFE7019801300190DBE784
:1067F00000200390FFE7039804B080BD80B582B00D
:10680000019017F0AFF90B20FCF7B6FA01990020C0
:10681000C0F60E006422FCF7DFFA17F0F9F902B0B7
:1068200080BD000080B541F6AC10C2F2000003F05C
:1068300009FC80BD80B541F2CC70C2F2000003F0CB
:1068400001FC80BD80B541F26C70C2F2000003F023
:10685000F9FB80BD80B541F60C20C2F2000003F0C8
:10686000F1FB80BD80B541F62C00C2F2000003F0C0
:10687000E9FB80BD80B541F68C00C2F2000003F058
:10688000E1FB80BD80B541F6EC00C2F2000003F0F0
:10689000D9FB80BD80B541F66C20C2F2000003F048
:1068A000D1FB80BD80B541F64C10C2F2000003F070
:1068B000C9FB80BD82B001900198007810384AF67B
:1068C000AB21CAF6AA21A0FB011000090090009993
:1068D00044F6E800C0F60200405C0199C8650098E3
:1068E000042807D3FFE701990868042262F309002E
:1068F000886506E00199086840F2FF329043886598
:10690000FFE70198806D02B07047000086B00590E7
:1069100000208DF813000598806A0390059880691F
:1069200010BBFFE70398029003281BD80299DFE809
:1069300001F0020D0218059890F82F00C00720B151
:10694000FFE701208DF81300FFE70CE00598C06A0F
:10695000B0F1C07F04D1FFE701208DF81300FFE7FD
:1069600001E000E0FFE745E005988069B0F5005FD1
:1069700025D1FFE70398019003281ED80199DFE88D
:1069800001F00206021101208DF8130016E00598AF
:1069900090F82F00C00720B1FFE701208DF8130009
:1069A000FFE70BE00598C06AB0F1C07F04D1FFE7B4
:1069B00001208DF81300FFE700E0FFE719E00398DE
:1069C0000090032804D3FFE70098032804D00EE0CA
:1069D00001208DF813000BE0059890F82F00C007F8
:1069E00020B1FFE701208DF81300FFE700E0FFE78B
:1069F000FFE7FFE79DF8130006B0704784B00390EF
:106A000002910192009303980168086820F48020A5
:106A100008600098039909684860039880684028D6
:106A200009D1FFE7019803990968886002980399E2
:106A30000968C86008E002980399096888600198AD
:106A400003990968C860FFE704B0704782B00090FE
:106A5000009820B9FFE701208DF8070074E0009846
:106A600000886FF3DF20B0F5B67F09D3FFE7009809
:106A700000886FF3DF2040F29561884204D3FFE77E
:106A800001208DF807005FE000980068C0F3CA207D
:106A9000B0F5B67F09D3FFE700980068C0F3CA20BD
:106AA00040F29561884204D3FFE701208DF807008A
:106AB0004AE0009881880068800D40EA81206FF3E9
:106AC000DF20B0F5B67F0DD3FFE70098818800681E
:106AD000800D40EA81206FF3DF2040F2956188420B
:106AE00004D3FFE701208DF807002DE0009880888F
:106AF000C0F34A00B0F5B67F09D3FFE7009880885D
:106B0000C0F34A0040F29561884204D3FFE70120B8
:106B10008DF8070018E0009881880020B0EB913FC5
:106B200004D1FFE701208DF807000DE00098808870
:106B3000000B800720B9FFE701208DF8070003E074
:106B400000208DF80700FFE79DF8070002B07047AE
:106B500080B584B002900191029820B9FFE7FE2031
:106B60008DF80F000EE0019820B9FFE7FE208DF8A8
:106B70000F0007E001982421F9F77FFB00208DF832
:106B80000F00FFE79DF90F0004B080BD80B584B011
:106B90000290029820B9FFE7FE208DF80F002BE04D
:106BA00042F2B230C2F200000078C00720B1FFE725
:106BB000FD208DF80F001FE017F004FB42F6E07196
:106BC000C2F20001086020B9FFE7FE208DF80F0037
:106BD00012E046F66552C0F6000200200190032143
:106BE000FCF78CFC019842F2B232C2F200020121A1
:106BF00011708DF80F00FFE79DF90F0004B080BD04
:106C000080B584B002900191029820B9FFE7FE2080
:106C10008DF80F009FE00298FFF718FF20B1FFE703
:106C2000FF208DF80F0096E001982421F9F725FB4D
:106C3000FFE70020C4F2A5400090029800886FF39F
:106C4000DF2000EE100AB8EE400A9FED451A30EE44
:106C5000410A30EE000A9DED002A80EE020A0198FA
:106C600080ED020A02980068C0F3CA2000EE100A04
:106C7000B8EE400A30EE410A30EE000A9DED002ADF
:106C800080EE020A019880ED030A0298818800686C
:106C9000800D40EA81206FF3DF2000EE100AB8EE8D
:106CA000400A30EE410A30EE000A9DED002A80EEE7
:106CB000020A019880ED000A02988088C0F34A0019
:106CC00000EE100AB8EE400A30EE410A30EE000A3B
:106CD0009DED002A80EE020A019880ED010A0298DB
:106CE0008088800B0199487502988088C0F3013034
:106CF000019908750298C0880199C8820298008994
:106D00000199088302984089019948830298007B81
:106D1000002818BF0120019908770298407B0028BD
:106D200018BF0120019948770298C0890199C8834A
:106D30000298008A00EE100AB8EE400A30EE410ACE
:106D40009DED001A80EE010A019880ED040A0020F2
:106D50008DF80F00FFE79DF90F0004B080BD00BF64
:106D60000000804480B542F6E070C2F20000006886
:106D7000802117F047F980BD80B582B000900020D7
:106D8000FCF75CFB009912220BF0BAFA20B9FFE77E
:106D900000208DF8070003E0FF208DF80700FFE7D3
:106DA0009DF9070002B080BD80B582B00190019AC4
:106DB0008020012117F078F98038B0FA80F040097E
:106DC00002B080BD7047000080B5012003F098FF3D
:106DD00080BD000080B5082003F092FF80BD000058
:106DE00080B5102003F08CFF80BD000080B520200E
:106DF00003F086FF80BD0000FFE700BFFDE7000055
:106E000080B584B003908DF80B100020019003989A
:106E100060B3FFE70398012828D0FFE70398022812
:106E200024D0FFE70398032820D0FFE70398042825
:106E30001CD0FFE70398052818D0FFE70398062821
:106E400014D0FFE70398072810D0FFE7039808281D
:106E50000CD0FFE70398092808D0FFE703980A2819
:106E600004D0FFE703980B2801D1FFE708E045F2C3
:106E70006510C0F6020040F2DB3116F0E3FCFFE7DC
:106E80009DF80B0078B1FFE79DF80B0001280AD0B0
:106E9000FFE79DF80B00022805D0FFE79DF80B00E7
:106EA000032801D1FFE708E045F26510C0F60200B3
:106EB0004FF4777116F0C6FCFFE79DF80B0018B988
:106EC000FFE70020019017E09DF80B00012804D196
:106ED000FFE74FF4807001900DE09DF80B00022851
:106EE00004D1FFE74FF40070019003E04FF44070CD
:106EF0000190FFE7FFE7FFE743F61041C4F202010C
:106F0000086820F440700860019A0868104308601F
:106F1000086820F0F8000860039A086840EAC20098
:106F200040F002000860086840F48030086004B057
:106F300080BD000043F60040C4F2020000688005F6
:106F400000281FD5FFE743F60041C4F2020108689C
:106F500020F400700860FFE743F60041C4F202012C
:106F6000086840F400600860086820F40060086069
:106F7000FFE743F60041C4F20201086840F40070E4
:106F80000860FFE743F60040C4F2020000684005D5
:106F900000281FD5FFE743F60041C4F2020108684C
:106FA00020F480600860FFE743F60041C4F202016C
:106FB000086840F480500860086820F48050086039
:106FC000FFE743F60041C4F20201086840F4806024
:106FD0000860FFE77047000080B582B08DF80700B9
:106FE00000919DF8070078B1FFE79DF807000128A0
:106FF0000AD0FFE79DF80700022805D0FFE79DF8BB
:107000000700032801D1FFE708E045F26510C0F64C
:1070100002004FF46F7116F015FCFFE7009801288D
:1070200001D1FFE708E045F26510C0F6020040F22A
:10703000BD3116F007FCFFE743F61041C4F2020130
:10704000086820F440700860086840F00400086098
:107050009DF80720086840EA022040F4803008606C
:1070600002B080BD80B582B001908DF80310019808
:10707000B0F1006F05D3FFE70198B0F1016F10D3B5
:10708000FFE7019847F60001C1F6FF71884209D376
:10709000FFE7019847F60F21C1F6FF71884201D83A
:1070A000FFE708E045F22B10C0F6020040F2BB21DA
:1070B00016F0C8FBFFE743F61041C4F2020108686E
:1070C00020F44070086008680860086840F001001B
:1070D00008609DF803000199087002B080BD0000AF
:1070E00080B584B00390019300920398B0F1006FD3
:1070F00005D3FFE70398B0F1016F10D3FFE70398C2
:1071000047F60001C1F6FF71884209D3FFE70398F3
:1071100047F60F21C1F6FF71884201D8FFE708E06A
:1071200045F22B10C0F6020040F2672116F08AFBF0
:10713000FFE743F61041C4F20201086820F44070F2
:107140000860086840F440700860086840F001007A
:107150000860009803990860BFF36F8F0198039946
:10716000486004B080BD000080B582B00190ADF8E9
:1071700002100198B0F1006F05D3FFE70198B0F15C
:10718000016F10D3FFE7019847F60001C1F6FF71C8
:10719000884209D3FFE7019847F60F21C1F6FF7136
:1071A000884201D8FFE708E045F22B10C0F6020044
:1071B00040F2A22116F046FBFFE743F61041C4F26D
:1071C0000201086820F440700860086840F480708C
:1071D0000860086840F001000860BDF802000199ED
:1071E000088002B080BD000080B582B0019000919F
:1071F0000198B0F1006F05D3FFE70198B0F1016F7E
:1072000010D3FFE7019847F60001C1F6FF718842ED
:1072100009D3FFE7019847F60F21C1F6FF718842B5
:1072200001D8FFE708E045F22B10C0F6020040F25B
:10723000892116F007FBFFE743F61041C4F2020173
:10724000086820F440700860086840F40070086026
:10725000086840F00100086000980199086002B0D9
:1072600080BD000043F60C40C4F202000068C00676
:1072700000280FD5FFE742F2CC31C2F20001C86905
:1072800040F01000C86143F60C41C4F20201102026
:107290000860FFE743F60C40C4F202000068800675
:1072A00000280FD5FFE742F2CC31C2F20001C869D5
:1072B00040F00800C86143F60C41C4F202012020EE
:1072C0000860FFE743F60C40C4F202000068400685
:1072D00000280FD5FFE742F2CC31C2F20001C869A5
:1072E00040F00400C86143F60C41C4F202014020A2
:1072F0000860FFE743F60C40C4F202000068000695
:1073000000280FD5FFE742F2CC31C2F20001C86974
:1073100040F00200C86143F60C41C4F20201802033
:107320000860FFE743F60C40C4F2020000688007E3
:1073300000280FD5FFE742F2CC31C2F20001C86944
:1073400040F02000C86143F60C41C4F20201022063
:107350000860FFE77047000080B584B0029000200D
:10736000019042F2CC31C2F20001C86104F0DAF8B7
:107370000190FFE743F60C40C4F202000068C0032E
:10738000002815D5FFE70298013080B1FFE7029889
:1073900040B1FFE704F0C6F80199401A029988420B
:1073A00004D9FFE703208DF80F0023E0FFE7E1E7B2
:1073B00043F60C40C4F202000068C00738B1FFE792
:1073C00043F60C41C4F2020101200860FFE743F6D6
:1073D0000C40C4F20200006810F0F20F06D0FFE784
:1073E000FFF740FF01208DF80F0003E000208DF82B
:1073F0000F00FFE79DF80F0004B080BD40F6CD10F0
:10740000C2F200007047000088B007900691059214
:1074100000200490039005990860FFE704980699FE
:10742000884260D2FFE7FFE70798017800200290CA
:1074300039B1FFE707980078203818BF0120029083
:10744000FFE70298C00720B1FFE7079801300790D7
:10745000EAE7FFE7079801780020019041B1FFE7D4
:10746000079800782038B0FA80F040090190FFE7D3
:107470000198C00720B1FFE7079801300790E9E7BE
:107480000798007868B3FFE70498013004900498E7
:107490000699884224D1FFE707980390FFE70798F1
:1074A00001780020009039B1FFE707980078203874
:1074B00018BF01200090FFE70098C00740B1FFE728
:1074C0000599086801300860079801300790E6E7E1
:1074D0000598006818B9FFE700200390FFE702E075
:1074E00000E000E09AE7039808B0704780B586B0E6
:1074F0000590049103920120029040F27830C2F28C
:1075000000000068002859D1FFE740F27831C2F24C
:10751000000140F2F020C2F200000860FFE740F2F4
:107520007830C2F200000068002846D0FFE740F241
:107530007830C2F20000006800680068019001988D
:10754000F8F7B2FE009005980099405C202805D01D
:10755000FFE705980099405C30BBFFE7059801996B
:10756000009AF8F7BFFEF0B9FFE740F27830C2F2B8
:1075700000000068006890F90C00002812D4FFE7B2
:10758000059817F077FA40F27831C2F200010968E5
:10759000096891F90C10884203D0FFE7002002909F
:1075A000FFE7FFE709E0FFE7FFE740F27831C2F2CB
:1075B0000001086840680860B1E7FFE740F27830F2
:1075C000C2F20000006890B1FFE7029878B9FFE7C7
:1075D0000498039A45F28341C0F60201F8F758FE79
:1075E00040F27831C2F200010020086029E040F248
:1075F0007830C2F200000068B8B1FFE740F278309E
:10760000C2F2000000680068836804980399059A34
:1076100098470290029838B9FFE740F27831C2F2F9
:10762000000100200860FFE70AE00498039A45F291
:10763000DB41C0F60201F8F72BFE00200290FFE7C5
:10764000FFE7029806B080BD80B586B003900020A9
:107650000190039858B9FFE74FF0500080F311886C
:10766000BFF36F8FBFF34F8F0490FFE7FEE7082053
:1076700018F06AF80290029858B9FFE74FF05000EE
:1076800080F31188BFF36F8FBFF34F8F0590FFE733
:10769000FEE70298B0B1FFE718F028FB03980299C3
:1076A0000860029900204860029840F22401C2F26A
:1076B00000010A6850600298086018F043FB01203E
:1076C0000190FFE7019806B080BD000080B584B04E
:1076D00047F61020C1F6FF700068039047F61420AB
:1076E000C1F6FF700068029047F61820C1F6FF70DF
:1076F000006801900199039808440390039888B1A9
:10770000FFE7039840F26811C2F2000100910231D4
:1077100008220AF09DFF00990298123104220AF013
:1077200097FFFFE704B080BD80B58EB006AB049331
:107730000C900B910A920C9820B9FFE7FF208DF86E
:10774000370054E10B9820B9FFE7FF208DF8370090
:107750004DE10A990C980268891A00EE101AB8EEE9
:10776000400A9FEDA51A80EE010A80ED010A0A98F1
:107770000C9908600C980B99097800F0FFF90B98A8
:1077800090ED020AB1EE400A80ED020A0B9890EDEE
:10779000010AB1EE400A80ED010A0C9810300B99F5
:1077A00091ED010ADFED950ACDED020AFDF7C6FE67
:1077B0009DED021A0C9890ED054A90ED430A90ED6C
:1077C0005B3A90ED5E2A32EE042A72EE430AFDF730
:1077D000F7FE9DED021A049880ED030A0C9890EDD7
:1077E000054A90ED440A90ED5B3A90ED5E2A32EE48
:1077F000042A72EE430AFDF7E3FE049981ED020AC2
:107800000B98083091ED020AD1ED030AFDF736FF1F
:107810000B9890ED021A0C9890ED050A30EE010AD3
:1078200080ED050A0B980430F9F78AFB0C98007B71
:107830000146039140B1FFE7039801281DD0FFE7FF
:10784000039802285CD074E000208DF81700FFE751
:107850009DF8170001280FDCFFE70C989DF8171022
:1078600000EB81010020C1F85401FFE79DF81700EB
:1078700001308DF81700EBE75BE00C9901F158003F
:10788000D1ED011A91ED040AD1ED5A0A9FED5C1A6F
:107890008DED011A0CF064FB049A9DED011A82ED46
:1078A000010A0C9901F11C0092ED010AD1ED011AB7
:1078B000D1ED590A0CF054FB9DED011A0C9880EDA6
:1078C000550A0C9901F1D000D1ED011A91ED050A8C
:1078D000D1ED5B0A0CF044FB049A9DED011A82ED98
:1078E000000A0C9901F1940092ED000AD1ED011A01
:1078F000D1ED570A0CF034FB0C9880ED560A18E0D5
:1079000000208DF81600FFE79DF8160001280FDC17
:10791000FFE70C989DF8161000EB81010020C1F8DC
:107920005401FFE79DF8160001308DF81600EBE7D3
:10793000FFE700208DF81500FFE79DF815000128EE
:107940001BDCFFE70C999DF8152001EB421000F5B8
:107950008A7001EB820191ED550A0AF0F1FE0C9854
:107960009DF8151000EB810080ED550AFFE79DF8AA
:10797000150001308DF81500DFE70C98806890F84D
:107980008C00C00740B1FFE70C9890ED550AB1EEAE
:10799000400A80ED550AFFE70C98806890F88D004A
:1079A000C00740B1FFE70C9890ED560AB1EE400ACF
:1079B00080ED560AFFE70C9890ED550AB5EE400AA7
:1079C000F1EE10FA02DAFFE700BFFFE70C9890ED46
:1079D000560AB6EE001AB4EE410AF1EE10FA02DDD4
:1079E000FFE700BFFFE700208DF83700FFE79DF9B4
:1079F00037000EB080BD00BF00007A44DB0FC940E5
:107A00000000000082B0019000910198D0F854016C
:107A1000009908600198D0F858010099486002B0B8
:107A20007047000082B0019000910198007B00999E
:107A3000087002B07047000080B58AB005AA0392B2
:107A4000024603980892079180ED010AC0ED000AF2
:107A5000089820B9FFE7FF208DF8270076E0079807
:107A6000089988600899002008730898806890F841
:107A70008D00C00720B1FFE706A8FDF7EFFDFFE787
:107A8000039890ED010A089880ED430A089880ED6C
:107A9000440A089901F58870896891ED220AB1EECF
:107AA000400ADFED2C0AFDF749FD039A089901F120
:107AB000580092ED000A896801F12002002102912C
:107AC0000CF0C6FB039A089901F11C0092ED000A24
:107AD0008A68012101910CF0BBFB039B0299089A73
:107AE00002F1D00093ED000A926860320CF0B0FB16
:107AF000039B0199089A02F1940093ED000A9268A1
:107B000040320CF0A5FB02988DF81300FFE79DF8BA
:107B10001300012816DCFFE7039A08999DF813006B
:107B200001EB401000F58A7092ED000A8968D1EDF2
:107B3000200A0AF061FEFFE79DF8130001308DF87E
:107B40001300E4E700208DF82700FFE79DF92700E8
:107B50000AB080BDDB0FC94082B00190009100994E
:107B6000019BD3F87401D3F87821D3F87C318B6072
:107B70004A600860002002B07047000080B584B001
:107B800002908DF80710029820B9FFE7FF208DF8CA
:107B90000F0065E09DF807000299097B884204D137
:107BA000FFE700208DF80F005AE000208DF8060056
:107BB000FFE79DF80600032811DCFFE702989DF817
:107BC0000610C1EB011100EB81001C300CF00CFC25
:107BD000FFE79DF8060001308DF80600E9E7002078
:107BE0008DF80500FFE79DF80500012812DCFFE78E
:107BF00002989DF8051000EB411000F58A709FED8A
:107C00001A0A0AF097FEFFE79DF8050001308DF88B
:107C10000500E8E702981030F9F792F90298007B26
:107C2000B0B9FFE79DF80700012805D1FFE70299E9
:107C3000D1F8680108610AE09DF80700022805D123
:107C4000FFE70299D1F874010861FFE7FFE7FFE75A
:107C50009DF807000299087300208DF80F00FFE7D8
:107C60009DF90F0004B080BD0000000080B584B015
:107C700002900191029820B9FFE7FF208DF80F00D4
:107C80002EE0019820B9FFE7FF208DF80F0027E0D4
:107C90000198406C0299C1F874010198406D0299F5
:107CA000C1F878010298806890F88C00C00730B164
:107CB000FFE7029800F5BA70FDF7D0FCFFE70298E5
:107CC000806890F88D00C00730B1FFE7029800F59A
:107CD000BC70FDF7C3FCFFE700208DF80F00FFE745
:107CE0009DF90F0004B080BD80B586B0049003916B
:107CF0000020029003980068122801D8FFE708E0EE
:107D000045F24E20C0F6020040F2896115F09AFD5E
:107D1000FFE70398406830B1FFE7039840681028F8
:107D200001D8FFE708E045F24E20C0F6020040F21D
:107D30008A6115F087FDFFE70398806818B3FFE7B5
:107D40000398806801281ED0FFE703988068022806
:107D500019D0FFE703988068032814D0FFE7039841
:107D6000806804280FD0FFE70398806805280AD0B0
:107D7000FFE703988068062805D0FFE7039880682E
:107D8000072801D1FFE708E045F24E20C0F60200C7
:107D900040F28B6115F056FDFFE7FFE7049890F87D
:107DA0003C00012804D1FFE702208DF81700F7E01E
:107DB0000499012081F83C00FFE7FFE70398006881
:107DC0000A281CD3FFE70398008800EB4000A0F1CD
:107DD0001E01072000FA01F204980168C868904368
:107DE000C86003998868098801EB41011E3900FACF
:107DF00001F204980168C8681043C86018E003984D
:107E0000008800EB4001072000FA01F204980168A5
:107E100008699043086103998868098801EB41016A
:107E200000FA01F204980168086910430861FFE74D
:107E30000398406806281BD8FFE70398406800EBCA
:107E40008000411F1F2000FA01F204980168486B6E
:107E50009043486303990888496801EB810105391B
:107E600000FA01F204980168486B104348633DE052
:107E7000039840680C281CD8FFE70398406800EB83
:107E80008000A0F123011F2000FA01F2049801688C
:107E9000086B9043086303990888496801EB8101E6
:107EA000233900FA01F204980168086B1043086353
:107EB0001BE00398406800EB8000A0F141011F2007
:107EC00000FA01F204980168C86A9043C8620399F5
:107ED0000888496801EB8101413900FA01F20498F0
:107EE0000168C86A1043C862FFE7FFE742F200304A
:107EF000C4F2010001900498006842F20001C4F24B
:107F0000010188420BD1FFE703980068122806D1CF
:107F1000FFE70199486840F480004860FFE7049853
:107F2000006842F20001C4F2010188422ED1FFE74D
:107F300003980068102805D0FFE70398006811280F
:107F400024D1FFE70199486840F400004860039895
:107F50000068102819D1FFE740F22800C2F20000A3
:107F600000684DF68361C4F21B31A0FB0110800C48
:107F700000EB800040000290FFE7029820B1FFE78D
:107F8000029801380290F8E7FFE7FFE7FFE704995E
:107F9000002081F83C00FFE700208DF81700FFE784
:107FA0009DF8170006B080BD81B000900098006871
:107FB000C06C01B07047000080B584B00290002012
:107FC0008DF80700029820B9FFE701208DF80F0017
:107FD000C7E10298006842F20001C4F20101884240
:107FE00012D0FFE70298006842F20011C4F20101CA
:107FF000884209D0FFE70298006842F20021C4F2EB
:108000000101884201D1FFE708E045F24E20C0F6A9
:10801000020040F2431115F015FCFFE7029840689A
:1080200090B1FFE702984068B0F5803F0CD0FFE7C1
:1080300002984068B0F5003F06D0FFE7029840681C
:10804000B0F5403F01D1FFE708E045F24E20C0F611
:1080500002004FF4A27115F0F5FBFFE7029880686B
:1080600090B1FFE702988068B0F1807F0CD0FFE705
:1080700002988068B0F1007F06D0FFE70298806820
:10808000B0F1407F01D1FFE708E045F24E20C0F695
:10809000020040F2451115F0D5FBFFE70298006998
:1080A00028B1FFE702980069012801D1FFE708E045
:1080B00045F24E20C0F602004FF4A37115F0C2FB4A
:1080C000FFE70298007E28B1FFE70298007E0128B2
:1080D00001D1FFE708E045F24E20C0F6020040F271
:1080E000471115F0AFFBFFE70298806A002862D0C5
:1080F000FFE70298806AB0F1807F5CD0FFE70298CA
:10810000806AB0F1007F56D0FFE70298806AB0F134
:10811000407F50D0FFE70298806AB0F1806F4AD06C
:10812000FFE70298806AB0F1A06F44D0FFE70298A1
:10813000806AB0F1C06F3ED0FFE70298806AB0F16C
:10814000E06F38D0FFE70298806AB0F1006F32D05C
:10815000FFE70298806AB0F1106F2CD0FFE7029819
:10816000806AB0F1206F26D0FFE70298806AB0F1F4
:10817000306F20D0FFE70298806AB0F1406F1AD0CC
:10818000FFE70298806AB0F1506F14D0FFE70298C1
:10819000806AB0F1606F0ED0FFE70298806AB0F19C
:1081A000706F08D0FFE70298806A0121C0F6007165
:1081B000884201D1FFE708E045F24E20C0F60200F8
:1081C0004FF4A47115F03EFBFFE70298C06830B190
:1081D000FFE70298C068B0F5006F01D1FFE708E043
:1081E00045F24E20C0F6020040F2491115F02AFB7C
:1081F000FFE70298C06930B1FFE70298C069102814
:1082000001D8FFE708E045F24E20C0F602004FF427
:10821000A57115F017FBFFE7029890F8300030B118
:10822000FFE7029890F83000012801D1FFE708E04D
:1082300045F24E20C0F6020040F24B1115F002FB51
:10824000FFE702984069012809D0FFE702984069DA
:1082500028B1FFE702984069022801D1FFE708E052
:1082600045F24E20C0F602004FF4A67115F0EAFA6E
:10827000FFE7029890F8200030B1FFE7029890F8ED
:108280002000012801D1FFE708E045F24E20C0F6AA
:10829000020040F24D1115F0D5FAFFE70298806A0E
:1082A0000121C0F60071884221D0FFE70298C06A20
:1082B00090B1FFE70298C06AB0F1805F0CD0FFE791
:1082C0000298C06AB0F1005F06D0FFE70298C06A6A
:1082D000B0F1405F01D1FFE708E045F24E20C0F663
:1082E000020040F2511115F0ADFAFFE7FFE70298E6
:1082F000006C50B9FFE7029800F038F802990020AE
:108300004864029981F83C00FFE70298006CC006BF
:10831000002817D4FFE70298006C40F0020020F418
:108320008850029908640298F8F740FB02990020EF
:1083300048640298006C40F0010020F002000299AD
:10834000086403E001208DF80700FFE7FFE70299CA
:10835000002081F83C00FFE79DF807008DF80F0032
:10836000FFE79DF80F0004B080BD000080B58AB023
:1083700009900020089007900690059004900998B5
:10838000006842F20001C4F20101884212D1FFE705
:10839000FFE70020039043F64400C4F202000168A6
:1083A00041F480710160006800F4807003900398CC
:1083B000FFE73AE00998006842F20021C4F20101A7
:1083C000884231D1FFE7FFE70020029043F64400E6
:1083D000C4F20200016841F480610160006800F4A9
:1083E000806002900298FFE7FFE70020019043F6CB
:1083F0003000C4F20200016841F020010160006811
:1084000000F0200001900198FFE74FF48060049095
:10841000032005900020069041F20040C4F20200C3
:1084200004A902F089FCFFE7FFE70AB080BD000065
:1084300080B584B0029001910020009002980068FD
:1084400080684005002816D5FFE70298006880681C
:10845000C00500280FD5FFE70299086C40F0200006
:108460000864FFE70299002081F83C00FFE7012043
:108470008DF80F006DE003F055F80090FFE70298CB
:108480000068006800F00200022829D0FFE7019888
:10849000013020B3FFE7019840B1FFE703F042F855
:1084A0000099401A0199884218D9FFE7029800689C
:1084B000006800F0020002280FD0FFE70299086C64
:1084C00040F004000864FFE70299002081F83C00B6
:1084D000FFE703208DF80F003BE0FFE7FFE7CEE763
:1084E000029801686FF0120008600299086C40F46D
:1084F0000070086402980068806810F0405F24D122
:10850000FFE70298007E00BBFFE702980068C06AA0
:1085100010F4700F07D0FFE70298006880684005EC
:10852000002812D4FFE70299086C20F480700864D8
:108530000298006CC004002806D4FFE70299086C7A
:1085400040F001000864FFE7FFE700208DF80F000E
:10855000FFE79DF80F0004B080BD000080B584B037
:108560000290002001900298007E28B1FFE7029857
:10857000007E012801D1FFE708E045F24E20C0F659
:10858000020040F2D32115F05DF9FFE70298C06ABE
:1085900090B1FFE70298C06AB0F1805F0CD0FFE7AE
:1085A0000298C06AB0F1005F06D0FFE70298C06A87
:1085B000B0F1405F01D1FFE708E045F24E20C0F680
:1085C00002004FF4357115F03DF9FFE7FFE702981F
:1085D00090F83C00012804D1FFE702208DF80F003D
:1085E000D4E00299012081F83C00FFE7FFE7029800
:1085F00000688068C007F0B9FFE7029801688868E2
:1086000040F00100886040F22800C2F200000068DB
:108610004DF68361C4F21B31A0FB0110800C00EB0E
:1086200040000190FFE7019820B1FFE70198013871
:108630000190F8E7FFE7029800688068C00700280B
:1086400000F09580FFE70298006C40F4807040F2E3
:1086500001618843029908640298006840684005F7
:10866000002809D5FFE70298006C40F4805020F400
:10867000005002990864FFE70298006CC0040028CB
:1086800006D5FFE70299486C20F00600486403E035
:10869000029900204864FFE7FFE70299002081F873
:1086A0003C00FFE742F20030C4F201000090029863
:1086B00001686FF02200086000984068C006E8BBBF
:1086C000FFE70298006842F20001C4F2010188420B
:1086D00024D0FFE70298006842F20011C4F20101C1
:1086E000884208D1FFE742F20430C4F2010000687A
:1086F000C00698B1FFE70298006842F20021C4F278
:108700000101884219D1FFE742F20430C4F20100AE
:10871000006800F01F000F280FD8FFE702980068DC
:10872000806810F0405F07D1FFE702980168886811
:1087300040F080408860FFE7FFE717E0029800689C
:1087400042F20001C4F2010188420ED1FFE7029813
:108750000068806810F0405F07D1FFE70298016869
:10876000886840F080408860FFE7FFE70AE00299F0
:10877000086C40F0100008640299486C40F0010059
:108780004864FFE700208DF80F00FFE79DF80F0019
:1087900004B080BD80B584B002900191029890F839
:1087A00020008DF80300019848F67F71C0F20301A4
:1087B000884201D8FFE708E045F28620C0F60200B3
:1087C0004FF4D06115F03EF8FFE79DF80300012853
:1087D00005D0FFE79DF8030002280AD1FFE7019AC0
:1087E0000298016848691043486100208DF80F0025
:1087F00008E00299486A40F48020486201208DF820
:108800000F00FFE79DF80F0004B080BD80B588B071
:108810000690059104920393069890F820008DF835
:10882000070006980068806800900598806828B165
:10883000FFE705988068042801D1FFE708E045F2CA
:108840008620C0F6020040F2E94114F0FBFFFFE78A
:108850000598C06828B1FFE70598C068022801D1D3
:10886000FFE708E045F28620C0F6020040F2EA4148
:1088700014F0E8FFFFE705980069082801D8FFE732
:1088800008E045F28620C0F6020040F2EB4114F009
:10889000D9FFFFE70598806890B9FFE70598016860
:1088A0000020B0EBD12F01D1FFE708E045F2862090
:1088B000C0F6020040F2EE4114F0C4FFFFE711E001
:1088C000059841680020B0EB517F01D1FFE708E037
:1088D00045F28620C0F6020040F2F24114F0B2FFE9
:1088E000FFE7FFE70598007D28B1FFE70598007DC9
:1088F000012801D1FFE708E045F28620C0F602001A
:1089000040F2F44114F09EFFFFE79DF807000128B4
:1089100006D0FFE79DF80700022840F08D80FFE7B2
:108920009DF80300400700280CD4FFE79DF80300E2
:108930000007002806D4FFE79DF80300C0060028C2
:1089400071D5FFE70098C0F30160029002980328F8
:1089500009D3FFE70699486A40F400004862012005
:108960008DF81F0071E0029901208840039908608A
:108970000598806868B9FFE705980168C06840EA13
:10898000415006990968029A01EB0211C1F8800171
:108990000EE005994A688868C96840EAC200084341
:1089A00006990968029A01EB0211C1F88001FFE7FC
:1089B0000598006906990968029A01EB0211C1F84D
:1089C00084010598007D01280CD1FFE70698006816
:1089D000029900EB0111D1F8840140F48070C1F8D4
:1089E0008401FFE70498406806990968029A01EB40
:1089F0000211C1F88C010498006806990968029A6E
:108A000001EB0211C1F8880106980068029900EB99
:108A10000111D1F8800140F00100C1F8800100206F
:108A20008DF81F0011E00699486A40F40010486272
:108A300001208DF81F0008E00699486A40F4802064
:108A4000486201208DF81F00FFE79DF81F0008B065
:108A500080BD000080B586B0049003910498006842
:108A60000190049890F820008DF803009DF8030011
:108A7000012806D0FFE79DF80300022840F052814C
:108A8000FFE70398408808B9FFE708E045F2862031
:108A9000C0F602004FF4547114F0D4FEFFE70398BF
:108AA000C08808B9FFE708E045F28620C0F602005A
:108AB00040F2513114F0C6FEFFE70398408908B92F
:108AC000FFE708E045F28620C0F6020040F252318E
:108AD00014F0B8FEFFE70398C08908B9FFE708E083
:108AE00045F28620C0F6020040F2533114F0AAFE8F
:108AF000FFE70398806928B1FFE7039880690128A0
:108B000001D1FFE708E045F28620C0F602004FF4ED
:108B1000557114F097FEFFE70398C06928B1FFE78D
:108B20000398C069012801D1FFE708E045F28620DB
:108B3000C0F6020040F2553114F084FEFFE70398BE
:108B4000006928B1FFE703980069012801D1FFE718
:108B500008E045F28620C0F6020040F2563114F0DB
:108B600071FEFFE70398006A28B1FFE70398006AE7
:108B7000012801D1FFE708E045F28620C0F6020097
:108B800040F2573114F05EFEFFE746F20040C4F2B7
:108B900000000190039840691B2801D8FFE708E016
:108BA00045F28620C0F6020040F2723114F04AFE0F
:108BB000FFE70398406A1B2801D8FFE708E045F269
:108BC0008620C0F6020040F2733114F03BFEFFE74E
:108BD0000199D1F8000240F00100C1F800020199AA
:108BE000D1F8000220F47C50C1F800020398426AD8
:108BF0000199D1F8000240EA0220C1F8000203986E
:108C0000406900F01F01012088400290029A0199FA
:108C1000D1F81C029043C1F81C020398C069F0B956
:108C2000FFE7029A0199D1F80C029043C1F80C02B7
:108C3000039A9088D168526940EA0140019901EB9A
:108C4000C201C1F84002039A10889168526940EA53
:108C50000140019901EBC201C1F84402FFE703980A
:108C6000C06901281ED1FFE7029A0199D1F80C02D0
:108C70001043C1F80C02039A90881168526940EAC7
:108C80000140019901EBC201C1F84002039A9089A9
:108C90009168526940EA0140019901EBC201C1F8B3
:108CA0004402FFE70398806940B9FFE7029A0199FF
:108CB000D1F804029043C1F8040207E0029A019936
:108CC000D1F804021043C1F80402FFE703980069D9
:108CD00040B9FFE7029A0199D1F814029043C1F814
:108CE000140207E0029A0199D1F814021043C1F866
:108CF0001402FFE70398006A012808D1FFE7029AEF
:108D00000199D1F81C021043C1F81C02FFE7019938
:108D1000D1F8000220F00100C1F8000200208DF817
:108D2000170008E00499486A40F480204862012056
:108D30008DF81700FFE79DF8170006B080BD000012
:108D400080B582B001900198FAF784FD8DF8030098
:108D50009DF80300032819D0FFE79DF8030040F2B7
:108D6000F822C2F20002342110FB0120006B60B136
:108D7000FFE79DF8030040F2F822C2F2000234211E
:108D800010FB0120006B8047FFE7FFE702B080BDCA
:108D900080B586B00490039102920193049890F8F4
:108DA00020008DF80300039820B1FFE70398012805
:108DB00001D1FFE708E045F28620C0F602004FF43B
:108DC000BE6114F03FFDFFE79DF80300012806D0C7
:108DD000FFE79DF80300022840F0D780FFE70398E3
:108DE00080B9FFE704980068C068800748B9FFE7CA
:108DF0000499486A40F40010486201208DF8170079
:108E0000CCE00FE0049800680069800748B9FFE7EC
:108E10000499486A40F40010486201208DF8170058
:108E2000BCE0FFE704980068039900EB0110D0F85C
:108E3000B00100F00400029988600298806858B977
:108E4000FFE704980068039900EB0110D0F8B00127
:108E5000400D029908600AE004980068039900EB4D
:108E60000110D0F8B001C00802994860FFE70498EB
:108E70000068039900EB0110D0F8B00100F0020087
:108E80000299C86004980068039900EB0110D0F8BB
:108E9000B40100F00F00029908610498006803997A
:108EA00000EB0110D0F8B40180B2000A0299886189
:108EB00004980068039900EB0110D0F8B401000C8D
:108EC0000299486104980068039900EB0110D0F8FA
:108ED000B8010199087004980068039900EB01102B
:108EE000D0F8B801000A0199487004980068039905
:108EF00000EB0110D0F8B801000C019988700498BB
:108F00000068039900EB0110D0F8B801000E019938
:108F1000C87004980068039900EB0110D0F8BC01F8
:108F20000199087104980068039900EB0110D0F8CA
:108F3000BC01000A0199487104980068039900EB8C
:108F40000110D0F8BC01000C0199887104980068E8
:108F5000039900EB0110D0F8BC01000E0199C87113
:108F6000039838B9FFE704980168C86840F020000A
:108F7000C86006E004980168086940F020000861B4
:108F8000FFE700208DF8170008E00499486A40F4D4
:108F90008020486201208DF81700FFE79DF8170038
:108FA00006B080BD80B58AB009900020089009986D
:108FB0000068406907900998006840680690099821
:108FC00000688068059009980068C0680490099856
:108FD00000680069039009980068806902909DF814
:108FE0001C00C007002800F09480FFE79DF81400E3
:108FF000C00758B3FFE709980168012088609DF811
:1090000014008007002804D5FFE7099800F042FE0D
:109010001BE09DF814004007002805D5FFE70898DD
:1090200040F4006008900FE09DF81400000700284D
:1090300005D5FFE7089840F48050089003E00998B0
:1090400000F000FEFFE7FFE7FFE7FFE79DF81500F0
:10905000C00760B3FFE7099801684FF4807088602B
:109060009DF815008007002804D5FFE7099800F057
:109070005FFE1BE09DF815004007002805D5FFE7BF
:10908000089840F4005008900FE09DF81500000784
:10909000002805D5FFE7089840F48040089003E0D9
:1090A000099800F01DFEFFE7FFE7FFE7FFE79DF8E7
:1090B0001600C00760B3FFE7099801684FF48030DD
:1090C00088609DF816008007002804D5FFE70998FE
:1090D00000F07EFE1BE09DF816004007002805D535
:1090E000FFE7089840F4004008900FE09DF8160054
:1090F0000007002805D5FFE7089840F48030089065
:1091000003E0099800F03CFEFFE7FFE7FFE7FFE719
:10911000FFE79DF81C000007002810D5FFE79DF829
:109120001000C006002809D5FFE7089840F4007039
:109130000890099801681020C860FFE7FFE79DF8D4
:109140001C00400700280FD5FFE79DF8100000071E
:10915000002808D5FFE7099801680820C860099829
:1091600000F062FCFFE7FFE79DF81C008007002885
:109170000BD5FFE709980068C068800720B1FFE7BA
:10918000099800F079FCFFE7FFE79DF81C00400616
:10919000002810D5FFE79DF80C00C006002809D56F
:1091A000FFE7089840F48060089009980168102053
:1091B0000861FFE7FFE79DF81C00800600280FD537
:1091C000FFE79DF80C000007002808D5FFE7099885
:1091D000016808200861099800F076FCFFE7FFE7C6
:1091E0009DF81C00C00600280BD5FFE70998006811
:1091F0000069800720B1FFE7099800F08DFCFFE7C8
:10920000FFE79DF81E00800700280FD5FFE79DF8B7
:109210001800C006002808D5FFE70998016810204B
:109220004860099800F0A0FCFFE7FFE79DF81E00EA
:10923000C00778B1FFE79DF818000007002808D59F
:10924000FFE70998016808204860099800F0E8FDE8
:10925000FFE7FFE79DF81D000006002840F18D8024
:10926000FFE79DF818004007002840F18180FFE7E4
:109270009DF81D00C00750B1FFE79DF80800C0072A
:1092800028B1FFE7089840F001000890FFE79DF83B
:109290001D00800700280BD5FFE79DF80800800718
:1092A000002805D5FFE7089840F002000890FFE786
:1092B0009DF81D00400700280BD5FFE79DF808002A
:1092C0004007002805D5FFE7089840F00400089003
:1092D000FFE79DF81D000007002848D5FFE79DF82F
:1092E000080010F0700F42D0FFE7029800F0700005
:1092F00001460191102814D0FFE70198202815D0CD
:10930000FFE70198302816D0FFE70198402817D0D2
:10931000FFE70198502818D0FFE70198602819D07E
:109320001DE0089840F00800089019E0089840F007
:109330001000089014E0089840F0200008900FE01A
:10934000089840F0400008900AE0089840F080003B
:10935000089005E0089840F48070089000E0FFE76E
:1093600009980168886920F070008861FFE7FFE7CD
:109370000998016804204860FFE7089848B1FFE7B2
:10938000089A0999486A104348620998FFF7D8FC7F
:10939000FFE70AB080BD000080B584B0029002985B
:1093A00020B9FFE701208DF80F0063E20298006802
:1093B00046F20041C4F20001884209D0FFE702985A
:1093C000006846F60001C4F20001884201D1FFE7BF
:1093D00008E045F28620C0F6020040F21D1114F0AC
:1093E00031FAFFE70298007E28B1FFE70298007E7D
:1093F000012801D1FFE708E045F28620C0F602000F
:109400004FF48F7114F01EFAFFE70298407E28B1E6
:10941000FFE70298407E012801D1FFE708E045F20E
:109420008620C0F6020040F21F1114F00BFAFFE78D
:109430000298807E28B1FFE70298807E012801D142
:10944000FFE708E045F28620C0F602004FF4907175
:1094500014F0F8F9FFE70298C07E28B1FFE7029800
:10946000C07E012801D1FFE708E045F28620C0F662
:10947000020040F2211114F0E5F9FFE70298007FA5
:1094800028B1FFE70298007F012801D1FFE708E03B
:1094900045F28620C0F602004FF4917114F0D2F923
:1094A000FFE70298407F28B1FFE70298407F01283C
:1094B00001D1FFE708E045F28620C0F6020040F245
:1094C000231114F0BFF9FFE70298806890B1FFE71D
:1094D00002988068B0F1804F0CD0FFE70298806856
:1094E000B0F1004F06D0FFE702988068B0F1404F1E
:1094F00001D1FFE708E045F28620C0F602004FF4F4
:10950000927114F09FF9FFE70298C06890B1FFE7ED
:109510000298C068B0F1807F0CD0FFE70298C06865
:10952000B0F1007F06D0FFE70298C068B0F1407F3D
:1095300001D1FFE708E045F28620C0F6020040F2C4
:10954000251114F07FF9FFE70298006900285AD02E
:10955000FFE702980069B0F5803F54D0FFE702981A
:109560000069B0F5003F4ED0FFE702980069B0F502
:10957000403F48D0FFE702980069B0F5802F42D005
:10958000FFE702980069B0F5A02F3CD0FFE70298F2
:109590000069B0F5C02F36D0FFE702980069B0F53A
:1095A000E02F30D0FFE702980069B0F5002F2AD0F5
:1095B000FFE702980069B0F5102F24D0FFE702986A
:1095C0000069B0F5202F1ED0FFE702980069B0F5C2
:1095D000302F18D0FFE702980069B0F5402F12D065
:1095E000FFE702980069B0F5502F0CD0FFE7029812
:1095F0000069B0F5602F06D0FFE702980069B0F56A
:10960000702F01D1FFE708E045F28620C0F6020086
:109610004FF4937114F016F9FFE70298406950B3C4
:10962000FFE702984069B0F5801F24D0FFE7029859
:109630004069B0F5001F1ED0FFE702984069B0F501
:10964000401F18D0FFE702984069B0F5800F12D094
:10965000FFE702984069B0F5A00F0CD0FFE7029831
:109660004069B0F5C00F06D0FFE702984069B0F539
:10967000E00F01D1FFE708E045F28620C0F60200C6
:1096800040F2271114F0DEF8FFE70298406838B185
:10969000FFE702984068B0F5806F01D8FFE708E067
:1096A00045F28620C0F602004FF4947114F0CAF817
:1096B000FFE7029890F8200020B9FFE7029800F039
:1096C000DDF8FFE702980168086820F002000860F2
:1096D00001F028FF0190FFE70298006840688007CA
:1096E000002815D5FFE701F01DFF0199401A0B284E
:1096F0000DD3FFE70299486A40F4003048620299AE
:10970000052081F8200001208DF80F00B2E0E3E78A
:1097100002980168086840F00100086001F002FF4B
:109720000190FFE7029800684068C007A8B9FFE70A
:1097300001F0F8FE0199401A0B280DD3FFE70299BA
:10974000486A40F4003048620299052081F8200000
:1097500001208DF80F008DE0E4E70298007E0128DB
:1097600007D1FFE702980168086840F080000860B0
:1097700006E002980168086820F080000860FFE7B2
:109780000298407E012807D1FFE702980168086827
:1097900040F04000086006E002980168086820F088
:1097A00040000860FFE70298807E012807D1FFE7AC
:1097B00002980168086840F02000086006E00298FE
:1097C0000168086820F020000860FFE70298C07E6A
:1097D000012807D1FFE702980168086820F010000F
:1097E000086006E002980168086840F01000086010
:1097F000FFE70298007F012807D1FFE70298016880
:10980000086840F00800086006E0029801680868EF
:1098100020F008000860FFE70298407F012807D188
:10982000FFE702980168086840F00400086006E05D
:1098300002980168086820F004000860FFE7029BB6
:1098400019685A689868D3F80CC040EA0C00D3F83D
:1098500010C040EA0C005B691843013A1043C8612C
:10986000029900204862029A012182F820108DF8A6
:109870000F00FFE79DF80F0004B080BD80B594B0E5
:10988000139000201290119010900F900E9013984A
:10989000006846F20041C4F20001884253D1FFE75C
:1098A00040F2BC30C2F20000016801310160006882
:1098B000012812D1FFE7FFE700200D9043F640009A
:1098C000C4F20200016841F000710160006800F01C
:1098D00000700D900D98FFE7FFE7FFE700200C9068
:1098E00043F63000C4F20200016841F00801016053
:1098F000006800F008000C900C98FFE703200E9021
:1099000002210F91002107911091119009201290CE
:1099100040F60040C4F202000EA901F00DFA079AC9
:10992000142005900521069102F018FA059802F01E
:10993000FDF90699079A1520089002F00FFA089889
:1099400002F0F4F96EE01398006846F60001C4F2E4
:109950000001884265D1FFE7FFE700200B9043F646
:109960004000C4F20200016841F0806101600068BB
:1099700000F080600B900B98FFE740F2BC30C2F221
:1099800000000168013101600068012812D1FFE781
:10999000FFE700200A9043F64000C4F2020001688D
:1099A00041F000710160006800F000700A900A98B0
:1099B000FFE7FFE7FFE70020099043F63000C4F21D
:1099C0000200016841F002010160006800F002003D
:1099D00009900998FFE760200E9002200F90002068
:1099E00003901090032011900920129040F2004043
:1099F000C4F202000EA901F09FF9039A40200190E1
:109A00000521029102F0AAF9019802F08FF902995A
:109A1000039A4120049002F0A1F9049802F086F91B
:109A2000FFE7FFE714B080BD80B582B001900198D8
:109A3000F9F710FF8DF803009DF80300032819D0F3
:109A4000FFE79DF8030040F2F822C2F20002342141
:109A500010FB0120C06960B1FFE79DF8030040F2F0
:109A6000F822C2F20002342110FB0120C0698047B5
:109A7000FFE7FFE702B080BD80B582B0019001989A
:109A8000F9F7E8FE8DF803009DF80300032819D0CC
:109A9000FFE79DF8030040F2F822C2F200023421F1
:109AA00010FB0120806960B1FFE79DF8030040F2E0
:109AB000F822C2F20002342110FB012080698047A5
:109AC000FFE7FFE702B080BD80B582B0019001984A
:109AD000F9F7C0FE8DF803009DF80300032819D0A4
:109AE000FFE79DF8030040F2F822C2F200023421A1
:109AF00010FB0120406A60B1FFE79DF8030040F2CF
:109B0000F822C2F20002342110FB0120406A804793
:109B1000FFE7FFE702B080BD80B582B001900198F9
:109B2000F9F798FE8DF803009DF80300032819D07B
:109B3000FFE79DF8030040F2F822C2F20002342150
:109B400010FB0120006A60B1FFE79DF8030040F2BE
:109B5000F822C2F20002342110FB0120006A804783
:109B6000FFE7FFE702B080BD80B582B001900198A9
:109B7000F9F770FE8DF803009DF80300032819D053
:109B8000FFE79DF8030040F2F822C2F20002342100
:109B900010FB0120806A60B1FFE79DF8030040F2EE
:109BA000F822C2F20002342110FB0120806A8047B3
:109BB000FFE7FFE702B080BD80B584B00290029855
:109BC00090F8200001282FD1FFE70299022081F8A8
:109BD000200002980168086820F00100086001F088
:109BE000A1FC0190FFE7029800684068C007A8B197
:109BF000FFE701F097FC0199401A0B280DD3FFE70E
:109C00000299486A40F4003048620299052081F8C0
:109C1000200001208DF80F000FE0E4E702990020FA
:109C200048628DF80F0008E00299486A40F400206D
:109C3000486201208DF80F00FFE79DF80F0004B087
:109C400080BD000080B582B001900198F9F702FE56
:109C50008DF803009DF80300032819D0FFE79DF855
:109C6000030040F2F822C2F20002342110FB01206E
:109C7000C06860B1FFE79DF8030040F2F822C2F22D
:109C80000002342110FB0120C0688047FFE7FFE796
:109C900002B080BD80B582B001900198F9F7DAFD7D
:109CA0008DF803009DF80300032817D0FFE79DF807
:109CB00003003421414340F2F820C2F20000405832
:109CC00058B1FFE79DF803003421414340F2F820EA
:109CD000C2F2000040588047FFE7FFE702B080BDB6
:109CE00080B582B001900198F9F7B4FD8DF80300BA
:109CF0009DF80300032819D0FFE79DF8030040F208
:109D0000F822C2F20002342110FB0120006960B188
:109D1000FFE79DF8030040F2F822C2F2000234216E
:109D200010FB012000698047FFE7FFE702B080BD1C
:109D300080B582B001900198F9F78CFD8DF8030091
:109D40009DF80300032819D0FFE79DF8030040F2B7
:109D5000F822C2F20002342110FB0120406860B1F9
:109D6000FFE79DF8030040F2F822C2F2000234211E
:109D700010FB012040688047FFE7FFE702B080BD8D
:109D800080B582B001900198F9F764FD8DF8030069
:109D90009DF80300032819D0FFE79DF8030040F267
:109DA000F822C2F20002342110FB0120406960B1A8
:109DB000FFE79DF8030040F2F822C2F200023421CE
:109DC00010FB012040698047FFE7FFE702B080BD3C
:109DD00080B582B001900198F9F73CFD8DF8030041
:109DE0009DF80300032819D0FFE79DF8030040F217
:109DF000F822C2F20002342110FB0120806860B119
:109E0000FFE79DF8030040F2F822C2F2000234217D
:109E100010FB012080688047FFE7FFE702B080BDAC
:109E200080B582B001900198F9F714FD8DF8030018
:109E30009DF80300032819D0FFE79DF8030040F2C6
:109E4000F822C2F20002342110FB0120C06A60B186
:109E5000FFE79DF8030040F2F822C2F2000234212D
:109E600010FB0120C06A8047FFE7FFE702B080BD1A
:109E700080B582B00090009820B9FFE701208DF8EE
:109E8000070023E00098006843F20001C4F20201D9
:109E9000884201D1FFE707E045F2BE20C0F602008C
:109EA000682113F0CFFCFFE70098407938B9FFE74D
:109EB000009900200871009800F00CF8FFE7009965
:109EC0000120487100208DF80700FFE79DF807008A
:109ED00002B080BD82B001900198006843F2000199
:109EE000C4F20201884212D1FFE7FFE70020009090
:109EF00043F63000C4F20200016841F48051016071
:109F0000006800F4805000900098FFE7FFE702B07F
:109F10007047000080B584B002900298806D019077
:109F200001F000FB0090029890F8350002280DD057
:109F3000FFE7029980204865FFE70299002081F839
:109F40003400FFE701208DF80F0054E0029801680B
:109F5000086820F01600086002980168486920F03F
:109F6000800048610298006C20B9FFE70298806C7D
:109F700038B1FFE702980168086820F0080008601F
:109F8000FFE702980168086820F001000860FFE719
:109F9000029800680068C007C0B1FFE701F0C2FA8C
:109FA0000099401A062810D3FFE70299202048653F
:109FB000FFE70299002081F83400FFE702990320AF
:109FC00081F835008DF80F0015E0E1E70298C16DCA
:109FD0003F20884001998860FFE70299002081F8BE
:109FE0003400FFE70299012081F83500FFE70020E7
:109FF0008DF80F00FFE79DF80F0004B080BD000052
:10A0000082B00090009890F83500022807D0FFE752
:10A0100000998020486501208DF807000EE0009926
:10A02000052081F8350000980168086820F00100DB
:10A030000860FFE700208DF80700FFE79DF80700A4
:10A0400002B0704780B586B005900020039040F2C2
:10A050002800C2F20000006848F2B511C1F64E3186
:10A06000A0FB0110800A02900598806D0190019874
:10A070000068049004980599C96DC840000700283D
:10A080001AD5FFE70598006800684007002812D538
:10A09000FFE705980168086820F00400086005984B
:10A0A000C16D08208840019988600599486D40F08D
:10A0B00001004865FFE7FFE704980599C96DC840AE
:10A0C000C007A0B1FFE705980068406900060028B6
:10A0D0000CD5FFE70598C16D012088400199886083
:10A0E0000599486D40F002004865FFE7FFE70498D6
:10A0F0000599C96DC8404007002814D5FFE70598A9
:10A1000000680068800700280CD5FFE70598C16D3E
:10A1100004208840019988600599486D40F004004A
:10A120004865FFE7FFE704980599C96DC840C00678
:10A13000002847D5FFE70598006800680007002859
:10A140003FD5FFE70598C16D1020884001998860D0
:10A15000059800680068400300281AD5FFE70598B5
:10A16000006800680003002809D4FFE70598006C28
:10A1700020B1FFE70598016C8847FFE708E00598E4
:10A18000806C20B1FFE70598816C8847FFE7FFE707
:10A1900016E0059800680068C005002807D4FFE7AE
:10A1A00005980168086820F008000860FFE7059836
:10A1B000006C20B1FFE70598016C8847FFE7FFE7D7
:10A1C000FFE7FFE704980599C96DC840800600289D
:10A1D00040F18D80FFE7059800680068C006002800
:10A1E00040F18480FFE70598C16D202088400199E7
:10A1F0008860059890F83500052834D1FFE7059868
:10A200000168086820F01600086005980168486930
:10A2100020F0800048610598006C20B9FFE70598A0
:10A22000806C38B1FFE705980168086820F00800E5
:10A230000860FFE70598C16D3F208840019988605C
:10A24000FFE70599002081F83400FFE70599012018
:10A2500081F835000598006D20B1FFE70598016D84
:10A260008847FFE77BE00598006800684003002806
:10A270001AD5FFE70598006800680003002809D494
:10A28000FFE70598406C20B1FFE70598416C8847CF
:10A29000FFE708E00598C06B20B1FFE70598C16BA8
:10A2A0008847FFE7FFE720E0059800680068C005E1
:10A2B000002811D4FFE705980168086820F0100015
:10A2C0000860FFE70599002081F83400FFE7059951
:10A2D000012081F83500FFE70598C06B20B1FFE74A
:10A2E0000598C16B8847FFE7FFE7FFE7FFE70598A1
:10A2F000406DA0B3FFE70598406DC00730B3FFE79E
:10A300000599052081F8350005980168086820F056
:10A3100001000860FFE7039801300390029988422A
:10A3200001D9FFE707E0FFE7059800680068C0076C
:10A330000028F0D1FFE7FFE70599002081F83400FD
:10A34000FFE70599012081F83500FFE70598C06C0B
:10A3500020B1FFE70598C16C8847FFE7FFE706B02B
:10A3600080BD000080B586B004900020039001F00D
:10A37000D9F80290049820B9FFE701208DF8170062
:10A3800087E20498006846F21001C4F20201884294
:10A3900000F08880FFE70498006846F22801C4F2C4
:10A3A000020188427ED0FFE70498006846F240012F
:10A3B000C4F20201884275D0FFE70498006846F2B3
:10A3C0005801C4F2020188426CD0FFE7049800688B
:10A3D00046F27001C4F20201884263D0FFE704989C
:10A3E000006846F28801C4F2020188425AD0FFE7B1
:10A3F0000498006846F2A001C4F20201884251D0DC
:10A40000FFE70498006846F2B801C4F202018842EE
:10A4100048D0FFE70498006846F21041C4F20201F8
:10A4200088423FD0FFE70498006846F22841C4F212
:10A430000201884236D0FFE70498006846F24041A6
:10A44000C4F2020188422DD0FFE70498006846F26A
:10A450005841C4F20201884224D0FFE70498006802
:10A4600046F27041C4F2020188421BD0FFE7049813
:10A47000006846F28841C4F20201884212D0FFE728
:10A480000498006846F2A041C4F20201884209D053
:10A49000FFE70498006846F2B841C4F2020188421E
:10A4A00001D1FFE707E045F2DB10C0F60200B8215A
:10A4B00013F0C8F9FFE70498406850B3FFE7049829
:10A4C0004068B0F1007F24D0FFE704984068B0F105
:10A4D000806F1ED0FFE704984068B0F1C06F18D0BD
:10A4E000FFE704984068B0F1006F12D0FFE70498CE
:10A4F0004068B0F1206F0CD0FFE704984068B0F1DD
:10A50000406F06D0FFE704984068B0F1606F01D15A
:10A51000FFE707E045F2DB10C0F60200B92113F0B7
:10A5200091F9FFE70498806850B1FFE704988068CC
:10A53000402805D0FFE704988068802801D1FFE714
:10A5400007E045F2DB10C0F60200BA2113F07AF9F9
:10A55000FFE70498C068B0F5007F04D0FFE70498D7
:10A56000C06808B9FFE707E045F2DB10C0F602005B
:10A57000BB2113F067F9FFE704980069B0F5806F1D
:10A5800004D0FFE70498006908B9FFE707E045F247
:10A59000DB10C0F60200BC2113F054F9FFE7049869
:10A5A000406960B1FFE704984069B0F5006F06D0DC
:10A5B000FFE704984069B0F5805F01D1FFE707E04D
:10A5C00045F2DB10C0F60200BD2113F03BF9FFE7B6
:10A5D0000498806960B1FFE704988069B0F5005F76
:10A5E00006D0FFE704988069B0F5804F01D1FFE7FE
:10A5F00007E045F2DB10C0F60200BE2113F022F99D
:10A60000FFE70498C06958B1FFE70498C069B0F546
:10A61000807F05D0FFE70498C069202801D1FFE7BB
:10A6200007E045F2DB10C0F60200BF2113F00AF983
:10A63000FFE70498006A90B1FFE70498006AB0F55C
:10A64000803F0CD0FFE70498006AB0F5003F06D0C9
:10A65000FFE70498006AB0F5403F01D1FFE707E04B
:10A6600045F2DB10C0F60200C02113F0EBF8FFE763
:10A670000498406A28B1FFE70498406A042801D191
:10A68000FFE707E045F2DB10C0F60200C12113F03E
:10A69000D9F8FFE70498406A00285BD0FFE70498E8
:10A6A000806A78B1FFE70498806A01280AD0FFE742
:10A6B0000498806A022805D0FFE70498806A03287E
:10A6C00001D1FFE707E045F2DB10C0F60200C6212A
:10A6D00013F0B8F8FFE70498C06A90B1FFE7049858
:10A6E000C06AB0F5000F0CD0FFE70498C06AB0F163
:10A6F000807F06D0FFE70498C06AB0F1C07F01D127
:10A70000FFE707E045F2DB10C0F60200C72113F0B7
:10A7100099F8FFE70498006B90B1FFE70498006B8D
:10A72000B0F5001F0CD0FFE70498006BB0F5800F68
:10A7300006D0FFE70498006BB0F5C00F01D1FFE72A
:10A7400007E045F2DB10C0F60200C82113F07AF8EA
:10A75000FFE7FFE7FFE70499002081F83400FFE7F7
:10A760000499022081F8350004980168086820F0F7
:10A7700001000860FFE7049800680068C00790B116
:10A78000FFE700F0CFFE0299401A06280AD3FFE740
:10A790000499202048650499032081F835008DF83C
:10A7A000170076E0E7E704980068006803900398D4
:10A7B00048F23F01CFF21001084003900499009144
:10A7C0004868D1F808C0CB680A6940EA0C00184311
:10A7D00010434A6910438A691043CA691043096AE1
:10A7E00001430398084303900498406A042808D161
:10A7F000FFE70499C86A096B014303980843039073
:10A80000FFE70398049909680860049800684069A4
:10A810000390039820F0070003900498416A03987E
:10A82000084303900498406A04281AD1FFE704986B
:10A83000816A0398084303900498C06A80B1FFE7D7
:10A840000498FCF763F850B1FFE70499402048658D
:10A850000499012081F835008DF8170019E0FFE711
:10A86000FFE703980499096848610498FCF722F807
:10A8700001900498C16D3F20884001998860049937
:10A8800000204865049A012182F835108DF81700E0
:10A89000FFE79DF8170006B080BD000080B588B0C6
:10A8A000069005910492039300208DF80B00069802
:10A8B000806D0190039828B1FFE7BDF80E0008B93C
:10A8C000FFE708E045F2DB10C0F602004FF4E67146
:10A8D00012F0B8FFFFE7FFE7069890F83400012870
:10A8E00004D1FFE702208DF81F0045E00699012002
:10A8F00081F83400FFE7FFE7069890F8350001285B
:10A900002BD1FFE70699022081F835000699002037
:10A91000486506980599049A039BFCF76FF806981A
:10A92000C16D3F20884001998860069801680868D9
:10A9300040F0160008600698006C38B1FFE70698F2
:10A940000168086840F008000860FFE706980168A1
:10A95000086840F00100086009E0FFE70699002060
:10A9600081F83400FFE702208DF80B00FFE79DF827
:10A970000B008DF81F00FFE79DF81F0008B080BD99
:10A9800080B584B0039000F0CDFD02900398019053
:10A990000198013048B1FFE740F2E020C2F2000028
:10A9A0000178019808440190FFE7FFE700F0BAFD45
:10A9B0000299401A0199884201D2FFE7F6E704B0F4
:10A9C00080BD000080B586B00490039101208DF811
:10A9D0000B0000200190FFE742F2CC30C2F20000F1
:10A9E000007E012804D1FFE702208DF8170094E0D3
:10A9F00042F2CC31C2F2000101200876FFE7FFE706
:10AA00000498006828B1FFE704980068012801D184
:10AA1000FFE707E045F26510C0F60200AB2112F037
:10AA200011FFFFE74CF25030FCF796FC8DF80B005D
:10AA30009DF80B00002863D1FFE703994FF0FF302A
:10AA4000086004980068012814D1FFE70499087C85
:10AA50004968FCF7C1FA4CF25030FCF77DFC8DF8E8
:10AA60000B0043F61041C4F20201086820F0040014
:10AA7000086042E004988168C068084440B1FFE77C
:10AA800004988168C06808440C2801D8FFE707E0F3
:10AA900045F26510C0F60200C32112F0D3FEFFE7B5
:10AAA000049880680190FFE7019804998A68C96852
:10AAB0001144884220D2FFE701980499097CFCF7F1
:10AAC0009FF94CF25030FCF747FC8DF80B0043F631
:10AAD0001041C4F20201086820F0FA0008609DF8F5
:10AAE0000B0020B1FFE701980399086004E0FFE73D
:10AAF000019801300190D7E7FFE7FCF71BFAFFE769
:10AB0000FFE742F2CC31C2F2000100200876FFE7F5
:10AB10009DF80B008DF81700FFE79DF8170006B0B1
:10AB200080BD000043F61041C4F20201086840F005
:10AB3000004008600020704780B588B006900591FD
:10AB40000393029201208DF80700FFE742F2CC3018
:10AB5000C2F20000007E012804D1FFE702208DF838
:10AB60001F0069E042F2CC31C2F2000101200876F8
:10AB7000FFE7FFE7069860B1FFE70698012808D0D5
:10AB8000FFE70698022804D0FFE70698032801D1C2
:10AB9000FFE707E045F22B10C0F60200A42112F0F7
:10ABA00051FEFFE74CF25030FCF7D6FB8DF8070062
:10ABB0009DF8070098BBFFE7069830B9FFE70598B6
:10ABC0009DF80810FCF74EFA1AE00698012806D105
:10ABD000FFE70598BDF80810FCF7C6FA0FE00698E5
:10ABE000022805D1FFE705980299FCF7FDFA05E078
:10ABF0000598029A039BFCF773FAFFE7FFE7FFE76C
:10AC00004CF25030FCF7A8FB8DF8070043F61041DA
:10AC1000C4F20201086820F001000860FFE7FFE7C6
:10AC200042F2CC31C2F2000100200876FFE79DF825
:10AC300007008DF81F00FFE79DF81F0008B080BDDA
:10AC400081B000208DF8030043F61040C4F20200EA
:10AC50000068C00FD8B1FFE743F60441C4F2020117
:10AC600040F22310C4F26750086048F6AB10CCF6EF
:10AC7000EF50086043F61040C4F202000068C00FB5
:10AC800020B1FFE701208DF80300FFE7FFE79DF803
:10AC9000030001B07047000080B582B0ADF8060037
:10ACA00000208DF80500FFE79DF805000F2824DC43
:10ACB000FFE7BDF806009DF80510C840C007A8B121
:10ACC000FFE79DF8051040F27C30C2F2000050F81A
:10ACD000210050B1FFE79DF8051040F27C30C2F230
:10ACE000000050F821008047FFE7FFE7FFE79DF8ED
:10ACF000050001308DF80500D6E702B080BD0000E8
:10AD000080B582B0ADF8060043F61440C4F20100ED
:10AD10000068BDF8061008420CD0FFE7BDF8060039
:10AD200043F61441C4F201010860BDF80600FFF7C4
:10AD3000B3FFFFE702B080BD80B58EB00D900C91DF
:10AD400000200A90099008900D980021C4F2020199
:10AD5000884240D0FFE70D9840F20041C4F2020162
:10AD6000884238D0FFE70D9840F60001C4F2020196
:10AD7000884230D0FFE70D9840F60041C4F202014E
:10AD8000884228D0FFE70D9841F20001C4F2020189
:10AD9000884220D0FFE70D9841F20041C4F2020141
:10ADA000884218D0FFE70D9841F60001C4F2020175
:10ADB000884210D0FFE70D9841F60041C4F202012D
:10ADC000884208D0FFE70D9842F20001C4F2020168
:10ADD000884201D1FFE707E045F2A210C0F6020069
:10ADE000AC2112F02FFDFFE70C98008828B1FFE797
:10ADF0000C98408808B9FFE707E045F2A210C0F6BA
:10AE00000200AD2112F01EFDFFE70C9840680028FB
:10AE100049D0FFE70C984068012844D0FFE70C9820
:10AE2000406811283FD0FFE70C98406802283AD0CC
:10AE3000FFE70C984068122835D0FFE70C9840686F
:10AE40000021C1F2110188422DD0FFE70C98406823
:10AE50000021C1F22101884225D0FFE70C9840680B
:10AE60000021C1F2310188421DD0FFE70C984068F3
:10AE70000021C1F21201884215D0FFE70C9840680A
:10AE80000021C1F2220188420DD0FFE70C984068F2
:10AE90000021C1F23201884205D0FFE70C984068DA
:10AEA000032801D1FFE707E045F2A210C0F6020037
:10AEB000AE2112F0C7FCFFE70C98806850B1FFE7A5
:10AEC0000C988068012805D0FFE70C98806802285C
:10AED00001D1FFE707E045F2A210C0F60200AF2162
:10AEE00012F0B0FCFFE700200B90FFE70B980F2853
:10AEF00000F2B082FFE70B99012088400A900C987D
:10AF000000680A990840099009980A99884240F017
:10AF10009C82FFE70C98406800F00300012807D0EE
:10AF2000FFE70C98406800F0030002284BD1FFE7D0
:10AF30000C98C06878B1FFE70C98C06801280AD067
:10AF4000FFE70C98C068022805D0FFE70C98C0689E
:10AF5000032801D1FFE707E045F2A210C0F6020086
:10AF6000C12112F06FFCFFE70D98806808900B98E4
:10AF70004100032000FA01F10898884308900C98DA
:10AF8000C0680B99490000FA01F10898084308903D
:10AF900008980D9988600D98406808900B990120D9
:10AFA00000FA01F10898884308900C984068C0F3B3
:10AFB00000100B9900FA01F10898084308900898CE
:10AFC0000D994860FFE70C98406800F003000328E3
:10AFD00018D0FFE70D98C06808900B984100032037
:10AFE00000FA01F10898884308900C9880680B9942
:10AFF000490000FA01F108980843089008980D9953
:10B00000C860FFE70C98406800F00300022840F099
:10B01000EE80FFE70C980069002800F0B980FFE798
:10B020000C980069092800F0B380FFE70C980069CC
:10B03000002800F0AD80FFE70C980069002800F0C0
:10B04000A780FFE70C980069002800F0A180FFE7C7
:10B050000C980069002800F09B80FFE70C980069BD
:10B06000012800F09580FFE70C980069012800F0A6
:10B070008F80FFE70C980069022800F08980FFE7C5
:10B080000C980069022800F08380FFE70C980069A3
:10B0900002287DD0FFE70C980069032878D0FFE7ED
:10B0A0000C980069042873D0FFE70C980069042805
:10B0B0006ED0FFE70C980069042869D0FFE70C9870
:10B0C0000069052864D0FFE70C98006905285FD067
:10B0D000FFE70C98006909285AD0FFE70C9800692F
:10B0E000062855D0FFE70C980069092850D0FFE7E3
:10B0F0000C98006907284BD0FFE70C9800690728D7
:10B1000046D0FFE70C980069072841D0FFE70C986C
:10B11000006908283CD0FFE70C980069082837D060
:10B12000FFE70C980069082832D0FFE70C98006907
:10B1300009282DD0FFE70C980069092828D0FFE7DF
:10B140000C9800690A2823D0FFE70C9800690A28A8
:10B150001ED0FFE70C9800690B2819D0FFE70C9868
:10B1600000690C2814D0FFE70C9800690C280FD058
:10B17000FFE70C9800690D280AD0FFE70C980069DA
:10B180000C2805D0FFE70C9800690F2801D1FFE7D4
:10B1900007E045F2A210C0F60200DC2112F052FBDB
:10B1A000FFE70D980B996FF0030202EA5101084482
:10B1B000006A08900B9800F0070081000F2000FA49
:10B1C00001F10898884308900C9800690B9901F0E8
:10B1D0000701890000FA01F10898084308900898CF
:10B1E0000D990B9B02EA530211440862FFE70D9888
:10B1F000006808900B984100032000FA01F10898BC
:10B20000884308900C98406800F003000B994900AF
:10B2100000FA01F108980843089008980D99086011
:10B220000C98C079C006002840F10E81FFE7FFE7C7
:10B230000020079043F64400C4F20200016841F484
:10B2400080410160006800F4804007900798FFE7A4
:10B250000B9820F0030043F60801C4F201014058A6
:10B2600008900B9800F0030081000F2000FA01F114
:10B270000898884308900D980021C4F20201884282
:10B2800003D1FFE7002006905EE00D9840F20041F8
:10B29000C4F20201884203D1FFE70120059050E08B
:10B2A0000D9840F60001C4F20201884203D1FFE785
:10B2B0000220049042E00D9840F60041C4F20201E1
:10B2C000884203D1FFE70320039034E00D9841F258
:10B2D0000001C4F20201884203D1FFE7042002907A
:10B2E00026E00D9841F20041C4F20201884203D1E8
:10B2F000FFE70520019018E00D9841F60001C4F227
:10B300000201884203D1FFE7062000900AE00D9970
:10B3100041F60042C4F202020820914208BF072011
:10B320000090FFE700980190FFE701980290FFE787
:10B3300002980390FFE703980490FFE704980590B4
:10B34000FFE705980690FFE70698C0B20B9901F059
:10B350000301890000FA01F1089808430890089851
:10B360000B9921F0030143F60802C4F20102885050
:10B3700043F60040C4F2010000680890099908985B
:10B38000884308900C988079C00728B1FFE7099995
:10B39000089808430890FFE7089843F60041C4F274
:10B3A0000101086043F60440C4F2010000680890FF
:10B3B00009990898884308900C988079800700289C
:10B3C00005D5FFE70999089808430890FFE7089812
:10B3D00043F60441C4F20101086043F60840C4F298
:10B3E00001000068089009990898884308900C9813
:10B3F0008079C006002805D5FFE709990898084319
:10B400000890FFE7089843F60841C4F2010108607C
:10B4100043F60C40C4F201000068089009990898AE
:10B42000884308900C9880798006002805D5FFE7AE
:10B430000999089808430890FFE7089843F60C41DB
:10B44000C4F201010860FFE7FFE7FFE70B98013056
:10B450000B904BE50EB080BD80B582B00190ADF889
:10B460000210BDF8020020B1FFE7002008B9FFE795
:10B4700008E045F2A210C0F602004FF4BD7112F0D0
:10B48000E1F9FFE701980069BDF80210084204D015
:10B49000FFE701208DF8010003E000208DF8010096
:10B4A000FFE79DF8010002B080BD000080B582B0CA
:10B4B0000190ADF802108DF80120BDF8020020B116
:10B4C000FFE7002008B9FFE708E045F2A210C0F648
:10B4D000020040F29B1112F0B5F9FFE79DF8010060
:10B4E00028B1FFE79DF80100012801D1FFE708E03E
:10B4F00045F2A210C0F602004FF4CE7112F0A2F98C
:10B50000FFE79DF8010028B1FFE7BDF802000199AF
:10B51000886105E0BDF80200000401998861FFE739
:10B5200002B080BD49F24060C2F20000006870477E
:10B5300080B58EB00C900C9820B9FFE701208DF8F3
:10B54000370002E20C98006845F20041C4F20001A5
:10B55000884212D0FFE70C98006845F60001C4F25B
:10B560000001884209D0FFE70C98006845F60041C9
:10B57000C4F20001884201D1FFE708E045F2F6205D
:10B58000C0F6020040F2BF1112F05CF9FFE70C9820
:10B59000406850B1FFE70C98406841F68021C0F246
:10B5A0000601884201D8FFE708E045F2F620C0F620
:10B5B00002004FF4E07112F045F9FFE70C98806843
:10B5C00030B1FFE70C988068B0F5804F01D1FFE7FC
:10B5D00008E045F2F620C0F6020040F2C11112F078
:10B5E00031F9FFE70C98C068800A08B9FFE708E066
:10B5F00045F2F620C0F602004FF4E17112F022F994
:10B60000FFE70C980069B0F5804F06D0FFE70C9873
:10B610000069B0F5404F01D1FFE708E045F2F620A0
:10B62000C0F6020040F2C31112F00CF9FFE70C98CB
:10B63000406928B1FFE70C984069012801D1FFE774
:10B6400008E045F2F620C0F602004FF4E27112F075
:10B65000F9F8FFE70C9880696FF0FE01084201D10C
:10B66000FFE708E045F2F620C0F6020040F2C511FF
:10B6700012F0E8F8FFE70C98C06928B1FFE70C98D2
:10B68000C069402801D1FFE708E045F2F620C0F686
:10B6900002004FF4E37112F0D5F8FFE70C98006A4E
:10B6A00028B1FFE70C98006A802801D1FFE708E085
:10B6B00045F2F620C0F6020040F2C71112F0C2F8BF
:10B6C000FFE70C9890F83D0040B9FFE70C99002087
:10B6D00081F83C000C9800F03DF9FFE70C9924201C
:10B6E00081F83D000C980168086820F001000860AE
:10B6F0000C980168086840F4004008600C980168E4
:10B70000086820F40040086001F054FE0A900C988C
:10B71000406848F2A061C0F2010188420BD8FFE7FF
:10B720000A9948F28042C0F21E020020914238BFBE
:10B73000012009900AE00A9940F60012C0F23D0289
:10B740000020914238BF01200990FFE709980128A5
:10B7500004D1FFE701208DF83700F6E00A984DF696
:10B760008361C4F21B31A0FB0110800C0B900C987C
:10B770000068406820F03F000B9908430C99096865
:10B7800048600C980068006A20F03F0008900C9810
:10B79000406848F2A061C0F20101884204D8FFE786
:10B7A0000B98013007900EE00B984FF496714843C8
:10B7B00044F6D351C1F26201A0FB0101012000EB6C
:10B7C00091100790FFE70898079908430C990968BA
:10B7D00008620C980068C0694CF6FF7188430690B7
:10B7E0000C98406848F2A061C0F2010188421FD85D
:10B7F000FFE70A9801380C9949684900B0FBF1F05D
:10B8000001306FF31F30032803D8FFE704200590B1
:10B810000BE00A9801380C9949684900B0FBF1F037
:10B8200001306FF31F300590FFE7059804904CE05E
:10B830000C98806868B9FFE70A9801380C99496844
:10B8400001EB4101B0FBF1F001306FF31F300390C9
:10B850000DE00A9801380C99496819225143B0FB50
:10B86000F1F00130042161F31F300390FFE70398EA
:10B87000000518B9FFE70120029023E00C988068CA
:10B8800068B9FFE70A9801380C99496801EB410152
:10B89000B0FBF1F001306FF31F3001900DE00A981A
:10B8A00001380C99496819225143B0FBF1F001307D
:10B8B000042161F31F300190FFE7019840F400403C
:10B8C0000290FFE702980490FFE706980499084366
:10B8D0000C990968C8610C980068006820F0C000E5
:10B8E0000C9B1968DA691B6A1A43104308600C98AC
:10B8F0000068806848F2FF3188430C9A1168D36869
:10B9000012691A43104388600C980068C06820F0E0
:10B91000FF000C9B19685A699B691A431043C86061
:10B920000C980168086840F0010008600C9900203C
:10B9300008640C9A202182F83D100C9908630C9938
:10B9400081F83E008DF83700FFE79DF837000EB014
:10B9500080BD000080B594B013900020129011902B
:10B9600010900F900E901398006845F20041C4F2B9
:10B970000001884235D1FFE7FFE700200D9043F634
:10B980003000C4F20200016841F002010160006869
:10B9900000F002000D900D98FFE74FF440700E90FC
:10B9A00012200F900120109003201190042012907B
:10B9B00040F20040C4F202000EA9FFF7BDF9FFE714
:10B9C00000200C9043F64000C4F20200016841F4EC
:10B9D00000110160006800F400100C900C98FFE763
:10B9E000FBE01398006845F60001C4F200018842AC
:10B9F0005FD1FFE7FFE700200B9043F63000C4F271
:10BA00000200016841F020010160006800F02000A0
:10BA10000B900B98FFE703200E9012210F9101214C
:10BA2000109111900420129041F20040C4F20200E3
:10BA30000EA9FFF781F9FFE700200A9043F64000C6
:10BA4000C4F20200016841F480010160006800F462
:10BA500080000A900A98FFE741F26C70C2F2000081
:10BA6000069046F2B801C4F2020101604FF0606135
:10BA70004160402181600021C1604FF48062026119
:10BA800041618161C1614FF4003202624162FEF79F
:10BA900069FC18B1FFE7FBF7AFF9FFE7FFE7139881
:10BAA00041F26C71C2F20001416313988863FFE7B1
:10BAB00092E01398006845F60041C4F20001884204
:10BAC00040F08980FFE7FFE70020099043F630004F
:10BAD000C4F20200016841F004010160006800F056
:10BAE000040009900998FFE7FFE70020089043F65B
:10BAF0003000C4F20200016841F0010101600068F9
:10BB000000F0010008900898FFE74FF400700E90D5
:10BB1000122001900F9001200290109003200390BA
:10BB2000119004200490129040F60000C4F202002C
:10BB30000EA90591FFF700F9DDF804C0029B039AF6
:10BB4000049805994FF4807ECDF838E0CDF83CC0DC
:10BB50001093119212900020C4F20200FFF7ECF84B
:10BB6000FFE70020079043F64000C4F2020001689E
:10BB700041F400010160006800F40000079007989C
:10BB8000FFE741F2CC70C2F20000009046F24001A3
:10BB9000C4F2020101604FF0C06141600021816088
:10BBA000C1604FF48062026141618161C1610162E3
:10BBB0004162FEF7D7FB18B1FFE7FBF71DF9FFE77E
:10BBC000FFE7139841F2CC71C2F200018163139830
:10BBD0008863FFE7FFE7FFE7FFE714B080BD0000E1
:10BBE00040F2E020C2F20000027849F24061C2F265
:10BBF00000010868104408607047000080B543F6F3
:10BC00000041C4F20201086840F40070086008684E
:10BC100040F480600860086840F480700860032089
:10BC200000F0D0F80F2000F005F800F03BF80020FD
:10BC300080BD000080B582B0009040F22800C2F2C2
:10BC40000000006840F2E021C2F200010A784FF4DF
:10BC50007A71B1FBF2F1B0FBF1F003F005FB20B11A
:10BC6000FFE701208DF8070018E000980F280DD895
:10BC7000FFE700994FF0FF30002200F06FF80098C6
:10BC800040F2E421C2F20001086003E001208DF8D7
:10BC9000070003E000208DF80700FFE79DF807008C
:10BCA00002B080BD80B582B0FFE70020019043F66E
:10BCB0004400C4F20200016841F480410160006860
:10BCC00000F4804001900198FFE7FFE7002000901A
:10BCD00043F64000C4F20200016841F08051016067
:10BCE000006800F0805000900098FFE76FF00100BE
:10BCF0000F21002200F032F802B080BD80B582B082
:10BD00008DF807009DF90700002801D4FFE707E040
:10BD100045F21320C0F60200CE2111F093FDFFE79B
:10BD20009DF9070011F0F0FC02B080BD80B582B033
:10BD30008DF807009DF90700002801D4FFE707E010
:10BD400045F21320C0F60200BE2111F07BFDFFE793
:10BD50009DF9070011F0F4FC02B080BD80B586B0FB
:10BD60008DF81700049103920020029003980F2889
:10BD700001D8FFE707E045F21320C0F60200AA2130
:10BD800011F060FDFFE704980F2801D8FFE707E0F6
:10BD900045F21320C0F60200AB2111F053FDFFE77E
:10BDA00011F0E6FC02909DF91700019002980499A9
:10BDB000039A07F0C5FE0146019811F0E1FC06B0B8
:10BDC00080BD000080B582B001900198072810D096
:10BDD000FFE7019806280CD0FFE70198052808D056
:10BDE000FFE70198042804D0FFE70198032801D158
:10BDF000FFE707E045F21320C0F60200922111F0A0
:10BE000021FDFFE7019811F0FFFC02B080BD0000AA
:10BE100082B001908DF8031002B0704782B001909B
:10BE2000ADF80210BDF802000199096848620020CF
:10BE300002B0704784B003908DF80B10ADF8082065
:10BE400003980068406A00909DF80B0048B9FFE72E
:10BE5000BDF80810009840EA01400399096888621B
:10BE600033E003980068816A009800EB114000906D
:10BE700000208DF80700FFE79DF807009DF80B10E4
:10BE80000139884213D2FFE7039800689DF8071034
:10BE900000EB8100D0F80411009800EB11400090F5
:10BEA000FFE79DF8070001308DF80700E4E7BDF8D3
:10BEB0000810009840EA0140039909689DF80B209A
:10BEC00001EB8201C1F80001FFE7002004B07047D8
:10BED00080B582B001900198D0F804040FF072FB95
:10BEE00002B080BD80B582B001908DF80310019A38
:10BEF000D2F804049DF80310C1EBC10302EB8302E6
:10BF0000926C0FF03DFA02B080BD000080B582B0A7
:10BF100001908DF80310019AD2F804049DF80310E3
:10BF2000C1EBC10302EB8302D2F808220FF0CEFA74
:10BF300002B080BD80B582B001900198D0F80404B1
:10BF40000FF046FB02B080BD80B584B002908DF842
:10BF500007109DF80700000600280FD5FFE702989C
:10BF60009DF8071001F00F01C1EBC10100EB81004A
:10BF70003C3000900099012048700FE002989DF835
:10BF8000071001F00F01C1EBC10100EB810000F5CA
:10BF9000FE700090009900204870FFE79DF80700B0
:10BFA00000F00F0000990870FFE7029890F8BC03BA
:10BFB000012804D1FFE702208DF80F0014E0029958
:10BFC000012081F8BC03FFE7FFE7029800680099B1
:10BFD00010F0C2FAFFE70299002081F8BC03FFE7E6
:10BFE00000208DF80F00FFE79DF80F0004B080BD22
:10BFF00080B584B002908DF807109DF8070000F01E
:10C000000F0002994968884204D9FFE701208DF8A2
:10C010000F004DE09DF80700000600280FD5FFE750
:10C0200002989DF8071001F00F01C1EBC10100EB70
:10C0300081003C3000900099012048700FE0029888
:10C040009DF8071001F00F01C1EBC10100EB810069
:10C0500000F5FE700090009900204870FFE70099FD
:10C06000002088709DF8070000F00F00009908700C
:10C07000FFE7029890F8BC03012804D1FFE70220F3
:10C080008DF80F0014E00299012081F8BC03FFE74E
:10C09000FFE702980068009910F0E2FDFFE70299BF
:10C0A000002081F8BC03FFE700208DF80F00FFE7B8
:10C0B0009DF80F0004B080BD82B001908DF8031090
:10C0C00001989DF8031001F00F01C1EBC10100EBD5
:10C0D0008100D0F8140202B07047000080B586B02D
:10C0E00004908DF80F10ADF80C208DF80B30002067
:10C0F0008DF80A009DF80F00000600280FD5FFE715
:10C1000004989DF80F1001F00F01C1EBC10100EB85
:10C1100081003C3001900199012048700FE00498A3
:10C120009DF80F1001F00F01C1EBC10100EB810080
:10C1300000F5FE700190019900204870FFE79DF81E
:10C140000F0000F00F0001990870BDF80C00019974
:10C1500088609DF80B000199C8700198407820B163
:10C16000FFE701990878C880FFE79DF80B000228D7
:10C1700004D1FFE7019900200871FFE7FFE7049869
:10C1800090F8BC03012804D1FFE702208DF81700C6
:10C1900015E00499012081F8BC03FFE7FFE704984C
:10C1A0000068019910F094F8FFE70499002081F8E5
:10C1B000BC03FFE79DF80A008DF81700FFE79DF824
:10C1C000170006B080BD000080B586B005908DF8E0
:10C1D00013100392029305989DF8131001F00F01BC
:10C1E000C1EBC10100EB810000F5FE7001900398E6
:10C1F0000199C860029801994861019900208861FD
:10C20000019948709DF8130000F00F000199087023
:10C2100005980069012804D1FFE703980199086196
:10C22000FFE79DF81300000738B9FFE7059A10688B
:10C230000199127C10F0CCFB06E0059A1068019978
:10C24000127C10F0B1FDFFE7002006B080BD0000B9
:10C2500080B584B002908DF807109DF8070000F0BB
:10C260000F0002994968884204D9FFE701208DF840
:10C270000F0058E09DF80700000600280FD5FFE7E3
:10C2800002989DF8071001F00F01C1EBC10100EB0E
:10C2900081003C3000900099012048700DE0029828
:10C2A0009DF80710C1EBC10100EB810000F5FE70A5
:10C2B0000090009900204870FFE7009901208870E5
:10C2C0009DF8070000F00F0000990870FFE7029842
:10C2D00090F8BC03012804D1FFE702208DF80F007D
:10C2E00021E00299012081F8BC03FFE7FFE70298F3
:10C2F0000068009910F004FD9DF80700000740B9A0
:10C30000FFE7029A1068117C02F5717210F058FC78
:10C31000FFE7FFE70299002081F8BC03FFE7002058
:10C320008DF80F00FFE79DF80F0004B080BD0000FE
:10C3300080B586B005908DF813100392029305988E
:10C340009DF8131001F00F01C1EBC10100EB81005A
:10C350003C30019003980199C860029801994861A6
:10C360000199002088610199012048709DF813000F
:10C3700000F00F000199087005980069012804D1A8
:10C38000FFE7039801990861FFE79DF81300000794
:10C3900038B9FFE7059A10680199127C10F018FB74
:10C3A00006E0059A10680199127C10F0FDFCFFE789
:10C3B000002006B080BD000080B58CB00B900B98BB
:10C3C00000680A900A9809900B98006810F01EFF08
:10C3D000002840F01A83FFE70B98006810F082FFF6
:10C3E00008B9FFE711E30B98006810F07BFF8007A6
:10C3F000002807D5FFE70B980168486900F00200A4
:10C400004861FFE70B98006810F06CFFC006002839
:10C4100062D5FFE70B980168886920F010008861F9
:10C420000A98006A03900B98039901F00F01C1EB81
:10C43000C10100EB810000F5FE700290039800F44A
:10C44000F0110220B0EB514F23D1FFE7BDF80C00F3
:10C4500047F6F07108421BD0FFE70A980299C968B5
:10C46000039AC2F30A1210F04BFF039847F6F071DB
:10C4700000EA0103029AD06800EB1310D060039821
:10C4800000EA01020299886900EB12108861FFE757
:10C490001BE0039800F4F0110620B0EB514F12D1CD
:10C4A000FFE70A980B9901F57171082210F028FF37
:10C4B000039847F6F07100EA01020299886900EBDF
:10C4C0001210886100E0FFE7FFE70B9801688869B8
:10C4D00040F010008861FFE70B98006810F002FF41
:10C4E0000003002870D5FFE7002005900B98006836
:10C4F00010F0A6FE0790FFE70798002863D0FFE73B
:10C500009DF81C00C007002856D0FFE70B98006874
:10C510009DF8141010F0CEFE06909DF81800C0078C
:10C5200060B1FFE70998059900EB41110120C1F8BE
:10C53000080B0B98059907F087FBFFE79DF818009B
:10C54000000700280CD5FFE70998059900EB411179
:10C550000820C1F8080B0B98059907F02FFBFFE79F
:10C560009DF81800C006002808D5FFE7099805992E
:10C5700000EB41111020C1F8080BFFE79DF81800EF
:10C580008006002808D5FFE70998059900EB4111BE
:10C590002020C1F8080BFFE79DF81900800600284D
:10C5A00009D5FFE70998059900EB41114FF40050B8
:10C5B000C1F8080BFFE7FFE70598013005900798E1
:10C5C0004008079098E7FFE70B98006810F08AFE94
:10C5D0004003002840F1AC80FFE70B98006810F0A2
:10C5E0001DFE079000200590FFE70798002800F047
:10C5F0009E80FFE79DF81C00C007002800F0908097
:10C60000FFE70B9800689DF8141010F02BFE0690C1
:10C610009DF81800C00700283ED0FFE7059800F0FD
:10C620000F01012000FA01F10491049B099AD2F84C
:10C6300034189943C2F834180999059A01EB42114C
:10C64000C1F808090B98006901281FD1FFE70B9872
:10C650000599C1EBC10100EB81014A6C886C104463
:10C660008864059888B9FFE70B980599C1EBC1016B
:10C6700000EB8100006D40B9FFE70B99086801F5F8
:10C680007172012110F09CFAFFE7FFE70B989DF80B
:10C690001410FFF727FCFFE79DF81800000700289B
:10C6A00008D5FFE70998059900EB41110820C1F86A
:10C6B0000809FFE79DF81800C006002808D5FFE725
:10C6C0000998059900EB41111020C1F80809FFE70E
:10C6D0009DF818004006002808D5FFE7099805993D
:10C6E00000EB41114020C1F80809FFE79DF8180050
:10C6F0008007002808D5FFE70998059900EB41114C
:10C700000220C1F80809FFE79DF81800000600287C
:10C7100005D5FFE70B98059907F088FBFFE7FFE7D2
:10C720000598013005900798400807905DE7FFE7FE
:10C730000B98006810F0D6FDC00F00B3FFE7099911
:10C74000D1F8040820F00100C1F804080B9890F813
:10C75000F403012808D1FFE70B98002180F8F413B7
:10C760000B98FFF755FB03E00B9800F061FBFFE728
:10C770000B980168486900F000404861FFE70B989A
:10C78000006810F0AFFD0005002811D5FFE70998FB
:10C79000D0F80808C00720B1FFE70B9800F0D6FBDF
:10C7A000FFE70B980168486900F400604861FFE703
:10C7B0000B98006810F096FDC004002840F19080AE
:10C7C000FFE70999D1F8040820F00100C1F8040836
:10C7D0000B980068102110F0C9FC00200890FFE7BA
:10C7E00008980B99496888423BD2FFE70998089955
:10C7F00000EB41114FF67F30C1F808090999089AFA
:10C8000001EB4212D2F8001921F40011C2F800190C
:10C810000999089A01EB4212D2F8001941F000611F
:10C82000C2F800190999089A01EB4211C1F8080BE6
:10C830000998089900EB4111D1F8000B20F4001081
:10C84000C1F8000B0998089900EB4111D1F8000BD1
:10C8500040F00060C1F8000BFFE708980130089035
:10C86000BEE70999D1F81C0840F00110C1F81C0876
:10C870000B98006B78B1FFE70999D1F8840840F074
:10C880000B00C1F884080999D1F8440840F00B0066
:10C89000C1F844080FE00999D1F8140842F22B02BC
:10C8A0001043C1F814080999D1F8100840F00B00A2
:10C8B000C1F81008FFE70999D1F8000820F4FE60DC
:10C8C000C1F800080B9A1068117C02F5717210F023
:10C8D00077F90B980168486900F480504861FFE7D8
:10C8E0000B98006810F0FEFC800400281FD5FFE7BD
:10C8F0000B9800680FF05CFD0B98006810F060FC6E
:10C900000B99C8600B980068019000F04DFD01463E
:10C9100001980B9A127B10F079FD0B9800F05EFAEB
:10C920000B980168486900F400504861FFE70B98D4
:10C93000006810F0D7FC000700280AD5FFE70B9825
:10C9400000F080FA0B980168486900F0080048611F
:10C95000FFE70B98006810F0C5FCC00200280ED558
:10C96000FFE7002005900B989DF8141000F050F898
:10C970000B980168486900F480104861FFE70B9844
:10C98000006810F0AFFC800200280ED5FFE7002001
:10C9900005900B989DF8141000F048F80B9801686A
:10C9A000486900F400104861FFE70B98006810F038
:10C9B00099FC400000280AD5FFE70B98FFF788FA9A
:10C9C0000B980168486900F080404861FFE70B98C8
:10C9D000006810F087FC4007002815D5FFE70B988A
:10C9E0000068406803909DF80C004007002804D5BB
:10C9F000FFE70B98FFF79EFAFFE7039A0B98016891
:10CA0000486810434860FFE7FFE70CB080BD0000B6
:10CA100080B582B001908DF803100198D0F804041D
:10CA20009DF803100EF066FE02B080BD80B582B0A6
:10CA300001908DF803100198D0F804049DF80310BC
:10CA40000EF084FE02B080BD2DE9F04F97B0159036
:10CA5000159820B9FFE701208DF85B0060E115987B
:10CA60000068B0F1A04F08D0FFE7159800680021DA
:10CA7000C4F20401884201D1FFE707E045F2BB00A0
:10CA8000C0F60200872110F0DDFEFFE71598006870
:10CA90001490159890F8BD0340B9FFE71599002050
:10CAA00081F8BC03159800F041F9FFE715990320C0
:10CAB00081F8BD031498C06BC005002804D4FFE7BB
:10CAC000159900200861FFE7159800680FF076FFC0
:10CAD000159810900168119141688268C368D0F878
:10CAE00010C044698569C669076AD0F82480D0F807
:10CAF0002890D0F82CA0D0F830B0D0F834E06846B8
:10CB00001290C0F824E01198DDF848E0CEF820B08B
:10CB1000CEF81CA0CEF81890CEF81480CEF8107085
:10CB2000CEF80C60CEF80850CEF80440CEF800C025
:10CB30000FF054FC40B1FFE71599022081F8BD03C6
:10CB400001208DF85B00EBE01598006800210F9143
:10CB500010F0FEFB0F988DF84F00FFE79DF84F0097
:10CB600015994968884245D2FFE715989DF84F10FE
:10CB7000C1EBC10100EB8101012081F83D009DF86E
:10CB80004F001599C0EBC00201EB820181F83C0017
:10CB90009DF84F001599C0EBC00201EB8201A1F88E
:10CBA000420015989DF84F10C1EBC10100EB8101C7
:10CBB000002081F83F0015999DF84F20C2EBC2027A
:10CBC00001EB8201486415999DF84F20C2EBC20227
:10CBD00001EB8201886415999DF84F20C2EBC202D7
:10CBE00001EB82010865FFE79DF84F0001308DF8E9
:10CBF0004F00B3E700208DF84F00FFE79DF84F008E
:10CC00001599496888423ED2FFE715989DF84F1064
:10CC1000C1EBC10100EB8101002081F8FD019DF80D
:10CC20004F10159AC1EBC10302EB830282F8FC118D
:10CC300015999DF84F20C2EBC20201EB820181F8E9
:10CC4000FF0115999DF84F20C2EBC20201EB820152
:10CC5000C1F8040215999DF84F20C2EBC20201EB06
:10CC60008201C1F8080215999DF84F20C2EBC2025B
:10CC700001EB8201C1F81002FFE79DF84F0001307F
:10CC80008DF84F00BAE715980C9001680D91416836
:10CC90008268C368D0F810C044698569C669076AAC
:10CCA000D0F82480D0F82890D0F82CA0D0F830B05C
:10CCB000D0F834E068460E90C0F824E00D98DDF816
:10CCC00038E0CEF820B0CEF81CA0CEF81890CEF800
:10CCD0001480CEF81070CEF80C60CEF80850CEF864
:10CCE0000440CEF800C00FF007FD40B1FFE71599F2
:10CCF000022081F8BD0301208DF85B0010E015993A
:10CD000000200B9081F838001599012081F8BD03AF
:10CD1000159800680FF0DAFC0B988DF85B00FFE7C0
:10CD20009DF85B0017B0BDE8F08F000080B58AB0B9
:10CD300009900020089007900690059004900998AB
:10CD40000068B0F1A04F47D1FFE7FFE70020039054
:10CD500043F63000C4F20200016841F001010160B5
:10CD6000006800F0010003900398FFE74FF4C05003
:10CD700004900220059000200690032007900A20CE
:10CD800008900020C4F2020004A9FDF7D5FFFFE7D8
:10CD900043F63401C4F20201086840F080000860E4
:10CDA000FFE70020029043F64400C4F2020001684D
:10CDB00041F480410160006800F4804002900298D4
:10CDC000FFE7FFE74320019005210022FEF7C6FFA1
:10CDD0000198FEF7ABFFFFE70AB080BD80B582B0D7
:10CDE000019001208DF803000198C06820B9FFE789
:10CDF00000208DF803000CE00198C068022804D1DF
:10CE0000FFE701208DF8030002E0F9F7F5FFFFE7E7
:10CE1000FFE70198D0F804049DF803100EF094FD8C
:10CE20000198D0F804040EF005FD02B080BD0000AA
:10CE300080B582B001900198D0F804040EF04AFD4C
:10CE400002B080BD80B582B001900198D0F8040492
:10CE50000EF052FD02B080BD80B584B002908DF816
:10CE60000710FFE7029890F8BC03012804D1FFE700
:10CE700002208DF80F001AE00299012081F8BC030E
:10CE8000FFE7FFE79DF80700029981F83800029854
:10CE900000689DF8071010F08BFAFFE70299002058
:10CEA00081F8BC03FFE700208DF80F00FFE79DF835
:10CEB0000F0004B080BD000080B582B001900199E0
:10CEC000D1F8040401F571710EF068FD02B080BD67
:10CED00080B584B00290029800680190FFE7029844
:10CEE00090F8BC03012804D1FFE702208DF80F0061
:10CEF00027E00299012081F8BC03FFE7FFE70298D1
:10CF0000806A01280BD1FFE702988069012806D0CA
:10CF1000FFE70199886B40F480308863FFE702984F
:10CF2000006810F0F3F8029800680FF0B9FBFFE713
:10CF30000299002081F8BC03FFE700208DF80F0064
:10CF4000FFE79DF80F0004B080BD000080B582B0FF
:10CF500001900198D0F804040EF0A2FD0198016838
:10CF6000D1F8000E40F00100C1F8000E0198006AEF
:10CF700048B1FFE74EF61051CEF20001086840F0CC
:10CF800006000860FFE702B080BD000080B584B0F5
:10CF900002900191029820B9FFE701208DF80F005F
:10CFA000FDE10298006830B1FFE7029800680F28A1
:10CFB00001D8FFE708E045F2F300C0F602004FF4A5
:10CFC000177110F03FFCFFE70198E0B1FFE701980F
:10CFD000012818D0FFE70198022814D0FFE7019834
:10CFE000032810D0FFE7019804280CD0FFE7019830
:10CFF000052808D0FFE70198062804D0FFE701982C
:10D00000072801D1FFE708E045F2F300C0F602006F
:10D0100040F25D2110F016FCFFE7019843F6004155
:10D02000C4F20201096801F00701884212D9FFE742
:10D03000019943F60040C4F202000170006800F05C
:10D0400007000199884204D0FFE701208DF80F0006
:10D05000A5E1FFE7029800788007002860D5FFE788
:10D06000029800784007002809D5FFE743F6080139
:10D07000C4F20201086840F4E0500860FFE702983B
:10D0800000780007002809D5FFE743F60801C4F23D
:10D090000201086840F460400860FFE70298806879
:10D0A00040B3FFE702988068802823D0FFE702980A
:10D0B000806890281ED0FFE702988068A02819D0C9
:10D0C000FFE702988068B02814D0FFE702988068D4
:10D0D000C0280FD0FFE702988068D0280AD0FFE769
:10D0E00002988068E02805D0FFE702988068F02861
:10D0F00001D1FFE708E045F2F300C0F602004FF46B
:10D10000207110F09FFBFFE743F60801C4F2020113
:10D11000086820F0F000029A926810430860FFE768
:10D1200002980078C007002800F08C80FFE7029882
:10D13000406878B1FFE70298406801280AD0FFE70D
:10D1400002984068022805D0FFE70298406803284B
:10D1500001D1FFE708E045F2F300C0F6020040F21B
:10D16000872110F06FFBFFE702984068012811D17A
:10D17000FFE743F60000C4F20200006800F400314B
:10D180000020B0EB514F04D1FFE701208DF80F00D4
:10D1900005E12CE002984068022805D0FFE70298DC
:10D1A0004068032811D1FFE743F60000C4F20200F3
:10D1B000006800F000710020B0EB516F04D1FFE770
:10D1C00001208DF80F00EAE010E043F60000C4F201
:10D1D0000200006800F002010020B0EB510F04D102
:10D1E000FFE701208DF80F00D9E0FFE7FFE743F6E6
:10D1F0000801C4F20201086820F00300029A526894
:10D2000010430860FEF78EF90090FFE743F6080030
:10D21000C4F20200006800F00C0002994968B0EB0B
:10D22000810F0ED0FFE7FEF77DF90099401A41F219
:10D230008931884204D3FFE703208DF80F00AEE068
:10D24000E4E7FFE7019843F60041C4F202010968F0
:10D2500001F00701884212D2FFE7019943F600402E
:10D26000C4F202000170006800F0070001998842D2
:10D2700004D0FFE701208DF80F0090E0FFE702984F
:10D2800000784007002832D5FFE70298C068C0B197
:10D29000FFE70298C068B0F5805F12D0FFE7029800
:10D2A000C068B0F5A05F0CD0FFE70298C068B0F589
:10D2B000C05F06D0FFE70298C068B0F5E05F01D11B
:10D2C000FFE708E045F2F300C0F6020040F2C52196
:10D2D00010F0B8FAFFE743F60801C4F2020108684B
:10D2E00020F4E050029AD26810430860FFE70298E9
:10D2F00000780007002833D5FFE702980069C0B125
:10D30000FFE702980069B0F5805F12D0FFE702984E
:10D310000069B0F5A05F0CD0FFE702980069B0F596
:10D32000C05F06D0FFE702980069B0F5E05F01D169
:10D33000FFE708E045F2F300C0F602004FF4337156
:10D3400010F080FAFFE743F60801C4F20201086812
:10D3500020F46040029A126940EAC2000860FFE7C8
:10D3600000F04CF843F60801C4F202010968C9B2A2
:10D370000A0944F6D001C0F60201895CC84040F2B7
:10D380002801C2F20001086040F2E420C2F200006D
:10D390000068FEF74FFC00208DF80F00FFE79DF8B6
:10D3A0000F0004B080BD000040F22800C2F200006F
:10D3B0000068704780B5FFF7F7FF43F60801C4F235
:10D3C00002010968C1F3822244F6E001C0F60201BD
:10D3D000895CC84080BD000080B5FFF7E5FF43F6DB
:10D3E0000801C4F20201096889B24A0B44F6E0015F
:10D3F000C0F60201895CC84080BD000080B586B0DF
:10D400000020059004900390029043F60800C4F2B7
:10D410000200006800F00C000146019140B1FFE7F6
:10D42000019804280AD0FFE7019808280CD04FE0A3
:10D4300042F20040C0F2F40002904FE041F60030AA
:10D44000C0F2B700029049E043F60400C4F20200C3
:10D45000016801F03F01059100684002002813D5E2
:10D46000FFE743F60400C4F202000068C0F388102E
:10D4700041F60031C0F2B701A0FB0101059A00237B
:10D48000F2F79EFE049012E043F60400C4F202009C
:10D490000068C0F3881042F20041C0F2F401A0FB22
:10D4A0000101059A0023F2F78BFE0490FFE743F693
:10D4B0000400C4F20200006800F44031022000EBD6
:10D4C000D130039004980399B0FBF1F0029005E08D
:10D4D00042F20040C0F2F4000290FFE7029806B06A
:10D4E00080BD000080B586B00490049828B9FFE79D
:10D4F00001208DF8170000F048BC049800680F2840
:10D5000001D8FFE707E045F2F300C0F60200E8218A
:10D5100010F098F9FFE704980078C007002800F0A1
:10D52000BE80FFE70498406860B1FFE70498406858
:10D53000B0F5803F06D0FFE704984068B0F5A02F13
:10D5400001D1FFE707E045F2F300C0F60200ED214C
:10D5500010F078F9FFE743F60800C4F20200006813
:10D5600000F00C00042813D0FFE743F60800C4F2D3
:10D570000200006800F00C0008281ED1FFE743F607
:10D580000400C4F2020000684002002815D5FFE73D
:10D5900043F60000C4F20200006800F400310020ED
:10D5A000B0EB514F08D0FFE70498406820B9FFE77F
:10D5B00001208DF81700E8E370E0FFE70498406869
:10D5C000B0F5803F09D1FFE743F60001C4F2020144
:10D5D000086840F48030086020E004984068B0F5A6
:10D5E000A02F0DD1FFE743F60001C4F20201086845
:10D5F00040F480200860086840F4803008600CE047
:10D6000043F60001C4F20201086820F4803008608B
:10D61000086820F480200860FFE7FFE7FFE7049830
:10D620004068E8B1FFE7FDF77DFF0390FFE743F6B1
:10D630000000C4F20200006800F400310020B0EBEA
:10D64000514F0CD1FFE7FDF76DFF0399401A652894
:10D6500004D3FFE703208DF8170096E3E7E71CE00B
:10D66000FDF760FF0390FFE743F60000C4F20200FD
:10D67000006800F400310020B0EB514F0CD0FFE700
:10D68000FDF750FF0399401A652804D3FFE70320F4
:10D690008DF8170079E3E7E7FFE7FFE7FFE7049876
:10D6A00000788007002840F1B880FFE70498C06840
:10D6B00028B1FFE70498C068012801D1FFE708E01E
:10D6C00045F2F300C0F6020040F21F1110F0BAF864
:10D6D000FFE7049800691F2801D8FFE708E045F23A
:10D6E000F300C0F602004FF4907110F0ABF8FFE7C2
:10D6F00043F60800C4F20200006810F00C0F13D0CB
:10D70000FFE743F60800C4F20200006800F00C00D6
:10D7100008282CD1FFE743F60400C4F20200006899
:10D720004002002823D4FFE743F60000C4F20200C1
:10D73000006800F002010020B0EB510F09D0FFE7B4
:10D740000498C068012804D0FFE701208DF8170075
:10D750001BE343F60001C4F20201086820F0F80060
:10D76000049A126940EAC2000860FFE754E0049896
:10D77000C06870B3FFE70021C4F2472101200860B0
:10D78000FDF7D0FE0390FFE743F60000C4F202006D
:10D79000006800F002010020B0EB510F0CD1FFE750
:10D7A000FDF7C0FE0399401A032804D3FFE70320C6
:10D7B0008DF81700E9E2E7E743F60001C4F2020141
:10D7C000086820F0F800049A126940EAC200086074
:10D7D00021E00021C4F2472100200860FDF7A2FEED
:10D7E0000390FFE743F60000C4F20200006800F077
:10D7F00002010020B0EB510F0CD0FFE7FDF792FEC5
:10D800000399401A032804D3FFE703208DF817007B
:10D81000BBE2E7E7FFE7FFE7FFE7049800780007D0
:10D8200000285ED5FFE70498406928B1FFE7049817
:10D830004069012801D1FFE708E045F2F300C0F696
:10D8400002004FF4B0710FF0FDFFFFE7049840694C
:10D8500018B3FFE740F68061C4F247210120086059
:10D86000FDF760FE0390FFE743F67400C4F2020088
:10D87000006800F002010020B0EB510F0CD1FFE76F
:10D88000FDF750FE0399401A032804D3FFE7032055
:10D890008DF8170079E2E7E722E040F68061C4F2F4
:10D8A000472100200860FDF73DFE0390FFE743F6A7
:10D8B0007400C4F20200006800F002010020B0EB26
:10D8C000510F0CD0FFE7FDF72DFE0399401A0328F6
:10D8D00004D3FFE703208DF8170056E2E7E7FFE7E0
:10D8E000FFE7049800784007002840F1E680FFE752
:10D8F00000208DF807000498806850B1FFE7049875
:10D900008068012805D0FFE704988068052801D1C8
:10D91000FFE708E045F2F300C0F602004FF4C671DD
:10D920000FF090FFFFE743F64000C4F202000068EA
:10D93000C000002815D4FFE7FFE70020009043F661
:10D940004000C4F20200016841F0805101600068AB
:10D9500000F0805000900098FFE701208DF807004C
:10D96000FFE747F20000C4F200000068C00500288D
:10D9700022D4FFE747F20001C4F20001086840F436
:10D9800080700860FDF7CEFD0390FFE747F20000CE
:10D99000C4F200000068C00500280CD4FFE7FDF7C2
:10D9A000C1FD0399401A032804D3FFE703208DF833
:10D9B0001700EAE1EAE7FFE7FFE70498806801283B
:10D9C00009D1FFE743F67001C4F20201086840F094
:10D9D000010008601FE00498806805280DD1FFE76A
:10D9E00043F67001C4F20201086840F004000860C8
:10D9F000086840F0010008600CE043F67001C4F2D2
:10DA00000201086820F001000860086820F00400A6
:10DA10000860FFE7FFE7FFE704988068F8B1FFE7D9
:10DA2000FDF780FD0390FFE743F67000C4F20200AB
:10DA3000006800F002010020B0EB510F0ED1FFE7AB
:10DA4000FDF770FD0399401A41F28931884204D3F1
:10DA5000FFE703208DF8170097E1E5E71EE0FDF7EB
:10DA600061FD0390FFE743F67000C4F20200006816
:10DA700000F002010020B0EB510F0ED0FFE7FDF7E0
:10DA800051FD0399401A41F28931884204D3FFE7DE
:10DA900003208DF8170078E1E5E7FFE79DF8070020
:10DAA000012809D1FFE743F64001C4F202010868EA
:10DAB00020F080500860FFE7FFE70498806950B1CC
:10DAC000FFE704988069012805D0FFE70498806982
:10DAD000022801D1FFE708E045F2F300C0F602009A
:10DAE00040F2CF110FF0AEFEFFE7049880690028E6
:10DAF00000F04781FFE743F60800C4F20200006827
:10DB000000F00C00082800F0F080FFE7049880691E
:10DB1000022840F0C780FFE70498C06930B1FFE7F2
:10DB20000498C069B0F5800F01D1FFE708E045F225
:10DB3000F300C0F602004FF4EC710FF083FEFFE734
:10DB40000498006A3F2801D8FFE708E045F2F30097
:10DB5000C0F6020040F2D9110FF074FEFFE70498FE
:10DB6000406A322807D3FFE70498406AB0F5D87FAF
:10DB700001D8FFE708E045F2F300C0F602004FF4D9
:10DB8000ED710FF05FFEFFE70498806A02280FD066
:10DB9000FFE70498806A04280AD0FFE70498806AA7
:10DBA000062805D0FFE70498806A082801D1FFE71E
:10DBB00008E045F2F300C0F6020040F2DB110FF07E
:10DBC00041FEFFE70498C06A022806D3FFE70498E5
:10DBD000C06A0F2801D8FFE708E045F2F300C0F65D
:10DBE00002004FF4EE710FF02DFEFFE76021C4F24A
:10DBF000472100200860FDF795FC0390FFE743F6FE
:10DC00000000C4F20200006800F000710020B0EBD8
:10DC1000516F0CD0FFE7FDF785FC0399401A0328EC
:10DC200004D3FFE703208DF81700AEE0E7E704997F
:10DC3000C869D1F820C04B6A8A6A40EA0C0040EA01
:10DC40008310D2034FF6FF739A43A2F5803210433C
:10DC5000C96A40EA016043F60401C4F202010860A7
:10DC60006021C4F2472101200860FDF75BFC0390AE
:10DC7000FFE743F60000C4F20200006800F0007104
:10DC80000020B0EB516F0CD1FFE7FDF74BFC03997F
:10DC9000401A032804D3FFE703208DF8170074E02F
:10DCA000E7E721E06021C4F2472100200860FDF78A
:10DCB00039FC0390FFE743F60000C4F2020000685D
:10DCC00000F000710020B0EB516F0CD0FFE7FDF7C2
:10DCD00029FC0399401A032804D3FFE703208DF899
:10DCE000170052E0E7E7FFE74AE00498806901285F
:10DCF00004D1FFE701208DF8170046E043F6040049
:10DD0000C4F202000068029004988069012831D0B2
:10DD1000FFE7029800F480000499C969884229D17C
:10DD2000FFE7029800F03F000499096A884221D178
:10DD3000FFE7029847F6C07108400499496AB0EBC2
:10DD4000811F17D1FFE7029800F440300499896AD7
:10DD5000C9034FF6FF729143A1F58031884209D182
:10DD6000FFE7029800F070600499C96AB0EB016F98
:10DD700004D0FFE701208DF8170006E0FFE7FFE77A
:10DD8000FFE700208DF81700FFE79DF8170006B0A9
:10DD900080BD000080B582B00090009820B9FFE7F8
:10DDA00001208DF807002EE00098006840F6000181
:10DDB000C5F20601884201D1FFE707E045F22E30A7
:10DDC000C0F60200A3210FF03DFDFFE70098407967
:10DDD00038B9FFE7009900200871009800F018F8A2
:10DDE000FFE700990220487100980168086840F038
:10DDF00004000860009901204871009900208860A3
:10DE00008DF80700FFE79DF8070002B080BD000015
:10DE100082B001900198006840F60001C5F2060149
:10DE2000884212D1FFE7FFE70020009043F634005C
:10DE3000C4F20200016841F040010160006800F096
:10DE4000400000900098FFE7FFE702B07047000035
:10DE500080B582B00190019808F042FC8DF8030073
:10DE60009DF8030003281BD0FFE7019808F038FC59
:10DE7000014640F24040C2F2000000EB41108069D0
:10DE800068B1FFE7019808F02BFC014640F24040E2
:10DE9000C2F2000000EB411080698047FFE7FFE716
:10DEA00002B080BD80B584B00290029820B9FFE72F
:10DEB00001208DF80F00D2E10298006843F20001C2
:10DEC000C4F20101884212D0FFE70298006843F6CD
:10DED0000001C4F20001884209D0FFE702980068FF
:10DEE00043F60041C4F20001884201D1FFE708E097
:10DEF00045F26630C0F602004FF4A1710FF0A2FCAB
:10DF0000FFE70298406830B1FFE702984068B0F53B
:10DF1000827F01D1FFE708E045F26630C0F60200DB
:10DF200040F243110FF08EFCFFE70298806860B169
:10DF3000FFE702988068B0F5806F06D0FFE702988F
:10DF40008068B0F5004F01D1FFE708E045F2663088
:10DF5000C0F602004FF4A2710FF074FCFFE70298C4
:10DF6000C068B0F5006F04D0FFE70298C06808B938
:10DF7000FFE708E045F26630C0F6020040F24511C6
:10DF80000FF060FCFFE702988069B0F5007F0AD0CF
:10DF9000FFE70298806930B1FFE702988069B0F529
:10DFA000802F01D1FFE708E045F26630C0F602009D
:10DFB0004FF4A3710FF046FCFFE70298C06918B355
:10DFC000FFE70298C06908281ED0FFE70298C069E1
:10DFD000102819D0FFE70298C069182814D0FFE76D
:10DFE0000298C06920280FD0FFE70298C06928284E
:10DFF0000AD0FFE70298C069302805D0FFE70298F1
:10E00000C069382801D1FFE708E045F26630C0F664
:10E01000020040F247110FF015FCFFE70298006A7A
:10E0200028B1FFE70298006A802801D1FFE708E0E5
:10E0300045F26630C0F602004FF4A4710FF002FC06
:10E04000FFE70298406A28B1FFE70298406A10286B
:10E0500001D1FFE708E045F26630C0F6020040F269
:10E0600049110FF0EFFBFFE70298406A002863D1E7
:10E07000FFE70298006928B1FFE7029800690228CB
:10E0800001D1FFE708E045F26630C0F602004FF428
:10E09000A6710FF0D7FBFFE70298406928B1FFE7B0
:10E0A00002984069012801D1FFE708E045F2663097
:10E0B000C0F6020040F24D110FF0C4FBFFE70298DA
:10E0C0004068B0F5827F32D1FFE70298C06918B38B
:10E0D000FFE70298C06908281ED0FFE70298C069D0
:10E0E000102819D0FFE70298C069182814D0FFE75C
:10E0F0000298C06920280FD0FFE70298C06928283D
:10E100000AD0FFE70298C069302805D0FFE70298DF
:10E11000C069382801D1FFE708E045F26630C0F653
:10E12000020040F251110FF08DFBFFE703E002996E
:10E130000020C861FFE736E00298C06918B3FFE726
:10E140000298C06908281ED0FFE70298C06910280D
:10E1500019D0FFE70298C069182814D0FFE7029889
:10E16000C06920280FD0FFE70298C06928280AD08C
:10E17000FFE70298C069302805D0FFE70298C06920
:10E18000382801D1FFE708E045F26630C0F602000A
:10E1900040F25B110FF056FBFFE702990020086187
:10E1A00002994861FFE7029900208862029890F87E
:10E1B000510040B9FFE70299002081F85000029811
:10E1C00000F052F8FFE70299022081F8510002980E
:10E1D0000168086820F040000860029A0192116806
:10E1E0005068D2F808C0D36800F482700CF4044C74
:10E1F000604403F400631844136903F002031844F5
:10E20000536903F001031844936903F4007318443D
:10E21000D36903F038031844136A03F080031843EA
:10E22000926A02F4005210430860029A508B00F088
:10E2300004001168526A02F010021044486002980B
:10E240000168C86920F40060C8610299002048652F
:10E25000029A012182F851108DF80F00FFE79DF816
:10E260000F0004B080BD000080B592B01190002076
:10E2700010900F900E900D900C901198006843F242
:10E280000001C4F20101884240F0B680FFE7FFE7D9
:10E2900000200B9043F64400C4F20200016841F4F0
:10E2A00080510160006800F480500B900B98FFE7EC
:10E2B000FFE700200A9043F63000C4F20200016834
:10E2C00041F002010160006800F002000A900A9823
:10E2D000FFE7FFE70020099043F63000C4F2020098
:10E2E000016841F001010160006800F0010009903F
:10E2F0000998FFE718200C90022001900D90012052
:10E3000002900E90032003900F900520049010902F
:10E3100040F20040C4F202000CA90591FCF70CFD8C
:10E32000DDF804C0029B039A049805994FF0800E13
:10E33000CDF830E0CDF834C00E930F92109000204D
:10E34000C4F20200FCF7F8FC41F62C00C2F2000017
:10E35000069046F24041C4F2020101604FF0C061F4
:10E36000416000218160C1604FF4806202614161BF
:10E370008161C1614FF4403202624162FBF7F2FFFA
:10E3800018B1FFE7F8F738FDFFE7FFE7119841F60E
:10E390002C01C2F20001C16411988863FFE741F6C5
:10E3A0008C00C2F20000009046F25841C4F2020113
:10E3B00001604FF0C0614160402181600021C16077
:10E3C0004FF48062026141618161C1614FF40032AA
:10E3D00002624162FBF7C6FF18B1FFE7F8F70CFDD8
:10E3E000FFE7FFE7119841F68C01C2F2000181645A
:10E3F00011988863FFE73EE01198006843F600013A
:10E40000C4F20001884235D1FFE7FFE70020089001
:10E4100043F64000C4F20200016841F4804101600B
:10E42000006800F4804008900898FFE7FFE70020AC
:10E43000079043F63000C4F20200016841F0020187
:10E440000160006800F0020007900798FFE74FF4B2
:10E4500060400C9002200D9001200E9003200F9040
:10E460000520109040F20040C4F202000CA9FCF715
:10E4700063FCFFE7FFE712B080BD000080B588B005
:10E4800006900591ADF81220039300208DF8070047
:10E4900006984068B0F5827F16D1FFE7069880683D
:10E4A00090B9FFE70699042081F851000698059A73
:10E4B000BDF812300399EC46CCF80010114600F07C
:10E4C00089FB8DF81F00EDE0FFE7069890F85000FB
:10E4D000012804D1FFE702208DF81F00E2E0069931
:10E4E000012081F85000FFE7FFE7FDF71BF80290DD
:10E4F000069890F85100012804D0FFE702208DF81B
:10E500000700C0E0059820B1FFE7BDF8120020B970
:10E51000FFE701208DF80700B5E00699042081F897
:10E5200051000699002048650599069A9163BDF847
:10E530001210069A9187BDF81210069AD187069993
:10E540000863069988860699C8860699086406991C
:10E55000486406988068B0F5004F0DD1FFE7069833
:10E560000168086820F040000860069801680868A3
:10E5700020F480400860FFE706980068006800F01B
:10E580004000402807D0FFE706980168086840F07F
:10E5900040000860FFE70698C06880BBFFE7FFE720
:10E5A0000698C08F50B3FFE7069800688068C007E0
:10E5B00078B1FFE706980068007B0699896B0870C0
:10E5C0000699886B013088630699C88F0138C8871F
:10E5D00013E0FCF7A7FF0299401A0399884204D37D
:10E5E000FFE70398013018B9FFE7039820B9FFE768
:10E5F00003208DF8070046E0FFE7D1E72FE0FFE7B3
:10E600000698C08F50B3FFE7069800688068C0077F
:10E6100078B1FFE706980068C0680699896B0880A2
:10E620000699886B023088630699C88F0138C887BD
:10E6300013E0FCF777FF0299401A0399884204D34C
:10E64000FFE70398013018B9FFE7039820B9FFE707
:10E6500003208DF8070016E0FFE7D1E7FFE70698F3
:10E660000399029A07F078FF20B1FFE7069920206E
:10E670004865FFE70698406D20B1FFE701208DF85F
:10E680000700FFE7FFE70699012081F85100FFE747
:10E690000699002081F85000FFE79DF807008DF8EB
:10E6A0001F00FFE79DF81F0008B080BD80B584B053
:10E6B00002900191ADF8022000208DF8010002982F
:10E6C000C06C08B1FFE708E045F26630C0F6020012
:10E6D00040F2CA610FF0B6F8FFE70298806810BBFD
:10E6E000FFE702984068B0F5827F1CD1FFE70299EE
:10E6F000042081F851000298806C08B1FFE708E01F
:10E7000045F26630C0F6020040F2D1610FF09AF88F
:10E71000FFE70298019ABDF80230114600F01CFC98
:10E720008DF80F00A8E0FFE7029890F8500001284C
:10E7300004D1FFE702208DF80F009DE0029901202F
:10E7400081F85000FFE7FFE7029890F85100012898
:10E7500004D0FFE702208DF8010082E0019820B18B
:10E76000FFE7BDF8020020B9FFE701208DF80100A6
:10E7700077E00299042081F8510002990020486551
:10E780000199029A9163BDF80210029A9187BDF82F
:10E790000210029AD187029908640299486402998A
:10E7A00088860299C88602988068B0F5004F0DD11E
:10E7B000FFE702980168086820F0400008600298AE
:10E7C0000168086820F480400860FFE70298C16C87
:10E7D00046F2FD30C0F6010008640298C16C46F2B2
:10E7E0002D40C0F60100C8630298C16C46F2C930E2
:10E7F000C0F60100C8640298C16C00200865029B45
:10E8000019689A6BD86C0C31DB8FFCF747F860B154
:10E81000FFE70299486D40F01000486501208DF82F
:10E820000100029981F851001BE00298006800681D
:10E8300000F04000402807D0FFE702980168086810
:10E8400040F040000860FFE702980168486840F027
:10E850002000486002980168486840F00100486064
:10E86000FFE7FFE70299002081F85000FFE79DF8DD
:10E8700001008DF80F00FFE79DF80F0004B080BD88
:10E8800080B582B00190019807F02AFF8DF803004F
:10E890009DF8030003281BD0FFE7019807F020FF35
:10E8A000014640F24040C2F2000000EB41104068D7
:10E8B00068B1FFE7019807F013FF014640F24040BE
:10E8C000C2F2000000EB411040688047FFE7FFE71D
:10E8D00002B080BD80B582B00190019807F000FFC2
:10E8E0008DF803009DF8030003281BD0FFE7019873
:10E8F00007F0F6FE014640F24040C2F2000000EB95
:10E900004110006968B1FFE7019807F0E9FE014690
:10E9100040F24040C2F2000000EB41100069804725
:10E92000FFE7FFE702B080BD80B588B00690059193
:10E93000ADF81220039300208DF807000698806838
:10E9400030B1FFE706988068B0F5004F01D1FFE7CE
:10E9500008E045F26630C0F6020040F20A310EF0DF
:10E9600071FFFFE7FFE7069890F85000012804D1F7
:10E97000FFE702208DF81F0028E10699012081F8A9
:10E980005000FFE7FFE7FCF7CDFD0290BDF8120055
:10E99000ADF80400069890F85100012804D0FFE774
:10E9A00002208DF8070002E1059820B1FFE7BDF8CD
:10E9B000120020B9FFE701208DF80700F7E0069963
:10E9C000032081F851000699002048650599069AB0
:10E9D0001163BDF81210069A9186BDF81210069ABE
:10E9E000D18606998863069988870699C88706990B
:10E9F00048640699086406988068B0F5004F0DD108
:10EA0000FFE706980168086820F040000860069853
:10EA10000168086840F480400860FFE706980068D5
:10EA2000006800F04000402807D0FFE70698016822
:10EA3000086840F040000860FFE70698C068B0F53D
:10EA4000006F47D1FFE70698406828B1FFE7BDF89F
:10EA5000040001280ED1FFE706980168006B0088CA
:10EA6000C8600699086B023008630699C88E0138A1
:10EA7000C886FFE7FFE70698C08E50B3FFE7069809
:10EA800000688068800700280ED5FFE706980168B7
:10EA9000006B0088C8600699086B0230086306990D
:10EAA000C88E0138C88613E0FCF73CFD0299401A75
:10EAB0000399884204D3FFE70398013018B9FFE7B0
:10EAC000039820B9FFE703208DF807006FE0FFE708
:10EAD000D1E746E00698406828B1FFE7BDF804009A
:10EAE00001280ED1FFE706980168006B00780873D3
:10EAF0000699086B013008630699C88E0138C886EC
:10EB0000FFE7FFE70698C08E50B3FFE7069800685E
:10EB10008068800700280ED5FFE706980168006B23
:10EB2000007808730699086B013008630699C88E4F
:10EB30000138C88613E0FCF7F5FC0299401A0399E6
:10EB4000884204D3FFE70398013018B9FFE7039820
:10EB500020B9FFE703208DF8070028E0FFE7D1E7A1
:10EB6000FFE706980399029A07F068FD20B1FFE7D6
:10EB7000069920204865FFE70698806870B9FFE78E
:10EB8000FFE70020009006980068C0680090069893
:10EB90000068806800900098FFE7FFE70698406DE6
:10EBA00020B1FFE701208DF80700FFE7FFE7069996
:10EBB000012081F85100FFE70699002081F85000FC
:10EBC000FFE79DF807008DF81F00FFE79DF81F0085
:10EBD00008B080BD80B58EB0DDF840C00C900B91C0
:10EBE0000A92ADF826300120059000208DF8130020
:10EBF0000C98806808B9FFE708E045F26630C0F677
:10EC0000020040F27E410EF01DFEFFE7FFE70C9888
:10EC100090F85000012804D1FFE702208DF837005A
:10EC200095E10C99012081F85000FFE7FFE7FCF720
:10EC300079FC06900C9890F851008DF81F000C9804
:10EC400040680890BDF82600ADF824009DF81F002C
:10EC5000012812D0FFE70898B0F5827F09D1FFE7BD
:10EC60000C98806828B9FFE79DF81F00042804D09D
:10EC7000FFE702208DF813005AE10B9838B1FFE747
:10EC80000A9820B1FFE7BDF8260020B9FFE7012070
:10EC90008DF813004CE10C9890F85100042805D031
:10ECA000FFE70C99052081F85100FFE70C9900203F
:10ECB00048650A990C9A9163BDF826100C9AD18781
:10ECC000BDF826100C9A91870B990C9A1163BDF828
:10ECD00026100C9AD186BDF826100C9A91860C99B4
:10ECE00008640C9948640C980068006800F04000C3
:10ECF000402807D0FFE70C980168086840F0400002
:10ED00000860FFE70C98C068B0F5006F76D1FFE7A8
:10ED10000C98406828B1FFE7BDF8240001280ED107
:10ED2000FFE70C980168006B0088C8600C99086BBD
:10ED3000023008630C99C88E0138C886FFE7FFE7E8
:10ED40000C98C18E0120029039B9FFE70C98C08F52
:10ED5000002818BF01200290FFE70298C007002892
:10ED60004BD0FFE70C98006880688007002818D512
:10ED7000FFE70C98C08EA0B1FFE70598012810D1DD
:10ED8000FFE70C980168006B0088C8600C99086B5D
:10ED9000023008630C99C88E0138C886002005909F
:10EDA000FFE70C9800688068C007A8B1FFE70C98DF
:10EDB000C08F88B1FFE70C980068C0680C99896B18
:10EDC00008800C99886B023088630C99C88F0138D1
:10EDD000C88701200590FFE7FCF7A4FB0699401ABD
:10EDE0001099884208D3FFE71098013020B1FFE75F
:10EDF00003208DF813009BE0A2E778E00C984068B0
:10EE000028B1FFE7BDF8240001280ED1FFE70C98D8
:10EE10000168006B007808730C99086B0130086377
:10EE20000C99C88E0138C886FFE7FFE70C98C18EA1
:10EE30000120019039B9FFE70C98C08F002818BF56
:10EE400001200190FFE70198C00700284ED0FFE79E
:10EE50000C98006880688007002818D5FFE70C9898
:10EE6000C08EA0B1FFE70598012810D1FFE70C98EC
:10EE70000168006B007808730C99086B0130086317
:10EE80000C99C88E0138C88600200590FFE70C98C1
:10EE900000688068C007A8B1FFE70C98C08F88B1F0
:10EEA000FFE70C980068C0680C99896B08700C9992
:10EEB000886B013088630C99C88F0138C88701209E
:10EEC0000590FFE7FCF72EFB0699401A109988423F
:10EED00004D3FFE71098013018B9FFE7109820B964
:10EEE000FFE703208DF8130022E09FE7FFE70C986F
:10EEF0001099069A07F0A2FB38B1FFE701208DF8C0
:10EF000013000C992020486512E00C98806870B9B5
:10EF1000FFE7FFE7002003900C980068C0680390AB
:10EF20000C980068806803900398FFE7FFE7FFE70D
:10EF30000C99012081F85100FFE70C99002081F81D
:10EF40005000FFE79DF813008DF83700FFE79DF8AC
:10EF500037000EB080BD000080B588B006900591E6
:10EF60000492ADF80E3000208DF806000698C06CB3
:10EF700008B1FFE708E045F26630C0F602004FF442
:10EF8000E8610EF05FFCFFE70698806C08B1FFE7D0
:10EF900008E045F26630C0F6020040F241710EF022
:10EFA00051FCFFE70698806808B9FFE708E045F2E2
:10EFB0006630C0F6020040F244710EF043FCFFE7F9
:10EFC000FFE7069890F85000012804D1FFE70220DF
:10EFD0008DF81F00EFE00699012081F85000FFE74F
:10EFE000FFE7069890F851008DF8070006984068F2
:10EFF00002909DF80700012812D0FFE70298B0F5B3
:10F00000827F09D1FFE70698806828B9FFE79DF85D
:10F010000700042804D0FFE702208DF80600BFE0B7
:10F02000059838B1FFE7049820B1FFE7BDF80E005E
:10F0300020B9FFE701208DF80600B1E0069890F8AE
:10F040005100042805D0FFE70699052081F85100FA
:10F05000FFE70699002048650599069A1163BDF8F7
:10F060000E10069A9186BDF80E10069AD186049964
:10F07000069A9163BDF80E10069A9187BDF80E109E
:10F08000069AD1870699086406994864069890F80C
:10F09000510004280FD1FFE70698C16C46F2FD30FD
:10F0A000C0F6010008640698C16C46F22D40C0F617
:10F0B0000100C8630EE00698C16C46F21540C0F628
:10F0C000010008640698C16C46F2D140C0F6010008
:10F0D000C863FFE70698C16C46F2C930C0F601006C
:10F0E000C8640698C16C00200865069B19689A6B75
:10F0F000D86C0C31DB8FFBF7D1FB60B1FFE70699D1
:10F10000486D40F01000486501208DF80600069912
:10F1100081F8510044E006980168486840F0010019
:10F1200048600698816C002008640699896CC86361
:10F130000699896CC8640699896C0865069B1A68EB
:10F14000196B986C0C32DB8EFBF7A8FB60B1FFE704
:10F150000699486D40F01000486501208DF80600C2
:10F16000069981F851001BE006980068006800F0DD
:10F170004000402807D0FFE706980168086840F083
:10F1800040000860FFE706980168486840F02000EA
:10F19000486006980168486840F002004860FFE750
:10F1A000FFE70699002081F85000FFE79DF8060070
:10F1B0008DF81F00FFE79DF81F0008B080BD00001C
:10F1C00080B582B00190019807F08AFA8DF80300AB
:10F1D0009DF8030003281BD0FFE7019807F080FA91
:10F1E000014640F24040C2F2000000EB411080684E
:10F1F00068B1FFE7019807F073FA014640F240401A
:10F20000C2F2000000EB411080688047FFE7FFE793
:10F2100002B080BD80B582B00190019807F060FA1D
:10F220008DF803009DF8030003281BD0FFE7019829
:10F2300007F056FA014640F24040C2F2000000EBEF
:10F240004110406968B1FFE7019807F049FA0146AB
:10F2500040F24040C2F2000000EB4110406980479C
:10F26000FFE7FFE702B080BD80B582B00190019852
:10F2700007F0E4FF02B080BD81B0009001B070479C
:10F2800081B0009001B0704780B584B002900191C8
:10F2900000200090029800680021C4F20101884219
:10F2A00009D0FFE70298006840F20041C4F2010172
:10F2B000884201D1FFE708E045F2D630C0F60200EF
:10F2C00040F2B4710EF0BEFAFFE701980068B0F5A5
:10F2D000006F04D0FFE70198006808B9FFE708E075
:10F2E00045F2D630C0F6020040F2B5710EF0AAFA2F
:10F2F000FFE701984068B0F5806F04D0FFE7019800
:10F30000406808B9FFE708E045F2D630C0F60200D1
:10F3100040F2B6710EF096FAFFE70198806890B15E
:10F32000FFE701988068B0F5807F0CD0FFE7019877
:10F330008068B0F5007F06D0FFE701988068B0F5DF
:10F34000407F01D1FFE708E045F2D630C0F6020069
:10F3500040F2B7710EF076FAFFE70198C068FF2817
:10F3600001D8FFE708E045F2D630C0F602004FF4BE
:10F37000F7610EF067FAFFE701980069B0F5805F6A
:10F3800004D0FFE70198006908B9FFE708E045F2FB
:10F39000D630C0F6020040F2B9710EF053FAFFE722
:10F3A0000198406930B1FFE701984069B0F5005F0E
:10F3B00001D1FFE708E045F2D630C0F6020040F286
:10F3C000BA710EF03FFAFFE70198C069B0F5804FBF
:10F3D00004D0FFE70198C06908B9FFE708E045F2EB
:10F3E000D630C0F6020040F2BB710EF02BFAFFE7F8
:10F3F000FFE7029890F83C00012804D1FFE70220C3
:10F400008DF80F0044E00299012081F83C00FFE7ED
:10F41000FFE7009820F0FF000199C96808430090B9
:10F42000009820F440700199896808430090009882
:10F4300020F480600199496808430090009820F406
:10F4400000600199096808430090009820F48050FA
:10F450000199096908430090009820F4005001992F
:10F46000496908430090009820F480400199C969D7
:10F47000084300900098029909684864FFE70299E0
:10F48000002081F83C00FFE700208DF80F00FFE727
:10F490009DF80F0004B080BD80B586B00490039144
:10F4A000049800680021C4F2010188423CD0FFE7C3
:10F4B00004980068B0F1804F36D0FFE704980068E8
:10F4C00040F20041C4F2000188422DD0FFE70498C9
:10F4D000006840F60001C4F20001884224D0FFE732
:10F4E0000498006840F60041C4F2000188421BD035
:10F4F000FFE70498006841F20001C4F2000188426D
:10F5000012D0FFE70498006841F20041C4F2000104
:10F51000884209D0FFE70498006840F20041C4F235
:10F520000101884201D1FFE708E045F2D630C0F67C
:10F53000020040F277710EF085F9FFE7039800684A
:10F5400018B3FFE70398006810281ED0FFE7039860
:10F550000068202819D0FFE703980068302814D0ED
:10F56000FFE70398006840280FD0FFE70398006882
:10F5700050280AD0FFE703980068602805D0FFE70D
:10F5800003980068702801D1FFE708E045F2D63003
:10F59000C0F602004FF4EF610EF054F9FFE7039854
:10F5A0004068802804D0FFE70398406808B9FFE767
:10F5B00008E045F2D630C0F6020040F279710EF054
:10F5C00041F9FFE7FFE7049890F83C00012804D1D7
:10F5D000FFE702208DF817007EE00499012081F8F2
:10F5E0003C00FFE7FFE70499022081F83D00049802
:10F5F0000068406802900498006880680190029852
:10F6000020F070000290039801680298084302906D
:10F610000298049909684860049800680021C4F2BF
:10F62000010188423CD0FFE704980068B0F1804FA8
:10F6300036D0FFE70498006840F20041C4F20001B0
:10F6400088422DD0FFE70498006840F60001C4F21C
:10F650000001884224D0FFE70498006840F600418A
:10F66000C4F2000188421BD0FFE70498006840F212
:10F670000041C4F20101884212D0FFE704980068FB
:10F6800044F20001C4F20101884209D0FFE7049866
:10F69000006841F60001C4F2000188420ED1FFE784
:10F6A000019820F080000190039841680198084378
:10F6B00001900198049909688860FFE70499012086
:10F6C00081F83D00FFE70499002081F83C00FFE746
:10F6D00000208DF81700FFE79DF8170006B080BDE9
:10F6E00080B582B00090009820B9FFE701208DF826
:10F6F000070012E1009800680021C4F2010188426D
:10F7000072D0FFE700980068B0F1804F6CD0FFE73F
:10F710000098006840F20041C4F20001884263D0C2
:10F72000FFE70098006840F60001C4F2000188423B
:10F730005AD0FFE70098006840F60041C4F200018B
:10F74000884251D0FFE70098006841F20001C4F2FE
:10F750000001884248D0FFE70098006841F200416C
:10F76000C4F2000188423FD0FFE70098006840F2F1
:10F770000041C4F20101884236D0FFE700980068DA
:10F7800044F20001C4F2010188422DD0FFE7009845
:10F79000006844F20041C4F20101884224D0FFE72E
:10F7A0000098006844F60001C4F2010188421BD0B1
:10F7B000FFE70098006841F60001C4F200018842AA
:10F7C00012D0FFE70098006841F60041C4F2000142
:10F7D000884209D0FFE70098006842F20001C4F2B5
:10F7E0000001884201D1FFE708E045F29E30C0F6F3
:10F7F000020040F213110EF025F8FFE70098806830
:10F80000A0B1FFE70098806810280FD0FFE70098AC
:10F81000806820280AD0FFE700988068402805D03B
:10F82000FFE700988068602801D1FFE708E045F213
:10F830009E30C0F602004FF48A710EF003F8FFE725
:10F840000098006960B1FFE700980069B0F5807F1B
:10F8500006D0FFE700980069B0F5007F01D1FFE70F
:10F8600008E045F29E30C0F6020040F215110DF09E
:10F87000E9FFFFE70098806928B1FFE700988069F9
:10F88000802801D1FFE708E045F29E30C0F6020073
:10F890004FF48B710DF0D6FFFFE7009890F83D0014
:10F8A00040B9FFE70099002081F83C00009800F083
:10F8B00039F8FFE70099022081F83D00009951F8DE
:10F8C000040B07F06FFD0099012081F84600FFE767
:10F8D0000099012081F83E00009981F83F000099CD
:10F8E00081F84000009981F84100FFE7FFE70099A7
:10F8F000012081F84200009981F84300009981F8C5
:10F900004400009981F84500FFE70099012081F843
:10F910003D0000208DF80700FFE79DF8070002B0CA
:10F9200080BD000080B58AB0099009980068002168
:10F93000C4F2010188421BD1FFE7FFE700200890D5
:10F9400043F64400C4F20200016841F00101016085
:10F95000006800F0010008900898FFE71820019067
:10F9600005210022FCF7FAF90198FCF7DFF9B0E075
:10F970000998006840F20041C4F20001884212D1A7
:10F98000FFE7FFE70020079043F64000C4F20200C3
:10F99000016841F002010160006800F00200079078
:10F9A0000798FFE794E00998006840F60001C4F268
:10F9B0000001884212D1FFE7FFE70020069043F6DE
:10F9C0004000C4F20200016841F0040101600068D7
:10F9D00000F0040006900698FFE778E009980068B8
:10F9E00040F60041C4F20001884212D1FFE7FFE770
:10F9F0000020059043F64000C4F20200016841F087
:10FA000008010160006800F0080005900598FFE714
:10FA10005CE00998006841F20041C4F200018842AC
:10FA20001BD1FFE7FFE70020049043F64000C4F23B
:10FA30000200016841F020010160006800F0200030
:10FA400004900498FFE73720009005210022FCF77E
:10FA500085F90098FCF76AF937E00998006840F2E8
:10FA60000041C4F20101884212D1FFE7FFE7002004
:10FA7000039043F64400C4F20200016841F0020121
:10FA80000160006800F0020003900398FFE71BE0AC
:10FA90000998006844F20041C4F20101884212D181
:10FAA000FFE7FFE70020029043F64400C4F20200A3
:10FAB000016841F400310160006800F400300290F8
:10FAC0000298FFE7FFE7FFE7FFE7FFE7FFE7FFE752
:10FAD000FFE70AB080BD000080B584B002900298B4
:10FAE00000680021C4F20101884272D0FFE7029849
:10FAF0000068B0F1804F6CD0FFE70298006840F2D8
:10FB00000041C4F20001884263D0FFE70298006818
:10FB100040F60001C4F2000188425AD0FFE7029883
:10FB2000006840F60041C4F20001884251D0FFE76E
:10FB30000298006841F20001C4F20001884248D0F6
:10FB4000FFE70298006841F20041C4F200018842D8
:10FB50003FD0FFE70298006840F20041C4F2010183
:10FB6000884236D0FFE70298006844F20001C4F2F0
:10FB7000010188422DD0FFE70298006844F200415D
:10FB8000C4F20101884224D0FFE70298006844F6DD
:10FB90000001C4F2010188421BD0FFE7029800680F
:10FBA00041F60001C4F20001884212D0FFE702983A
:10FBB000006841F60041C4F20001884209D0FFE725
:10FBC0000298006842F20001C4F20001884201D1AB
:10FBD000FFE708E045F29E30C0F6020040F2CF1188
:10FBE0000DF030FEFFE7029890F83D00012804D0A8
:10FBF000FFE701208DF80F006AE00299022081F8EA
:10FC00003D0002980168C86840F00100C860029891
:10FC100000680021C4F2010188423CD0FFE702984D
:10FC20000068B0F1804F36D0FFE70298006840F2DC
:10FC30000041C4F2000188422DD0FFE7029800681D
:10FC400040F60001C4F20001884224D0FFE7029888
:10FC5000006840F60041C4F2000188421BD0FFE773
:10FC60000298006840F20041C4F20101884212D0BB
:10FC7000FFE70298006844F20001C4F201018842E3
:10FC800009D0FFE70298006841F60001C4F20001C4
:10FC9000884212D1FFE702980068806800F00700F0
:10FCA00001900198062807D0FFE7029801680868CC
:10FCB00040F001000860FFE706E00298016808686C
:10FCC00040F001000860FFE700208DF80F00FFE71B
:10FCD0009DF80F0004B080BD80B586B004900391FC
:10FCE000FFE7049890F83C00012805D1FFE70220C7
:10FCF0008DF8170000F069BC0499012081F83C00E0
:10FD0000FFE7FFE70499022081F83D0003980068AF
:10FD1000B0F5805F2DD0FFE703980068B0F5005F75
:10FD200027D0FFE70398006818B3FFE7039800683F
:10FD300010281ED0FFE703980068202819D0FFE79D
:10FD400003980068302814D0FFE703980068402823
:10FD50000FD0FFE70398006850280AD0FFE7039808
:10FD60000068602805D0FFE703980068702801D17B
:10FD7000FFE708E045F29E30C0F6020041F2224162
:10FD80000DF060FDFFE7049800688068029002981B
:10FD900020F077000290029820F47F4002900298B1
:10FDA000049909688860039800680190002800F0B1
:10FDB000A883FFE70198102800F0A383FFE70198CC
:10FDC000202800F09E83FFE70198302800F09983F7
:10FDD000FFE70198402800F00883FFE701985028CA
:10FDE00000F0EB81FFE70198602800F07282FFE7E6
:10FDF0000198702800F09180FFE70198B0F5805FCE
:10FE000006D0FFE70198B0F5005F00F03A81CDE33E
:10FE1000049800680021C4F20101884272D0FFE713
:10FE200004980068B0F1804F6CD0FFE70498006838
:10FE300040F20041C4F20001884263D0FFE7049819
:10FE4000006840F60001C4F2000188425AD0FFE782
:10FE50000498006840F60041C4F20001884251D085
:10FE6000FFE70498006841F20001C4F200018842F3
:10FE700048D0FFE70498006841F20041C4F2000155
:10FE800088423FD0FFE70498006840F20041C4F286
:10FE90000101884236D0FFE70498006844F200016F
:10FEA000C4F2010188422DD0FFE70498006844F2B3
:10FEB0000041C4F20101884224D0FFE704980068A1
:10FEC00044F60001C4F2010188421BD0FFE7049808
:10FED000006841F60001C4F20001884212D0FFE739
:10FEE0000498006841F60041C4F20001884209D03C
:10FEF000FFE70498006842F20001C4F20001884262
:10FF000001D1FFE708E045F29E30C0F6020041F261
:10FF10002E410DF097FCFFE749E3049800680021AB
:10FF2000C4F2010188423CD0FFE704980068B0F1B8
:10FF3000804F36D0FFE70498006840F20041C4F2D9
:10FF4000000188422DD0FFE70498006840F60001C8
:10FF5000C4F20001884224D0FFE70498006840F60C
:10FF60000041C4F2000188421BD0FFE704980068FA
:10FF700040F20041C4F20101884212D0FFE7049828
:10FF8000006844F20001C4F20101884209D0FFE791
:10FF90000498006841F60001C4F20001884201D1D2
:10FFA000FFE708E045F29E30C0F6020041F235411D
:10FFB0000DF048FCFFE70398806890B1FFE70398D5
:10FFC0008068B0F5805F0CD0FFE703988068B0F5DB
:10FFD000005F06D0FFE703988068B0F5405F01D16D
:10FFE000FFE708E045F29E30C0F6020041F23841DA
:10FFF0000DF028FCFFE703984068B0F5004F12D0E1
:020000040801F1
:10000000FFE70398406870B1FFE70398406850B17C
:10001000FFE703984068022805D0FFE7039840688F
:100020000A2801D1FFE708E045F29E30C0F6020041
:1000300041F239410DF006FCFFE70398C0680F2834
:1000400001D8FFE708E045F29E30C0F6020041F219
:100050003A410DF0F7FBFFE704980068039B5A68EC
:100060009968DB6807F00CFB0498006880680290D0
:10007000029840F07700029002980499096888601D
:1000800095E2049800680021C4F2010188422AD058
:10009000FFE704980068B0F1804F24D0FFE7049890
:1000A000006840F20041C4F2000188421BD0FFE723
:1000B0000498006840F60001C4F20001884212D0A2
:1000C000FFE70498006840F60041C4F2000188424E
:1000D00009D0FFE70498006840F20041C4F2010132
:1000E000884201D1FFE708E045F29E30C0F60200E9
:1000F00041F24D410DF0A6FBFFE70398806890B1F7
:10010000FFE703988068B0F5805F0CD0FFE70398A5
:100110008068B0F5005F06D0FFE703988068B0F50F
:10012000405F01D1FFE708E045F29E30C0F60200D3
:1001300041F250410DF086FBFFE703984068B0F5AF
:10014000004F12D0FFE70398406870B1FFE70398B3
:10015000406850B1FFE703984068022805D0FFE7E8
:10016000039840680A2801D1FFE708E045F29E3075
:10017000C0F6020041F251410DF064FBFFE7039825
:10018000C0680F2801D8FFE708E045F29E30C0F6AE
:10019000020041F252410DF055FBFFE70498006860
:1001A000039B5A689968DB6807F06AFA049801684B
:1001B000886840F480408860F9E104980068002174
:1001C000C4F2010188423CD0FFE704980068B0F116
:1001D000804F36D0FFE70498006840F20041C4F237
:1001E000000188422DD0FFE70498006840F6000126
:1001F000C4F20001884224D0FFE70498006840F66A
:100200000041C4F2000188421BD0FFE70498006857
:1002100040F20041C4F20101884212D0FFE7049885
:10022000006844F20001C4F20101884209D0FFE7EE
:100230000498006841F60001C4F20001884201D12F
:10024000FFE708E045F29E30C0F6020041F261414E
:100250000DF0F8FAFFE703984068B0F5004F12D0B0
:10026000FFE70398406870B1FFE70398406850B11A
:10027000FFE703984068022805D0FFE7039840682D
:100280000A2801D1FFE708E045F29E30C0F60200DF
:1002900041F264410DF0D6FAFFE70398C0680F28D9
:1002A00001D8FFE708E045F29E30C0F6020041F2B7
:1002B00065410DF0C7FAFFE704980068039A51689A
:1002C000D26807F093FC04980068502107F0F2F917
:1002D0006DE1049800680021C4F2010188423CD01D
:1002E000FFE704980068B0F1804F36D0FFE704982C
:1002F000006840F20041C4F2000188422DD0FFE7BF
:100300000498006840F60001C4F20001884224D03D
:10031000FFE70498006840F60041C4F200018842FB
:100320001BD0FFE70498006840F20041C4F20101CD
:10033000884212D0FFE70498006844F20001C4F23A
:100340000101884209D0FFE70498006841F60001E6
:10035000C4F20001884201D1FFE708E045F29E3077
:10036000C0F6020041F271410DF06CFAFFE703980C
:100370004068B0F5004F12D0FFE70398406870B1B5
:10038000FFE70398406850B1FFE7039840680228F0
:1003900005D0FFE7039840680A2801D1FFE708E08D
:1003A00045F29E30C0F6020041F274410DF04AFA67
:1003B000FFE70398C0680F2801D8FFE708E045F27F
:1003C0009E30C0F6020041F275410DF03BFAFFE7A6
:1003D00004980068039A5168D26807F02FFC0498CB
:1003E0000068602107F066F9E1E0049800680021E8
:1003F000C4F2010188423CD0FFE704980068B0F1E4
:10040000804F36D0FFE70498006840F20041C4F204
:10041000000188422DD0FFE70498006840F60001F3
:10042000C4F20001884224D0FFE70498006840F637
:100430000041C4F2000188421BD0FFE70498006825
:1004400040F20041C4F20101884212D0FFE7049853
:10045000006844F20001C4F20101884209D0FFE7BC
:100460000498006841F60001C4F20001884201D1FD
:10047000FFE708E045F29E30C0F6020041F28141FC
:100480000DF0E0F9FFE703984068B0F5004F12D097
:10049000FFE70398406870B1FFE70398406850B1E8
:1004A000FFE703984068022805D0FFE703984068FB
:1004B0000A2801D1FFE708E045F29E30C0F60200AD
:1004C00041F284410DF0BEF9FFE70398C0680F28A0
:1004D00001D8FFE708E045F29E30C0F6020041F285
:1004E00085410DF0AFF9FFE704980068039A516861
:1004F000D26807F07BFB04980068402107F0DAF827
:1005000055E0049800680021C4F2010188423CD003
:10051000FFE704980068B0F1804F36D0FFE70498F9
:10052000006840F20041C4F2000188422DD0FFE78C
:100530000498006840F60001C4F20001884224D00B
:10054000FFE70498006840F60041C4F200018842C9
:100550001BD0FFE70498006840F20041C4F201019B
:10056000884212D0FFE70498006844F20001C4F208
:100570000101884209D0FFE70498006841F60001B4
:10058000C4F20001884201D1FFE708E045F29E3045
:10059000C0F6020041F294410DF054F9FFE70498CF
:1005A00000680399096807F085F800E0FFE70499FF
:1005B000012081F83D00FFE70499002081F83C000C
:1005C000FFE700208DF81700FFE79DF8170006B041
:1005D00080BD000081B0009001B0704780B582B04E
:1005E000019001980068006900F002010020B0EB62
:1005F000510F28D0FFE701980068C06800F00201A1
:100600000020B0EB510F1DD0FFE7019801686FF09B
:10061000020008610199012008770198006880694B
:10062000800720B1FFE70198FFF7D4FF06E00198AB
:1006300000F04CFA019800F0A3FDFFE701990020BB
:100640000877FFE7FFE701980068006900F0040100
:100650000020B0EB910F29D0FFE701980068C06837
:1006600000F004010020B0EB910F1ED0FFE70198CD
:1006700001686FF004000861019902200877019871
:100680000068806910F4407F04D0FFE70198FFF70D
:10069000A1FF06E0019800F019FA019800F070FD42
:1006A000FFE7019900200877FFE7FFE7019800685E
:1006B000006900F008010020B0EBD10F28D0FFE75F
:1006C00001980068C06800F008010020B0EBD10F6D
:1006D0001DD0FFE7019801686FF0080008610199DB
:1006E0000420087701980068C069800720B1FFE7FF
:1006F0000198FFF76FFF06E0019800F0E7F9019815
:1007000000F03EFDFFE7019900200877FFE7FFE7D3
:1007100001980068006900F010010020B0EB111F83
:1007200029D0FFE701980068C06800F010010020A0
:10073000B0EB111F1ED0FFE7019801686FF01000A9
:10074000086101990820087701980068C06910F4D1
:10075000407F04D0FFE70198FFF73CFF06E00198D7
:1007600000F0B4F9019800F00BFDFFE701990020BB
:100770000877FFE7FFE7019800680069C00780B1CC
:10078000FFE701980068C068C00748B1FFE701981B
:1007900001686FF001000861019801F057F8FFE768
:1007A000FFE7019800680069C1B20020B0EBD11FDB
:1007B00013D0FFE701980068C068C1B20020B0EB19
:1007C000D11F09D0FFE7019801686FF08000086130
:1007D0000198FEF751FDFFE7FFE701980068006907
:1007E00000F040010020B0EB911F14D0FFE701980A
:1007F0000068C06800F040010020B0EB911F09D0F4
:10080000FFE7019801686FF040000861019801F06E
:1008100033F8FFE7FFE701980068006900F0200166
:100820000020B0EB511F14D0FFE701980068C068AA
:1008300000F020010020B0EB511F09D0FFE7019824
:1008400001686FF0200008610198FEF719FDFFE7CD
:10085000FFE702B080BD000080B592B0119000208B
:1008600010900F900E900D900C9011980068002140
:10087000C4F20101884222D1FFE7FFE700200B907C
:1008800043F63000C4F20200016841F0100101603B
:10089000006800F010000B900B98FFE74FF4D44075
:1008A0000C9002210D9101200E900F91109041F2B9
:1008B0000000C4F202000CA9FAF73EFA03E1119815
:1008C000006840F20041C4F20001884222D1FFE7F3
:1008D000FFE700200A9043F63000C4F202000168EE
:1008E00041F004010160006800F004000A900A98D9
:1008F000FFE74FF480700C9002200D9001210E91C3
:100900000F90109040F60000C4F202000CA9FAF714
:1009100013FAD7E01198006840F60001C4F2000114
:10092000884223D1FFE7FFE70020099043F630001B
:10093000C4F20200016841F008010160006800F0A3
:10094000080009900998FFE74FF480400C900220BE
:100950000D9001210E9103210F91109040F600405F
:10096000C4F202000CA9FAF7E7F9AAE011980068AE
:1009700040F60041C4F20001884222D1FFE7FFE7C0
:100980000020089043F63000C4F20200016841F0F4
:1009900080010160006800F0800008900898FFE77F
:1009A0004FF4E0500C9002200D9001210E910F9019
:1009B000109041F60040C4F202000CA9FAF7BCF90D
:1009C0007EE01198006840F20041C4F201018842C3
:1009D0004AD1FFE7FFE70020079043F63000C4F25A
:1009E0000200016841F480710160006800F48070C9
:1009F00007900798FFE7FFE70020069043F63000D6
:100A0000C4F20200016841F004010160006800F0D6
:100A1000040006900698FFE7402000900C9002200A
:100A200002900D90012101910E910F9003200390EF
:100A3000109042F20000C4F202000CA90491FAF7EF
:100A40007BF9DDF800C0019B029A03980499CDF868
:100A500030C00D920E930F92109040F60000C4F239
:100A60000200FAF769F92AE01198006844F200419F
:100A7000C4F20101884221D1FFE7FFE70020059081
:100A800043F63000C4F20200016841F02001016029
:100A9000006800F0200005900598FFE740200C90CA
:100AA00002200D900E900F900320109041F2004014
:100AB000C4F202000CA9FAF73FF9FFE7FFE7FFE7EE
:100AC000FFE7FFE7FFE712B080BD000081B00090B4
:100AD00001B0704780B586B00490039102920298ED
:100AE00080B1FFE7029804280CD0FFE7029808289D
:100AF00008D0FFE702980C2804D0FFE702983C28B2
:100B000001D1FFE708E045F29E30C0F6020041F255
:100B100017010CF097FEFFE703980068602805D0E6
:100B2000FFE703980068702801D1FFE708E045F26D
:100B30009E30C0F6020041F218010CF083FEFFE780
:100B40000398806828B1FFE703988068022801D1E4
:100B5000FFE708E045F29E30C0F6020041F21901BD
:100B60000CF070FEFFE70398006928B1FFE70398D7
:100B70000069042801D1FFE708E045F29E30C0F685
:100B8000020041F21A010CF05DFEFFE7FFE7049856
:100B900090F83C00012804D1FFE702208DF81700EF
:100BA000C3E10499012081F83C00FFE7FFE70298C8
:100BB00001900C2800F2AE810199DFE811F00D00E0
:100BC000AB01AB01AB019800AB01AB01AB01000184
:100BD000AB01AB01AB015501049800680021C4F2E0
:100BE0000101884260D0FFE704980068B0F1804FAF
:100BF0005AD0FFE70498006840F20041C4F20001B7
:100C0000884251D0FFE70498006840F60001C4F222
:100C10000001884248D0FFE70498006840F6004190
:100C2000C4F2000188423FD0FFE70498006840F218
:100C30000041C4F20101884236D0FFE70498006801
:100C400044F20001C4F2010188422DD0FFE704986C
:100C5000006844F20041C4F20101884224D0FFE759
:100C60000498006844F60001C4F2010188421BD0D8
:100C7000FFE70498006841F60001C4F200018842D1
:100C800012D0FFE70498006841F60041C4F2000169
:100C9000884209D0FFE70498006842F20001C4F2DC
:100CA0000001884201D1FFE708E045F29E30C0F61E
:100CB000020041F224010CF0C5FDFFE70498006832
:100CC000039906F00DFD04980168886940F008005A
:100CD000886104980168886920F00400886103989D
:100CE00002690498016888691043886113E10498D7
:100CF00000680021C4F2010188423CD0FFE704985B
:100D00000068B0F1804F36D0FFE70498006840F2E9
:100D10000041C4F2000188422DD0FFE7049800682A
:100D200040F60001C4F20001884224D0FFE7049895
:100D3000006840F60041C4F2000188421BD0FFE782
:100D40000498006840F20041C4F20101884212D0C8
:100D5000FFE70498006844F20001C4F201018842F0
:100D600009D0FFE70498006841F60001C4F20001D1
:100D7000884201D1FFE708E045F29E30C0F602004C
:100D800041F235010CF05EFDFFE70498006803991D
:100D900006F058FD04980168886940F40060886195
:100DA00004980168886920F480608861039802696A
:100DB00004980168886940EA02208861ABE00498E1
:100DC00000680021C4F2010188422AD0FFE704989C
:100DD0000068B0F1804F24D0FFE70498006840F22B
:100DE0000041C4F2000188421BD0FFE7049800686C
:100DF00040F60001C4F20001884212D0FFE70498D7
:100E0000006840F60041C4F20001884209D0FFE7C3
:100E10000498006840F20041C4F20101884201D107
:100E2000FFE708E045F29E30C0F6020041F24601BD
:100E30000CF008FDFFE704980068039906F0B8FD80
:100E400004980168C86940F00800C8610498016806
:100E5000C86920F00400C861039802690498016819
:100E6000C8691043C86156E0049800680021C4F2C4
:100E7000010188422AD0FFE704980068B0F1804F52
:100E800024D0FFE70498006840F20041C4F200015A
:100E900088421BD0FFE70498006840F60001C4F2C6
:100EA0000001884212D0FFE70498006840F6004134
:100EB000C4F20001884209D0FFE70498006840F2BC
:100EC0000041C4F20101884201D1FFE708E045F288
:100ED0009E30C0F6020041F257010CF0B3FCFFE770
:100EE00004980068039906F019FE04980168C8691F
:100EF00040F40060C86104980168C86920F480600B
:100F0000C8610398026904980168C86940EA022030
:100F1000C86100E0FFE7FFE70499002081F83C008A
:100F2000FFE700208DF81700FFE79DF8170006B0D7
:100F300080BD000080B582B00090009820B9FFE726
:100F400001208DF8070012E1009800680021C4F22A
:100F50000101884272D0FFE700980068B0F1804F2D
:100F60006CD0FFE70098006840F20041C4F2000135
:100F7000884263D0FFE70098006840F60001C4F2A1
:100F8000000188425AD0FFE70098006840F600410F
:100F9000C4F20001884251D0FFE70098006841F296
:100FA0000001C4F20001884248D0FFE700980068C1
:100FB00041F20041C4F2000188423FD0FFE70098AF
:100FC000006840F20041C4F20101884236D0FFE7D8
:100FD0000098006844F20001C4F2010188422DD05B
:100FE000FFE70098006844F20041C4F20101884222
:100FF00024D0FFE70098006844F60001C4F2010124
:1010000088421BD0FFE70098006841F60001C4F257
:101010000001884212D0FFE70098006841F60041C5
:10102000C4F20001884209D0FFE70098006842F24C
:101030000001C4F20001884201D1FFE708E045F257
:101040009E30C0F6020040F20E510CF0FBFBFFE7B1
:1010500000988068A0B1FFE70098806810280FD042
:10106000FFE70098806820280AD0FFE70098806892
:10107000402805D0FFE700988068602801D1FFE78D
:1010800008E045F29E30C0F6020040F20F510CF02D
:10109000D9FBFFE70098006960B1FFE7009800699D
:1010A000B0F5807F06D0FFE700980069B0F5007FBB
:1010B00001D1FFE708E045F29E30C0F602004FF490
:1010C000A2610CF0BFFBFFE70098806928B1FFE741
:1010D00000988069802801D1FFE708E045F29E3042
:1010E000C0F6020040F211510CF0ACFBFFE7009893
:1010F00090F83D0040B9FFE70099002081F83C00DE
:10110000009800F039F8FFE70099022081F83D00CF
:10111000009951F8040B06F045F90099012081F877
:101120004600FFE70099012081F83E00009981F810
:101130003F00009981F84000009981F84100FFE7E5
:10114000FFE70099012081F84200009981F84300EF
:10115000009981F84400009981F84500FFE7009963
:10116000012081F83D0000208DF80700FFE79DF881
:10117000070002B080BD000081B0009001B0704750
:1011800081B0009001B0704780B58CB00A90099191
:101190000A9800680021C4F20101884214D1FFE7D7
:1011A0000998002800F0E780FFE70998042800F07C
:1011B000E280FFE70998082800F0DD80FFE7099842
:1011C0000C2800F0D880FFE70A980068B0F1804F43
:1011D00014D1FFE70998002800F0CD80FFE70998B7
:1011E000042800F0C880FFE70998082800F0C380B1
:1011F000FFE709980C2800F0BE80FFE70A98006816
:1012000040F20041C4F20001884214D1FFE709987E
:10121000002800F0B080FFE70998042800F0AB80B8
:10122000FFE70998082800F0A680FFE709980C2836
:1012300000F0A180FFE70A98006840F60001C4F2C0
:101240000001884214D1FFE70998002800F093803C
:10125000FFE70998042800F08E80FFE70998082826
:1012600000F08980FFE709980C2800F08480FFE7F0
:101270000A98006840F60041C4F20001884210D18B
:10128000FFE70998002876D0FFE70998042872D074
:10129000FFE7099808286ED0FFE709980C286AD064
:1012A000FFE70A98006840F20041C4F20101884259
:1012B00010D1FFE7099800285DD0FFE709980428BE
:1012C00059D0FFE70998082855D0FFE709980C285E
:1012D00051D0FFE70A98006844F20001C4F201010E
:1012E000884208D1FFE70998002844D0FFE7099811
:1012F000042840D0FFE70A98006844F20041C4F295
:101300000101884203D1FFE70998A0B3FFE70A98DB
:10131000006844F60001C4F20101884203D1FFE7EE
:10132000099840B3FFE70A98006841F60001C4F24B
:101330000001884207D1FFE70998E0B1FFE709986B
:10134000042818D0FFE70A98006841F60041C4F26B
:101350000001884203D1FFE7099860B1FFE70A98CE
:10136000006842F20001C4F20001884204D1FFE7A4
:10137000099808B9FFE708E045F29E30C0F6020080
:1013800040F294510CF05EFAFFE7099828B9FFE7A4
:101390000A9890F83E0007901CE00998042805D1AF
:1013A000FFE70A9890F83F00069010E00998082897
:1013B00005D1FFE70A9890F84000059004E00A98EC
:1013C00090F841000590FFE705980690FFE7069822
:1013D0000790FFE70798012804D0FFE701208DF868
:1013E0002F00AFE0099828B9FFE70A99022081F899
:1013F0003E001EE00998042806D1FFE70A99022062
:1014000081F83F00049012E00998082806D1FFE710
:101410000A99022081F84000039005E00A99022011
:1014200081F841000390FFE703980490FFE70498D8
:10143000FFE70A98006809990122019206F080F8F6
:1014400001980A9909680022C4F2010291420290AF
:101450000CD0FFE70A9800684FF60041CBF6FE710A
:101460000844B0FA80F040090290FFE70298C007F4
:1014700038B1FFE70A980168486C40F400404864BE
:10148000FFE70A9800680021C4F2010188423CD0BD
:10149000FFE70A980068B0F1804F36D0FFE70A985E
:1014A000006840F20041C4F2000188422DD0FFE7FD
:1014B0000A98006840F60001C4F20001884224D076
:1014C000FFE70A98006840F60041C4F20001884234
:1014D0001BD0FFE70A98006840F20041C4F2010106
:1014E000884212D0FFE70A98006844F20001C4F273
:1014F0000101884209D0FFE70A98006841F600011F
:10150000C4F20001884212D1FFE70A98006880689F
:1015100000F0070008900898062807D0FFE70A980F
:101520000168086840F001000860FFE706E00A98DB
:101530000168086840F001000860FFE700208DF8AE
:101540002F00FFE79DF82F000CB080BD80B586B05E
:1015500005900491059800680021C4F201018842B9
:1015600014D1FFE70498002800F0E780FFE7049813
:10157000042800F0E280FFE70498082800F0DD80EE
:10158000FFE704980C2800F0D880FFE70598006872
:10159000B0F1804F14D1FFE70498002800F0CD800F
:1015A000FFE70498042800F0C880FFE704980828A3
:1015B00000F0C380FFE704980C2800F0BE80FFE72E
:1015C0000598006840F20041C4F20001884214D13D
:1015D000FFE70498002800F0B080FFE70498042893
:1015E00000F0AB80FFE70498082800F0A680FFE732
:1015F00004980C2800F0A180FFE70598006840F6E9
:101600000001C4F20001884214D1FFE704980028C9
:1016100000F09380FFE70498042800F08E80FFE735
:101620000498082800F08980FFE704980C2800F04F
:101630008480FFE70598006840F60041C4F200018D
:10164000884210D1FFE70498002876D0FFE704987D
:10165000042872D0FFE7049808286ED0FFE70498AA
:101660000C286AD0FFE70598006840F20041C4F2F8
:101670000101884210D1FFE7049800285DD0FFE700
:101680000498042859D0FFE70498082855D0FFE7AC
:1016900004980C2851D0FFE70598006844F2000137
:1016A000C4F20101884208D1FFE70498002844D021
:1016B000FFE70498042840D0FFE70598006844F24B
:1016C0000041C4F20101884203D1FFE70498A0B3AE
:1016D000FFE70598006844F60001C4F20101884262
:1016E00003D1FFE7049840B3FFE70598006841F68F
:1016F0000001C4F20001884207D1FFE70498E0B17D
:10170000FFE70498042818D0FFE70598006841F621
:101710000041C4F20001884203D1FFE7049860B1A0
:10172000FFE70598006842F20001C4F20001884218
:1017300004D1FFE7049808B9FFE708E045F29E30BE
:10174000C0F602004FF4B9610CF07CF8FFE7059891
:1017500000680499002205F0F3FE05980168012055
:101760000022C4F20102914203900CD0FFE70598D9
:1017700000684FF60041CBF6FE710844B0FA80F0E5
:1017800040090390FFE70398C007D8B1FFE7FFE7E0
:1017900005980068006A41F21111084210D1FFE774
:1017A00005980068006A40F24441084207D1FFE70B
:1017B00005980168486C20F400404864FFE7FFE7A3
:1017C000FFE7FFE7FFE705980068006A41F21111A3
:1017D000084210D1FFE705980068006A40F24441D2
:1017E000084207D1FFE705980168086820F001006A
:1017F0000860FFE7FFE7FFE7049828B9FFE70599CE
:10180000012081F83E001EE00498042806D1FFE77D
:101810000599012081F83F00029012E00498082801
:1018200006D1FFE70599012081F84000019005E00D
:101830000599012081F841000190FFE7019802908D
:10184000FFE70298FFE7002006B080BD81B000905E
:101850000098006841F20041C4F20001884208D1BA
:10186000FFE741F6C831C2F20001086801300860A4
:10187000FFE701B07047000081B0009001B07047F1
:1018800082B00190ADF8021002B0704780B582B00E
:101890000190019807F0BEFE8DF803009DF803004B
:1018A00004281BD0FFE79DF8030000EBC00140F2C5
:1018B000C040C2F2000000EB8100C06968B1FFE7E0
:1018C0009DF8030000EBC00140F2C040C2F20000EE
:1018D00000EB8100C0698047FFE7FFE702B080BDF1
:1018E00080B582B0019001980168C86820F49070BA
:1018F000C86001980168486920F0010048610198BA
:10190000006B012807D1FFE701980168C86820F043
:101910001000C860FFE70198006840694006002891
:101920002BD5FFE701980168486920F04000486125
:101930000198806B98B1FFE70198816B49F20150E3
:10194000C0F6010008650198806BF8F759FB28B1D3
:10195000FFE70198806B016D8847FFE70CE0019974
:101960000020C885019A202182F83E100199086361
:101970000198FFF78BFFFFE70CE001990020C88575
:10198000019A202182F83E10019908630198FFF71F
:101990007DFFFFE7002002B080BD000080B582B06F
:1019A0000190019807F036FE8DF803009DF80300C2
:1019B00004281BD0FFE79DF8030000EBC00140F2B4
:1019C000C040C2F2000000EB8100006968B1FFE78F
:1019D0009DF8030000EBC00140F2C040C2F20000DD
:1019E00000EB810000698047FFE7FFE702B080BDA0
:1019F00080B588B00790079800680068069007983F
:101A00000068C0680590079800684069049000204D
:101A100003900290069800F00F000390039888B995
:101A2000FFE79DF81800800600280AD5FFE79DF81B
:101A300014008006002804D5FFE7079807F01CFE75
:101A400078E1FFE70398002800F0B480FFE79DF8F5
:101A50001000C00738B9FFE7BDF8140010F4907FFC
:101A600000F0A880FFE79DF81800C00758B1FFE715
:101A70009DF81500C00730B1FFE70799086C40F0EA
:101A800001000864FFE79DF81800400700280BD507
:101A9000FFE79DF81000C00730B1FFE70799086C19
:101AA00040F002000864FFE79DF818008007002856
:101AB0000BD5FFE79DF81000C00730B1FFE707998D
:101AC000086C40F004000864FFE79DF81800000768
:101AD000002811D5FFE79DF814008006002805D4E2
:101AE000FFE79DF81000C00730B1FFE70799086CC9
:101AF00040F008000864FFE70798006C002858D001
:101B0000FFE79DF81800800600280AD5FFE79DF83A
:101B100014008006002804D5FFE7079807F0ACFD05
:101B2000FFE7079800684069C0F3801002900798AB
:101B3000006C0007002803D4FFE7029888B3FFE792
:101B4000079807F021FD07980068406940060028C3
:101B500022D5FFE707980168486920F040004861F6
:101B60000798806B98B1FFE70798816B49F2AD3019
:101B7000C0F6010008650798806BF8F741FA28B1B4
:101B8000FFE70798806B016D8847FFE703E0079840
:101B9000FFF704FFFFE703E00798FFF7FFFEFFE70B
:101BA00006E00798FFF7FAFE079900200864FFE7B0
:101BB000FFE7BFE00798006B012840F09B80FFE73C
:101BC0009DF81800C006002840F19480FFE79DF8BA
:101BD0001400C006002840F18D80FFE7FFE70020D9
:101BE00001900798006800680190079800684068B5
:101BF00001900198FFE707980068406940060028B7
